:100000000C94A00F0C94D10F0C94D10F0C94D10F21
:100010000C94D10F0C94D10F0C94D10F0C94D10FE0
:100020000C94D10F0C94D10F0C94D10F0C94D10FD0
:100030000C94D10F0C94F9AD0C94D10F0C94D10FFA
:100040000C94D10F0C94D28C0C94D10F0C94D10F32
:100050000C94D10F0C94D10F0C94B4260C94BFA91E
:100060000C94D10F0C94DD890C94D10F0C94D10F0A
:100070000C94D10F0C94D10F0C94D10F0C94D10F80
:100080000C94D10F0C94D10F0C94D10F0C94D10F70
:100090000C94D10F0C94D10F0C94D10F0C94F1A6A9
:1000A0000C94D10F0C94D10F0C94D10F0C94D10F50
:1000B0000C94D10F0C94D10F0C94D10F0C94D10F40
:1000C0000C94D10F0C94D10F0C94D10F0C94D10F30
:1000D0000C94D10F0C94D10F0C94D10F0C94D10F20
:1000E0000C94D10F01270F272B273927532761277E
:1000F0007B277F27812785278D2743A848A84DA8E0
:1001000057A8D0A861A869A871A87BA885A88FA8BE
:100110009EA8A8A8D0A8B2A8BCA8C6A8EEA8F1A876
:10012000E4A8E8A828A9F5A8F9A8FFA803A907A9A1
:100130000DA911A915A928A91BA91FA923A9084A16
:10014000D73B3BCE016E84BCBFFDC12F3D6C7431EB
:100150009ABD56833DDA3D00C77F11BED9E4BB4C42
:100160003E916BAAAABE000000803F05A84CCDB20C
:10017000D44EB93836A9020C50B9918688083CA6ED
:10018000AAAA2ABE000000803F007C3C3E5E2B3DB8
:100190003F2F5B5D3B2C2A225C004572723A204D5A
:1001A000415854454D50204245440054656D70659A
:1001B000726174757265206865617465642062653A
:1001C00064207377697463686564206F66662E20A7
:1001D0004D415854454D502074726967676572658A
:1001E00064202121004572723A204D494E54454DFC
:1001F00050003A204578747275646572207377698F
:100200007463686564206F66662E204D494E5445C0
:100210004D502074726967676572656420210045DE
:1002200072723A204D415854454D50003A2045785D
:10023000747275646572207377697463686564208D
:100240006F66662E204D415854454D50207472699A
:10025000676765726564202100202D20496E7661F4
:100260006C6964206578747275646572206E756D52
:10027000626572202100504944204175746F747585
:100280006E652066696E69736865642120507574B7
:1002900020746865206C617374204B702C204B694E
:1002A00020616E64204B6420636F6E7374616E74A2
:1002B000732066726F6D2061626F766520696E745F
:1002C0006F20436F6E66696775726174696F6E2E19
:1002D0006800504944204175746F74756E652066DE
:1002E00061696C6564212074696D656F75740020A7
:1002F000403A006F6B20543A006F6B20423A005036
:100300004944204175746F74756E65206661696C2F
:100310006564212054656D70657261747572652025
:10032000746F6F206869676800204B643A20002072
:100330004B693A2000204B703A200020436C6173D7
:100340007369632050494420002054753A200020EE
:100350004B753A2000206D61783A2000206D696E5F
:100360003A200020643A200020626961733A20003C
:100370001000C90210012C01400122017001180176
:10038000B0010E01F00104015002FA00B002F000C9
:100390003003E600D003DC009004D2007005C800F2
:1003A000A006BE000008B400B009AA00D00BA0004F
:1003B000600E960060118C000015820020197800F4
:1003C000C01D6E00A0226400B0275A00902C50007F
:1003D00000314600E0343C0010383200903A2800EA
:1003E000603C1E00A03D1400803E0A00203F00003B
:1003F00070012C0190012701B0012201C0011D01F3
:10040000F00118011002130130020E01600209010F
:1004100090020401C002FF000003FA004003F5004F
:100420008003F000D003EB002004E6007004E1003C
:10043000E004DC004005D700C005D2004006CD0036
:10044000D006C8008007C3003008BE00F008B9001D
:10045000C009B400B00AAF00B00BAA00D00CA500D0
:10046000000EA000500F9B00C0109600501291008B
:1004700000148C00C0158700B0178200B0197D00F1
:10048000D01B7800001E730040206E00902269008F
:10049000F024640040275F0090295A00E02B5500AB
:1004A000102E500020304B0010324600E033410047
:1004B00090353C001037370070383200A0392D00DD
:1004C000B03A2800A03B2300603C1E00103D1900FC
:1004D000903D1400103E0F00703E0A00C03E050023
:1004E000003F00004D383420582059205A20450044
:1004F00043616E6E6F7420656E74657220737562F1
:100500006469723A20004D3234004D323320257335
:10051000006175746F25692E67006572726F7220B5
:1005200077726974696E6720746F2066696C650004
:100530004E6F74207072696E74696E67000A002FC6
:10054000005344207072696E74696E67206279741A
:100550006520000A002E0044656C6574696F6E208A
:100560006661696C65642C2046696C653A200046BA
:10057000696C652064656C657465643A002E006F73
:1005800070656E206661696C65642C2046696C65D7
:100590003A200057726974696E6720746F2066692B
:1005A0006C653A20002E006F70656E206661696C84
:1005B00065642C2046696C653A20002E006F7065DA
:1005C0006E206661696C65642C2046696C653A2012
:1005D0000046696C652073656C6563746564002012
:1005E00053697A653A200046696C65206F70656EC4
:1005F00065643A20002E006F70656E206661696C3C
:1006000065642C2046696C653A20004E6F77206641
:10061000726573682066696C653A20004E6F7720BA
:10062000646F696E672066696C653A2000222070ED
:100630006F73002220706172656E743A2200535508
:1006400042524F5554494E452043414C4C20746111
:10065000726765743A2200747279696E6720746FEC
:100660002063616C6C207375622D67636F64652015
:1006700066696C6573207769746820746F6F206D8C
:10068000616E79206C6576656C732E204D41582023
:100690006C6576656C2069733A005344206361721F
:1006A00064206F6B006F70656E526F6F74206661AF
:1006B000696C656400766F6C756D652E696E697422
:1006C000206661696C656400534420696E6974201A
:1006D0006661696C0000002110422063308440A5EF
:1006E00050C660E770088129914AA16BB18CC1ADF9
:1006F000D1CEE1EFF13112100273325222B5529491
:1007000042F772D662399318837BB35AA3BDD39C48
:10071000C3FFF3DEE36224433420040114E664C71C
:1007200074A44485546AA54BB528850995EEE5CF98
:10073000F5ACC58DD55336722611163006D776F630
:10074000669556B4465BB77AA719973887DFF7FEE8
:10075000E79DD7BCC7C448E5588668A778400861BC
:100760001802282338CCC9EDD98EE9AFF948896938
:10077000990AA92BB9F55AD44AB77A966A711A50D0
:100780000A333A122AFDDBDCCBBFFB9EEB799B5888
:100790008B3BBB1AABA66C877CE44CC55C222C035C
:1007A0003C600C411CAEED8FFDECCDCDDD2AAD0BD8
:1007B000BD688D499D977EB66ED55EF44E133E3270
:1007C0002E511E700E9FFFBEEFDDDFFCCF1BBF3A28
:1007D000AF599F788F8891A981CAB1EBA10CD12D17
:1007E000C14EF16FE18010A100C230E3200450251A
:1007F0004046706760B9839893FBA3DAB33DC31C8E
:10080000D37FE35EF3B1029012F322D23235421469
:100810005277625672EAB5CBA5A89589856EF54FD9
:10082000E52CD50DC5E234C324A0148104667447B9
:100830006424540544DBA7FAB79987B8975FE77E2D
:10084000F71DC73CD7D326F2369106B01657667609
:1008500076154634564CD96DC90EF92FE9C899E979
:10086000898AB9ABA94458654806782768C018E159
:10087000088238A3287DCB5CDB3FEB1EFBF98BD8CD
:100880009BBBAB9ABB754A545A376A167AF10AD0A9
:100890001AB32A923A2EFD0FED6CDD4DCDAABD8B19
:1008A000ADE89DC98D267C076C645C454CA23C83F9
:1008B0002CE01CC10C1FEF3EFF5DCF7CDF9BAFBA6D
:1008C000BFD98FF89F176E367E554E745E932EB249
:1008D0003ED10EF01E53544F505045442E20005030
:1008E00072696E7465722073746F707065642064D1
:1008F000756520746F206572726F72732E20466961
:100900007820746865206572726F7220616E642051
:10091000757365204D39393920746F207265737491
:100920006172742E202854656D70657261747572E1
:10093000652069732072657365742E205365742079
:100940006974206166746572207265737461727473
:10095000696E6729004B494C4C45442E200050726B
:10096000696E7465722068616C7465642E206B69B1
:100970006C6C28292063616C6C656421006F6B00CE
:10098000526573656E643A20002200556E6B6E6F7F
:10099000776E20636F6D6D616E643A2022004D3278
:1009A000323020532569005A204F666673657420E3
:1009B0003A20007A5F6D61783A20007A5F6D696E47
:1009C0003A20005A204F6666736574005A204F66BD
:1009D00066736574206F6B002200556E6B6E6F77C7
:1009E0006E20636F6D6D616E643A2022007A5F6DD8
:1009F00061783A20007A5F6D696E3A2000795F6D08
:100A000061783A2000795F6D696E3A2000785F6DF9
:100A100061783A2000785F6D696E3A2000205A3A7A
:100A20000020593A0020436F756E7420583A200018
:100A300020453A00205A3A0020593A00583A0046D8
:100A400049524D574152455F4E414D453A4D6172B5
:100A50006C696E2056312E302E323B2053707269F5
:100A60006E7465722F6772626C206D617368757049
:100A700020666F722067656E36204649524D574199
:100A800052455F55524C3A68747470733A2F2F6711
:100A900069746875622E636F6D2F4D61726C696E3B
:100AA0004669726D776172652F4D61726C696E2057
:100AB00050524F544F434F4C5F56455253494F4E3F
:100AC0003A312E30204D414348494E455F545950EC
:100AD000453A507275736120693320455854525518
:100AE0004445525F434F554E543A31205555494481
:100AF0003A30303030303030302D303030302D30F2
:100B00003030302D303030302D30303030303030EB
:100B100030303030300A00507275736120693320F4
:100B20004F66662E005072757361206933207072B3
:100B30006970726176656E6100426564204F4B2E6C
:100B40000020423A0020453A00543A005A61687247
:100B50006976616E69206265642E2E2E005A616886
:100B6000726976616E69204F4B2E0020573A002043
:100B7000453A00543A005A6168726976616E692E8E
:100B80002E2E002042403A0020403A00202F003A0A
:100B900000205400202F0020423A00202F006F6BCD
:100BA00020543A002569206D696E2C202569207338
:100BB000656300456E642066696C65206C697374BA
:100BC00000426567696E2066696C65206C697374A4
:100BD000004E6F206D6F76652E0050727573612028
:100BE00069332070726970726176656E61004F6260
:100BF0006E6F76656E69207469736B7500576169F5
:100C00007420666F7220757365722E2E2E00536CE1
:100C10006565702E2E2E00256920686F7572732011
:100C20002569206D696E7574657300446F6E65206B
:100C30007072696E74696E672066696C65005354E2
:100C40004F505045442E20005072696E74657220DA
:100C500073746F707065642064756520746F2065AF
:100C600072726F72732E20466978207468652065F1
:100C700072726F7220616E6420757365204D393910
:100C80003920746F20726573746172742E20285439
:100C9000656D706572617475726520697320726527
:100CA0007365742E205365742069742061667465C1
:100CB000722072657374617274696E6729004E6F79
:100CC000204C696E65204E756D626572207769747F
:100CD0006820636865636B73756D2C204C61737459
:100CE000204C696E653A20004E6F20436865636B47
:100CF00073756D2077697468206C696E65206E75F8
:100D00006D6265722C204C617374204C696E653A7B
:100D10002000636865636B73756D206D69736D6129
:100D20007463682C204C617374204C696E653A20A2
:100D3000004C696E65204E756D6265722069732086
:100D40006E6F74204C617374204C696E65204E7513
:100D50006D6265722B312C204C617374204C696E6E
:100D6000653A20004D31313000446F6E652073616B
:100D700076696E672066696C652E006F6B004D3278
:100D800039002020506C616E6E6572427566666532
:100D90007242797465733A20002046726565204D71
:100DA000656D6F72793A20004A616E2032362032CA
:100DB00030313600436F6D70696C65643A200028ED
:100DC0006E6F6E652C2064656661756C7420636F50
:100DD0006E6669672900207C20417574686F723ADD
:100DE00020004A616E2032362032303136203139CF
:100DF0003A33363A313600204C61737420557064B2
:100E0000617465643A2000312E302E32004D6172DB
:100E10006C696E0020536F6674776172652052654D
:100E200073657400205761746368646F672052654E
:100E3000736574002042726F776E206F7574205254
:100E400065736574002045787465726E616C20521C
:100E50006573657400506F776572557000737461C7
:100E60007274002200656E717565696E67202200DC
:100E70002200656E717565696E67202200FFFFFFB5
:100E80000000A0400000A0400000004000005643C9
:100E9000000046431FC5484300000000000000005A
:100EA0001F856B3E00005643000046430000494347
:100EB00000000000000000001F856B3E6563686F46
:100EC0003A004572726F723A004B6172746120761B
:100ED000796A6D757461004B6172746120766C6F14
:100EE0007A656E610047312045343020463130301C
:100EF000004731204537302046343030004D3833FC
:100F000000473120452D38302046343030004D38F0
:100F100033002D2D3A2D2D002D2D2D005344000191
:100F200020000120004D3630300056796D656E6925
:100F3000742066696C616D656E7400507275746FB3
:100F40006B00507275746F6B00527963686C6F73CD
:100F5000742076656E742E00527963686C6F7374BA
:100F60002076656E742E004265640042656400540C
:100F70007279736B6100547279736B61005279639B
:100F8000686C6F737400527963686C6F7374004897
:100F90006C61766E69206E616269646B61005A6390
:100FA000686C6164697400464C4558202D202032DD
:100FB00033302F35300050502020202D2020323566
:100FC000342F3130300048495053202D2020323208
:100FD000302F3130300050455420202D2020323425
:100FE000302F393000504C4120202D20203231301C
:100FF0002F35300041425320202D20203235352F0F
:1010000031303000486C61766E69206E61626964CF
:101010006B61004D3834004D383420582059205A27
:101020002045004D3234004D323320257300052E0B
:101030002E00486C61766E69206E616269646B6136
:1010400000527963686C6F73742076656E742E003D
:10105000527963686C6F73742076656E742E0042EB
:1010600065640042656400547279736B6100547268
:1010700079736B61004E6173746176656E690058B7
:101080000059005A0045787472756465720045789D
:1010900074727564657200506F73756E6F7574202D
:1010A0005A00506F73756E6F7574205900506F73CE
:1010B000756E6F75742058004E6173746176656E3D
:1010C0006900473238004175746F20686F6D6500A4
:1010D0004D3834005679706E6F7574206D6F746F73
:1010E000727900473238205A004B616C6962726F26
:1010F000766174205A00506F73756E6F7574206F2F
:101100007375005465706C6F746100486C61766E25
:1011100069206E616269646B61005265763A2031C4
:1011200037352D316200686F77746F2E707275736A
:101130006133642E636F6D00666F72756D2E707211
:1011400075736133642E636F6D00707275736133F4
:10115000642E636F6D004669726D77617265202D34
:1011600020322E322E3200486C61766E69206E611C
:101170006269646B6100506F64706F7261004E61F0
:1011800073746176656E690056796A6D6F75742047
:1011900066696C616D656E74005A61766573742062
:1011A00066696C616D656E74005A61646E6120538E
:1011B00044206B61727461005469736B207A205310
:1011C00044005A61737461766974207469736B00AA
:1011D000506F6B7261636F76617400506F7A6173E8
:1011E0007461766974207469736B0050726564650C
:1011F00068726576004C6164697400496E666F724E
:101200006D6163650048617264636F646564204466
:10121000656661756C742053657474696E677320BC
:101220004C6F616465640046696C616D656E742025
:1012300073657474696E67733A2044697361626C94
:101240006564002020204D32303020440046696C17
:10125000616D656E742073657474696E67733A00AE
:101260002020204D3230392053004175746F2D52AB
:101270006574726163743A20533D3020746F20644A
:10128000697361626C652C203120746F20696E7403
:1012900065727072657420657874727564652D6FFF
:1012A0006E6C79206D6F7665732061732072657442
:1012B0007261637473206F72207265636F766572FA
:1012C000696573002046002020204D3230382053BD
:1012D000005265636F7665723A20533D45787472AB
:1012E00061206C656E67746820286D6D2920463A10
:1012F000537065656420286D6D2F6D2900205A009C
:101300002046002020204D32303720530052657493
:10131000726163743A20533D4C656E67746820288F
:101320006D6D2920463A537065656420286D6D2FD8
:101330006D29205A3A205A4C69667420286D6D290F
:10134000002044002049002020204D33303120501F
:10135000005049442073657474696E67733A0020C5
:101360005A0020590020204D323036205800486F56
:101370006D65206F666673657420286D6D293A006F
:10138000204500205A002058002042002054002010
:10139000204D323035205300416476616E636564C0
:1013A000207661726961626C65733A20533D4D69C4
:1013B0006E20666565647261746520286D6D2F739B
:1013C000292C20543D4D696E2074726176656C2025
:1013D000666565647261746520286D6D2F73292CB4
:1013E00020423D6D696E696D756D207365676D6531
:1013F0006E742074696D6520286D73292C20583D0A
:101400006D6178696D756D205859206A65726B2021
:10141000286D6D2F73292C20205A3D6D6178696DE0
:10142000756D205A206A65726B20286D6D2F7329A7
:101430002C2020453D6D6178696D756D2045206AD1
:1014400065726B20286D6D2F7329002054002020B9
:101450004D323034205300416363656C65726174B2
:10146000696F6E3A20533D616363656C65726174A8
:10147000696F6E2C20543D726574726163742061D3
:101480006363656C65726174696F6E00204500204E
:101490005A0020590020204D3230312058004D6133
:1014A00078696D756D20416363656C6572617469FF
:1014B0006F6E20286D6D2F7332293A002045002071
:1014C0005A0020590020204D3230332058004D6101
:1014D00078696D756D2066656564726174657320E9
:1014E000286D6D2F73293A00204500205A0020599D
:1014F0000020204D393220580053746570732070DD
:10150000657220756E69743A0045303A20005A3A87
:101510002000593A2000583A20004D53312C4D53A9
:10152000322050696E730A00656E6473746F707355
:10153000206869743A205A00205A3A00656E647334
:10154000746F7073206869743A20590020593A000A
:10155000656E6473746F7073206869743A20580004
:1015600020583A00656E6473746F707320686974F4
:101570003A200024F4D43050C38E20C2A2401782F7
:101580008B7011127A910D816CD90AA861E108C79C
:10159000586607615143061E4B5D05C145A7041AF5
:1015A000411104093D9803713931034036DB02656E
:1015B000339102D4305402802E1D02632CEE01754B
:1015C0002AC501B028A001102781018F2564012BB5
:1015D000244B01E0223401AC211F018D200D01803C
:1015E0001FFC00841EED00971DDF00B81CD200E632
:1015F0001BC600201BBC00641AB200B219A8000A66
:1016000019A0006A189900D117910040178B00B5F6
:1016100016840031167E00B31579003A157300C7A1
:10162000146F0058146A00EE1366008813630025D7
:10163000135E00C7125B006C12570015125400C1F4
:1016400011510070114F0021114B00D61049008D2F
:101650001047004610440002104200C00F400080B6
:101660000F3E00420F3C00060F3B00CB0E380093AC
:101670000E37005C0E3500270E3400F30D3200C12A
:101680000D3100900D3000600D2E00320D2D000543
:101690000D2C00D90C2B00AE0C2900850C29005C08
:1016A0000C2700350C27000E0C2600E80B2400C484
:1016B0000B2400A00B23007D0B23005A0B210039C3
:1016C0000B2100180B2000F80A1F00D90A1E00BBCE
:1016D0000A1E009D0A1D00800A1D00630A1C0047A7
:1016E0000A1B002C0A1B00110A1A00F7091A00DD58
:1016F000091900C4091900AB091900920917007BE8
:10170000091800630917004C091600360916002055
:101710000916000A091500F5081500E0081400CCA8
:10172000081400B8081400A4081400900813007DE1
:101730000812006B08130058081200460812003403
:10174000081100230811001208110001081100F00F
:10175000071000E0071000D0071000C0071000B00D
:10176000070F00A107100091070E0083070F0074F8
:10177000070F0065070E0057070E0049070E003BD4
:10178000070D002E070E0020070D0013070D0006A1
:10179000070D00F9060C00ED060D00E0060C00D464
:1017A000060C00C8060C00BC060C00B0060C00A419
:1017B000060B0099060C008D060B0082060B0077C5
:1017C000060B006C060B0061060A0057060B004C66
:1017D000060A0042060A0038060A002E060A0024FD
:1017E000060A001A060A001006090007060A00FD8C
:1017F000050900F4050900EB050900E2050900D917
:10180000050900D0050900C7050900BE050900B596
:10181000050800AD050800A50509009C0508009411
:101820000508008C050800840508007C0508007484
:101830000508006C050700650508005D05070056F2
:101840000508004E05070047050700400508003859
:10185000050700310507002A050700230507001CBE
:10186000050600160507000F05070008050600021B
:10187000050700FB040600F5040700EE040600E877
:10188000040600E2040700DB040600D5040600CFCE
:10189000040600C9040600C3040600BD040600B720
:1018A000040600B1040500AC040600A6040600A06E
:1018B0000405009B04060095040500900406008AB8
:1018C00004050085040500800406007A04050075FF
:1018D000040500700405006B040500660405006142
:1018E0000405005C04050057040500520405004D82
:1018F00004050048040500430405003E0404003AC2
:1019000004050035040500300404002C04050027FC
:10191000040400230405001E0404001A0404001635
:10192000040500110404000D04040009040500046A
:1019300004040000040400FC030400F8030400F4A1
:10194000030400F0030400EC030400E8030400E4D3
:10195000030400E0030400DC030400D8030400D403
:10196000030400D0030400CC030400C8030300C533
:1019700003030024F404D9201BC40C5C0E9804C497
:10198000095F0265077101F405F900FB04B3004823
:10199000048700C10369005803550003034500BED6
:1019A000023A008402310053022A00290225000471
:1019B000022000E4011C00C8011900AF01170098C3
:1019C0000114008401130071011000610110005125
:1019D000010E0043010D0036010B002B010B00200E
:1019E000010B00150109000C01090003010800FBAF
:1019F000000800F3000800EB000700E4000600DE2A
:101A0000000600D8000600D2000600CC000500C782
:101A1000000500C2000500BD000400B9000400B5C7
:101A2000000400B1000400AD000400A9000400A5FA
:101A3000000300A20003009F0004009B0003009825
:101A40000003009500020093000300900003008D46
:101A50000002008B00030088000200860002008460
:101A6000000300810002007F0002007D0002007B75
:101A70000002007900020077000100760002007485
:101A800000020072000100710002006F0002006D90
:101A90000001006C0002006A00010069000200679A
:101AA00000010066000100650001006400020062A0
:101AB00000010061000100600001005F0002005DA4
:101AC0000001005C0001005B0001005A00010059A8
:101AD00000010058000100570001005600010055A8
:101AE00000010054000100530000005300010052A7
:101AF00000010051000100500001004F0001004EA4
:101B00000000004E0001004D0001004C0001004BA0
:101B10000000004B0001004A00010049000100489C
:101B20000000004800010047000100460000004698
:101B30000001004500000045000100440001004391
:101B4000000000430001004200000042000100418B
:101B500000000041000100400001003F0000003F84
:101B60000001003E0000003E0001003D0000003D7D
:101B70000001003C0000003C0000003C0001003B74
:101B80000000003B0001003A0000003A000100396B
:101B90000000003900010038000000380000003863
:101BA0000001003700000037000100360000003659
:101BB000000000360001003500000035000000354F
:101BC0000001003400000034000000340001003344
:101BD000000000330000003300010032000000323A
:101BE000000000320001003100000031000000312F
:101BF0000001003000000030000000300001002F24
:101C00000000002F0000002F0000002F0001002E18
:101C10000000002E0000002E0001002D0000002D0D
:101C20000000002D0000002D0001002C0000002C01
:101C30000000002C0000002C0001002B0000002BF5
:101C40000000002B0000002B0001002A0000002AE9
:101C50000000002A0000002A0001002900000029DD
:101C600000000029000000290000002900010028D0
:101C700000000028000000280000002800000028C4
:101C800000010027000000270000002700000027B7
:101C900000000027000100260000002600000026AA
:101CA000000000260000002600010025000000259D
:101CB0000000002500000025000000250000002590
:101CC0000001002400000024000000240000002483
:101CD0000000002400010023000000230000002376
:101CE0000000002300000023000000230000002368
:101CF000000100220000002200000022000000225B
:101D0000000000220000002200010021000000214C
:101D1000000000210000002100000021000000213F
:101D20000000002100010020000000200000002031
:101D30000000002000000020000000200000002023
:101D4000000000200001001F0000001F0000001F15
:101D50000000001F0000001F0000001F0000001F07
:101D60000001001E0000001E0000001E0000001EFA
:101D700000000020746F6F206C6F6E6720657874B0
:101D8000727573696F6E2070726576656E746564C6
:101D90000020636F6C6420657874727573696F6E70
:101DA0002070726576656E746564000000090A0231
:101DB000080B0C0D070603040100000000000000E2
:101DC0000000000000000000000000000000000013
:101DD0000000000000000011100F000000000000D3
:101DE00000000000000000000000000000000000F3
:101DF00000000000000000000000000000000000E3
:101E0000000102102020080810204010204080020D
:101E10000102010804020101020408102040808030
:101E200040201008040201800402018040201008B4
:101E3000040201080402010102040810204080018C
:101E4000020408102040801008040880102040047C
:101E50004080102040048005050505070508080896
:101E600008020202020A0A0808040404040101012B
:101E70000101010101030303030303030304070733
:101E8000070C0C0C0C0C0C0C0C02020202060606D1
:101E900006060606060B0B0B0B0B0B0B0B07070AB4
:101EA0000A0A0A0A0A0505050404040808000020B5
:101EB000002300260029002C002F00320000010022
:101EC0000003010601090100002200250028002B63
:101ED000002E003100340002010000050108010B52
:101EE0000100002100240027002A002D00300033CB
:101EF0000001010000040107010A01024E414E49A0
:101F00004E495459494E46CDCCCC3D0AD7233C17B7
:101F1000B7D13877CC2B329595E6241FB14F0A0004
:101F20000020410000C84200401C4620BCBE4CCAF4
:101F30001B0E5AAEC59D7400AD64D17EC5A6B164BA
:101F400011241FBECFEFD1E2DEBFCDBF00E00CBF3A
:101F500015E0A0E0B2E0E2E1F4E701E00BBF02C06F
:101F600007900D92A03EB107D9F724E1A0EEB5E0AD
:101F700001C01D92AB3BB207E1F71FE1CEE3DFE109
:101F800000E006C022970109FE010BBF0E94B0B31A
:101F9000C833D10780E00807A9F70E94C9AA0C94AA
:101FA000F8B90C940000CF93DF93EC019C012C5FF7
:101FB0003F4F41E050E060E070E0898D9A8D0E94D3
:101FC000751A882399F04D895E896F89788D452B24
:101FD000462B472B59F44C815D816E817F814D8B5F
:101FE0005E8B6F8B788F998190689983DF91CF9109
:101FF0000895CF92DF92EF92FF920F931F93CF93AA
:10200000DF93EC0189899A89AB89BC89803E9F4F17
:10201000AF41B10510F080E06BC0CE01C4DF882372
:10202000D1F30E948918182F8823A9F3E98DFA8D1E
:10203000CC80DD80EE80FF8032E0C31AD108E10859
:10204000F108058404C0CC0CDD1CEE1CFF1C0A94B6
:10205000D2F786859785A089B189C80ED91EEA1E58
:10206000FB1E81E08093E605C092E907D092EA0763
:10207000E092EB07F092EC0780E092E0E9EEF5E009
:10208000DF019C011D9221503040E1F701E0E98D14
:10209000FA8D8481081790F429EE35E0B701A60186
:1020A000400F511D611D711D8091E7059091E8055C
:1020B0000E940F3D8823E1F00F5FE9CFC12C82E041
:1020C000D82EE12CF12C058404C0CC0CDD1CEE1CB8
:1020D000FF1C0A94D2F749895A896B897C894C0D77
:1020E0005D1D6E1D7F1D498B5A8B6B8B7C8B812FE9
:1020F000DF91CF911F910F91FF90EF90DF90CF90E4
:102100000895CF93DF93EC0141E0611101C040E0FD
:102110006C857D858E859F850E94C918882341F036
:10212000888920E2829FC001112487519A4F02C002
:1021300080E090E0DF91CF91089530E020E04EE222
:10214000DC015C91503271F0383029F4FB01E20F70
:10215000F11D40832F5FFB01E20FF11DDC015C915B
:1021600050832F5F3F5F01963B3051F7FB01E20F39
:10217000F11D10820895CF93DF93EB01FC012381C1
:10218000211102C080E00EC02250223020F48FE2E4
:102190008883198206C060E0B4DF009799F3BE011E
:1021A000CCDF81E0DF91CF910895FB012BE030E29D
:1021B00031932150E9F7DC0190E027E03A2FEB2F33
:1021C0008D9181110AC0DA013C931196EC9381E064
:1021D000FB019081903239F525C08F32A1F38E3208
:1021E00019F0EAE8F1E008C02A30E1F098E02AE0CE
:1021F000E5CF31963817B1F034913111FACF291764
:1022000088F03FED380F3E3568F431E0390FFB01BF
:10221000E90FF11D9FE9980F9A3108F480528083ED
:10222000932FCCCF80E008950F931F93CF93DF932C
:10223000EC018B018B81882311F080E042C0FB010F
:102240008789803139F18032C1F783E08B83F801CF
:10225000428D538D648D758D4D8B5E8B6F8B788F1A
:102260009E012F5E3F4FC8010E948019882329F3E9
:102270001A8F098F81E089831C821D821E821F8232
:10228000188619861A861B861C861D861E861F8642
:10229000188A17C082E08B831D8A1E8A1F8A188EB7
:1022A000FB01408D518D60E070E095E0440F551FBB
:1022B000661F771F9A95D1F7498B5A8B6B8B7C8B56
:1022C000D7CFDF91CF911F910F9108952F923F9219
:1022D0004F925F926F927F928F929F92AF92BF9236
:1022E000CF92DF92EF92FF920F931F93CF93DF93E2
:1022F000EC015B016A018B81811103C08FEF9FEFBD
:10230000C7C0898180FFFACF49895A896B897C8946
:1023100088859985AA85BB852601612C712C8A0147
:102320009B01081B190B2A0B3B0B4016510662063A
:10233000730618F06A01C81AD90A76013E0124E032
:10234000620E711CE114F10409F476C048855985C8
:102350006A857B854A0181E098222B811A012B0135
:10236000E9E05694479437942794EA95D1F7898DFC
:102370009A8DFC01223049F4628D738D848D958D88
:10238000620D731D841D951D3CC0148111501221D6
:1023900081149104C1F4111116C0452B462B472B13
:1023A00049F48D899E89AF89B88D8C839D83AE83D6
:1023B000BF8309C04C815D816E817F81930121D7EC
:1023C000882309F49BCFE98DFA8D6C817D818E8104
:1023D0009F816250710981099109058404C0660FCB
:1023E000771F881F991F0A94D2F726853785408961
:1023F0005189620F731F841F951F610F711D811D0D
:10240000911D20E032E02819390987012E153F057A
:1024100008F489010115F2E01F0769F52091E90729
:102420003091EA074091EB075091EC076217730770
:102430008407950719F41FC0C6012AC09501AB0196
:10244000BC018091E7059091E8050E949A3C8823A1
:1024500009F454CFA00EB11E88859985AA85BB8545
:10246000800F911FA11DB11D88879987AA87BB87FF
:10247000E01AF10A67CF40E08CD6882309F43ECFFA
:10248000B40167517A4FA801C5010E94CDB6E2CFD1
:10249000DF91CF911F910F91FF90EF90DF90CF9040
:1024A000BF90AF909F908F907F906F905F904F9074
:1024B0003F902F900895CF93DF931F92CDB7DEB753
:1024C00041E050E0BE016F5F7F4F00DF019719F4DC
:1024D000898190E002C08FEF9FEF0F90DF91CF9145
:1024E0000895CF92DF92EF92FF920F931F93CF93B5
:1024F000DF936C01EB017A01FC018381823060F093
:1025000000851185228533850F71112722273327F6
:10251000012B022B032B11F08FEF5CC041155105ED
:1025200011F0F70110821DE040E250E0BE01C6014B
:10253000CDDE8032910539F021E0892B09F420E0CD
:10254000822F819547C028812223C1F0253E61F367
:102550002E3251F33B853F733F3061F4E114F104B7
:1025600049F04A8D5B8D452B29F42F713FEF320FD7
:10257000343030F02B8523FDD7CF2CC080E02AC02B
:1025800030E021503109129FC001139F900D11249A
:10259000F701E80FF91F298120832B8121832D81E9
:1025A00022832F812383298524832E8525832889CF
:1025B00026832A8927832C8920872E892187288DA5
:1025C00022872C8D23872E8D2487288126FFD2CF2A
:1025D0001586D0CFDF91CF911F910F91FF90EF9093
:1025E000DF90CF9008951F93CF93DF93EC018B8101
:1025F000823018F480E090E023C0488559856A85D0
:102600007B85A5E07695679557954795AA95D1F76F
:10261000142F1F70CE014FDF97FDECCF48855985F1
:102620006A857B85415E5F4F6F4F7F4F4887598733
:102630006A877B8720E2129FC001112487519A4F3D
:10264000DF91CF911F9108954F925F926F927F9289
:10265000AF92BF92CF92DF92EF92FF920F931F93B0
:10266000CF93DF93EC016A017B012B81222349F098
:1026700089899A89AB89BC8984179507A607B7070A
:1026800010F480E06BC0223009F463C0C114D1049F
:10269000E104F10449F41C821D821E821F82188607
:1026A00019861A861B8659C088859985AA85BB8597
:1026B000E98DFA8DE585F0E03996AC01BD01415018
:1026C0005109610971090E2E04C0769567955795D9
:1026D00047950A94D2F79701860101501109210903
:1026E000310904C03695279517950795EA95D2F7D5
:1026F000041715072607370720F0892B8A2B8B2B09
:1027000049F48D899E89AF89B88D8C839D83AE8372
:10271000BF8304C0041B150B260B370B280139019E
:102720005E0184E0A80EB11C4114510461047104DF
:1027300081F04C815D816E817F819501898D9A8DBB
:1027400060D591E0491A5108610871088111ECCFF8
:1027500005C0C886D986EA86FB8681E0DF91CF91E5
:102760001F910F91FF90EF90DF90CF90BF90AF90AF
:102770007F906F905F904F9008950F931F93CF932A
:10278000DF93EC018B818823D1F1898187FF32C0EF
:1027900061E0CE01B6DC8C01009789F1FC018081FB
:1027A000853E69F18B81823040F449895A896B8971
:1027B0007C89448F558F668F778F4D895E896F89AD
:1027C000788DF801538F428F758B648BE091E00513
:1027D000F091E105309759F0B8016A5E7F4FC8016A
:1027E00048961995F801808D918D938B828B898104
:1027F0008F778983DF91CF911F910F918AC481E0F8
:10280000888380E0DF91CF911F910F910895CF933E
:10281000DF93EC01B2DF1B82DF91CF910895FC01C1
:1028200023812111F4CF08954F925F926F927F928E
:10283000AF92BF92CF92DF92EF92FF920F931F93CE
:10284000CF93DF9300D01F92CDB7DEB75C016A0152
:102850007B01FC0183818130E9F4818181FF1AC011
:10286000F50181899289A389B48984179507A60700
:10287000B70780F0892B8A2B8B2B09F472C0F501E6
:102880004084518462847384B701A601C501DCDEF3
:10289000811102C080E066C0F501818D928DC11466
:1028A000D104E104F10469F4458956896789708D82
:1028B00025D7882379F3F501158A168A178A108E91
:1028C00037C0F50144815581668177819E012F5F74
:1028D0003F4F97D48823F1F249815A816B817C81E3
:1028E000F501818D928DFC012789203139F4483F13
:1028F000FFEF5F0761057105D8F407C0483F2FEF70
:10290000520762072FE0720798F4F8D6882309F47B
:10291000C1CFF50144815581668177810FEF1FEFAB
:102920002FEF3FE0818D928D51D5882309F4B2CFEE
:10293000F501C18AD28AE38AF48A81818068818321
:10294000C5011BDF882309F4A5CFB701A6014C14EC
:102950005D046E047F0410F4B301A201C50174DEAE
:1029600001C081E00F900F900F900F90DF91CF91F9
:102970001F910F91FF90EF90DF90CF90BF90AF909D
:102980007F906F905F904F900895FF920F931F93E9
:10299000CF93DF93EC01F42E80E2689FF0011124C5
:1029A000E751FA4F8385817121F0842F827109F0FC
:1029B0004EC08091E9079091EA07A091EB07B09192
:1029C000EC078C879D87AE87BF87688B44895589C4
:1029D00060E070E0BA0155274427028D138D20E096
:1029E00030E0402B512B622B732B4D8B5E8B6F8B0A
:1029F000788F8385887151F4048D158D268D378DE0
:102A0000098B1A8B2B8B3C8B81E00BC08031F9F446
:102A10009E012F5E3F4F898D9A8D72D48823B9F025
:102A200084E08B838F2D8F7089831C821D821E8290
:102A30001F82188619861A861B86F4FE0BC040E09A
:102A400050E0BA01CE01F0DE811104C011C01B823A
:102A500080E00EC0F5FE0BC049895A896B897C89DC
:102A6000CE01DF91CF911F910F91FF90EDCD81E0CD
:102A7000DF91CF911F910F91FF900895AF92BF9278
:102A8000CF92DF92EF92FF920F931F93CF93DF933A
:102A90007C01EB016A01B22E898D9A8DF701928F2C
:102AA000818F40E050E0BA01CE01CEDDA12C088537
:102AB00019852A853B8589899A89AB89BC8908173C
:102AC00019072A073B07A0F585E036952795179546
:102AD00007958A95D1F70F70CE0185DD009709F42F
:102AE00081C0FC012081222311F0253EB9F4A11000
:102AF0000EC04091E9075091EA076091EB07709191
:102B0000EC07F7014487558766877787008BFC01C0
:102B10008081AA24A3948111CACF0AC04BE050E05F
:102B2000BC01C6010E94C0B6892B09F0C0CF58C0B5
:102B30008B2D8274823409F055C0AA2049F0F70128
:102B4000008961E0C701DDDAEC01009769F44AC051
:102B50008B81823009F446C0CE014BDA882309F418
:102B600041C0C9EED5E000E080E2FE0111928A95F5
:102B7000E9F78BE0F601DE0101900D928A95E1F70D
:102B8000E091E005F091E105309739F0BE01625F18
:102B90007F4FCE014096199508C081E298E2998B4B
:102BA000888B80E098E09F878E87888999899B8BA6
:102BB0008A8B998F888F8E859F859F8B8E8BA9D2CC
:102BC000882381F04B2D602FC701DF91CF911F919A
:102BD0000F91FF90EF90DF90CF90BF90AF90D5CE48
:102BE000B7FEF0CF80E0DF91CF911F910F91FF9062
:102BF000EF90DF90CF90BF90AF9008953F924F92AB
:102C00005F926F927F928F929F92AF92BF92CF927C
:102C1000DF92EF92FF920F931F93CF93DF93CDB785
:102C2000DEB7C354D1090FB6F894DEBF0FBECDBFD7
:102C30005C016B0124965FAF4EAF2497522E1C8E21
:102C40001F8E19821C826115710511F410E073C08A
:102C5000FC0183818111FACF2496EEADFFAD24975C
:102C600080818F3211F076011DC02496EEADFFAD4C
:102C7000249780818F3231F431962496FFAFEEAFE6
:102C80002497F3CFF60183818250823060F3F601FE
:102C9000618D728DCE010196C7DA8823B9F2CE011B
:102CA00001967C018E01045E1F4F3801FE013196B2
:102CB0004F01402E312E19C08823A9F121E0AE0129
:102CC000495C5F4FB701C801D9DE882309F4BECF44
:102CD000EC14FD0411F0C7019ADD0615170501F18A
:102CE000942D832D7801092F182FAE014E5B5F4F75
:102CF000BE01695C7F4F24968EAD9FAD249755DA57
:102D0000882309F4A3CF2496EEADFFAD24978081EC
:102D10008F3291F631962496FFAFEEAF2497F3CF22
:102D2000982D892DDFCF252DAE01495C5F4FB7016E
:102D3000C501A4DE182FCE01019671DDCE014C969F
:102D40006EDD812FCD5BDF4F0FB6F894DEBF0FBE77
:102D5000CDBFDF91CF911F910F91FF90EF90DF904A
:102D6000CF90BF90AF909F908F907F906F905F902B
:102D70004F903F900895CF93DF93EC0140E050E0F7
:102D8000BA0152DD882361F061E0CE01BAD9009723
:102D900039F025EEFC0120831B82DF91CF91B9C170
:102DA00080E0DF91CF9108951F93CF93DF93CDB74C
:102DB000DEB76B970FB6F894DEBF0FBECDBFAB0189
:102DC00019821C8222E0BC01CE01019617DF182F68
:102DD000882321F0CE010196CEDF182FCE01019677
:102DE0001EDD812F6B960FB6F894DEBF0FBECDBFF0
:102DF000DF91CF911F9108952F923F924F925F9252
:102E00006F927F928F929F92AF92BF92CF92DF92FA
:102E1000EF92FF920F931F93CF93DF9300D01F92F7
:102E20001F92CDB7DEB78C015B013A01DC0113962E
:102E30008C9113978130C1F411968C9181FF14C04D
:102E400082FF18C0F801418952896389748980859D
:102E50009185A285B38584179507A607B70751F01A
:102E6000C801F2DB811106C081E0F80180838FEF99
:102E70009FEF37C1630183C0D80159968D919C9112
:102E80005A97FC01F481F1501A012B0169E0569424
:102E90004794379427946A95D1F7F221FD834A012C
:102EA00021E09222FF2309F476C080E092E08819A5
:102EB000990976018C159D0508F47C01D801599675
:102EC000ED91FC915A9714962D903D904D905C9009
:102ED0001797B2E02B1A310841085108058404C045
:102EE000220C331C441C551C0A94D2F78685978506
:102EF000A089B189280E391E4A1E5B1EED812E0E57
:102F0000311C411C511CE114F2E0FF0609F089C09C
:102F10008091E9079091EA07A091EB07B091EC0747
:102F200082159305A405B50569F41092E6058FEFA7
:102F30009FEFDC018093E9079093EA07A093EB07EA
:102F4000B093EC079501B201A1018091E705909142
:102F5000E8050E940F3D882309F486CFF80180859B
:102F60009185A285B3858E0D9F1DA11DB11D808702
:102F70009187A287B387AE0CBF1CCE18DF08D8019B
:102F800018964D915D916D917C911B97C114D10460
:102F900009F072CF7AC08114910409F086CF14969B
:102FA0004D915D916D917C9117974115510561058A
:102FB000710559F455968D919D910D90BC91A02D60
:102FC0000097A105B10539F520C09E012F5F3F4F45
:102FD00018D1882309F448CF89819A81AB81BC81BB
:102FE000F801218D328DF9012789203139F4883F8C
:102FF000FFEF9F07A105B10540F40DC0883F2FEFFB
:103000009207A2072FE0B20730F0C8010E94D30F49
:1030100081114BCF29CFF80184839583A683B78391
:1030200044CF8114910411F5D80118964D915D910A
:103030006D917C911B9751968D919D910D90BC91B6
:10304000A02D481759076A077B0780F062D08823B4
:1030500009F40ACF81E08093E6052092E9073092D7
:10306000EA074092EB075092EC0707C041E0C2012B
:10307000B1018FD0882309F4F7CEA701B501C401AF
:1030800087519A4F0E94CDB669CF51968D919D91EF
:103090000D90BC91A02DF801218184179507A607FA
:1030A000B70738F4418B528B638B748B2068218374
:1030B0000CC08091E0059091E105892B31F06114FD
:1030C000710419F02068F8012183D80111968C91C0
:1030D00083FD02C0C30105C0C8014FDB8111FACFD7
:1030E000C3CE0F900F900F900F900F90DF91CF9164
:1030F0001F910F91FF90EF90DF90CF90BF90AF9016
:103100009F908F907F906F905F904F903F902F9007
:103110000895CF938091E6058823B9F14091E9079E
:103120005091EA076091EB077091EC0729EE35E0CA
:103130008091E7059091E8050E940F3DC82F81110D
:1031400002C0C0E023C04091E2055091E3056091C8
:10315000E4057091E505411551056105710591F092
:1031600029EE35E08091E7059091E8050E940F3D3A
:10317000882339F31092E2051092E3051092E405DA
:103180001092E5051092E60501C0C1E08C2FCF91A9
:103190000895CF92DF92EF92FF92CF936B017C0163
:1031A000C42F8091E9079091EA07A091EB07B091B5
:1031B000EC078C159D05AE05BF05C9F0AADF81118E
:1031C00002C080E018C029EE35E0B701A601809169
:1031D000E7059091E8050E949A3C882391F3C092FC
:1031E000E907D092EA07E092EB07F092EC0781E062
:1031F000C1118093E605CF91FF90EF90DF90CF90C3
:1032000008958F929F92AF92BF92CF92DF92EF92EA
:10321000FF920F931F93CF93DF93EC016A017B0121
:10322000890189859A85AB85BC850196A11DB11D53
:1032300084179507A607B70710F480E054C08F895C
:10324000803129F49927872F762F652F0BC0803284
:10325000A1F7CB01BA0127E09695879577956795F9
:103260002A95D1F78B889C88AD88BE88680D791D1A
:103270008A1D9B1D8090E9079090EA07A090EB07BC
:10328000B090EC07681579058A059B0581F48F8954
:10329000803191F4DD24EE24FF24F601EE0FFF1FB0
:1032A000E751FA4F80819181A0E0B0E016C040E084
:1032B00070DF8111ECCFC1CFE894C7F8DD24EE2494
:1032C000FF24F601EE0FFF1FEE0FFF1FE751FA4F2D
:1032D00080819181A281B381BF70F8018083918345
:1032E000A283B38381E0DF91CF911F910F91FF9073
:1032F000EF90DF90CF90BF90AF909F908F90089508
:103300004F925F926F927F92AF92BF92CF92DF9275
:10331000EF92FF920F931F93CF93DF9300D01F92F2
:10332000CDB7DEB78C0149835A836B837C83590107
:10333000C12CD12C7601412C42E0542E612C712CF1
:1033400049815A816B817C819E012F5F3F4FC8016B
:1033500058DF882341F1D301C201F801058404C07C
:10336000880F991FAA1FBB1F0A94D2F7C80ED91E37
:10337000EA1EFB1E49815A816B817C8187898031DD
:1033800039F481E0483F5F4F6105710538F4D8CFCB
:1033900081E0483F5F4F6F4F7F4090F2F501C08260
:1033A000D182E282F3820F900F900F900F90DF9105
:1033B000CF911F910F91FF90EF90DF90CF90BF9032
:1033C000AF907F906F905F904F9008954F925F9273
:1033D0006F927F928F929F92AF92BF92CF92DF9225
:1033E000EF92FF920F931F93CF93DF93EC014A016B
:1033F0005B0128013901423051056105710508F46E
:1034000062C049855A856B857C854F5F5F4F6F4FE2
:103410007F4F481559056A057B0508F454C08F890C
:10342000803129F4FF24EB2CDA2CC92C0CC080321B
:1034300009F049C07501640177E0F694E794D794E8
:10344000C7947A95D1F74B895C896D897E89C40EC2
:10345000D51EE61EF71E41E0C701B6019ADE88239D
:1034600091F19F89903159F49924AA24BB24F40145
:10347000EE0FFF1FE751FA4F5182408210C0E894CF
:1034800087F89924AA24BB24F401EE0FFF1FEE0F46
:10349000FF1FE751FA4F40825182628273829A89FC
:1034A000923090F04D815E816F8178854C0D5D1D6D
:1034B0006E1D7F1D4093E2055093E3056093E40584
:1034C0007093E50501C080E0DF91CF911F910F91CE
:1034D000FF90EF90DF90CF90BF90AF909F908F9034
:1034E0007F906F905F904F9008952F923F924F92F0
:1034F0005F926F927F928F929F92AF92BF92CF9284
:10350000DF92EF92FF920F931F93CF93DF93CDB78C
:10351000DEB72F970FB6F894DEBF0FBECDBF1C01EC
:103520004C875D876E877F873B872A87DC011996EA
:103530000D911D912D913C911C970F5F1F4F2F4FA7
:103540003F4F0D831E832F833887EA85FB8580805C
:103550009180A280B38081149104A104B10431F060
:10356000FFEF8F1A9F0AAF0ABF0A10C0DC018D90CF
:103570009D90AD90BC90B1E0B9870C851D852E85DE
:103580003F85013011052105310509F019867501C6
:103590006401412C512C3201F10181859285A38572
:1035A000B485481659066A067B0608F04EC00D81A0
:1035B0001E812F8138850C151D052E053F0550F401
:1035C000F2E0CF2ED12CE12CF12CA2E08A2E912C0E
:1035D000A12CB12C9E012F5F3F4FB701A601C10165
:1035E00010DE882391F149815A816B817C81D7015A
:1035F000C6010196A11DB11D452B462B472B19F085
:103600004C015D010FC0AC01BD01481959096A099F
:103610007B090C851D852E853F8540175107620764
:10362000730741F01FEF411A510A610A710A6C01D8
:103630007D01B2CF0FEF1FEF2FEF3FE0B701A601E3
:10364000C101C4DE8D83811113C01D823DC02601DE
:10365000370121E0421A510861087108970186017B
:10366000B301A201C101B2DE882379F373016201C3
:103670008C149D04AE04BF0450F3AA85BB854D9104
:103680005D916D917C914115510561057105A9F41C
:10369000EA85FB8580829182A282B382F985FF232D
:1036A00099F00FEF801A900AA00AB00AD1018D920A
:1036B0009D92AD92BC92139707C095018401C10100
:1036C00085DE8111E5CFC1CF8D812F960FB6F8949D
:1036D000DEBF0FBECDBFDF91CF911F910F91FF9045
:1036E000EF90DF90CF90BF90AF909F908F907F90A2
:1036F0006F905F904F903F902F900895AF92BF9240
:10370000CF92DF92EF92FF920F931F93CF93DF93AD
:1037100000D01F92CDB7DEB75C016A017B0182E069
:1037200090E0A0E0B0E0F50180839183A283B383B1
:103730009E012F5F3F4FB701A601C50162DD8111D8
:1037400002C080E023C000E010E09801B701A601AC
:10375000C5013CDE8823A9F3C980DA80EB80FC80B8
:10376000F5018789803149F481E0F8EFCF16FFEF4A
:10377000DF06E104F10450F4DBCF81E098EFC916D5
:103780009FEFD906E9069FE0F90690F20F900F909F
:103790000F900F90DF91CF911F910F91FF90EF90BD
:1037A000DF90CF90BF90AF9008957F928F929F92BD
:1037B000AF92BF92CF92DF92EF92FF920F931F933F
:1037C000CF93DF93EC01142F7093E8056093E70526
:1037D0001F8A82E090E0A0E0B0E088839983AA830A
:1037E000BB831092E6051092E2051092E305109259
:1037F000E4051092E5058FEF9FEFDC018093E90768
:103800009093EA07A093EB07B093EC07442349F1A8
:10381000453008F0DEC040E060E070E0CB01B9DC8C
:10382000882309F4D6C020E1129FF0011124E95643
:10383000F84F80818F7709F0CCC084859585A68567
:10384000B78584369105A105B10508F4C2C0C084CE
:10385000D184E284F384C114D104E104F10421F49D
:10386000B8C0C12CD12C760140E0C701B60191DC73
:10387000782E882309F4ADC08091F4059091F50568
:103880008115924009F0A5C03091F905332309F460
:10389000A0C08091F7059091F805892B09F499C093
:1038A0002091F605222309F494C03A8B2C831D86BF
:1038B00030E041E050E06D85062FCA01062E02C0BF
:1038C000880F991F0A94E2F72817390731F081E031
:1038D000860F8D87683078F37CC02091FF0530918A
:1038E00000062115310519F040E050E008C0209194
:1038F0000D0630910E0640910F06509110062D8353
:103900003E834F8358878091F7059091F8054601D3
:103910005701880E991EA11CB11C8B8A9C8AAD8A06
:10392000BE8AE091FA05F091FB05F98FE88FA0912E
:10393000F905B0E00E94A0B3680D791D8A1D9B1D9A
:103940006A8F7B8F8C8F9D8FB5E0EE0FFF1FBA952E
:10395000E1F7E150FE4FEF2FFF27E695DC01CB01A9
:103960008E0F9F1FA11DB11D8E879F87A88BB98BBE
:103970008090FC059090FD058114910419F0A12C14
:10398000B12C08C08090090690900A06A0900B0602
:10399000B0900C06A7019601281B390B4A0B5B0B54
:1039A000DA01C901880D991DAA1DBB1D04C0B69579
:1039B000A795979587950A95D2F789879A87AB87B8
:1039C000BC87853F3FE09307A105B10520F48CE05B
:1039D0008F8B712C15C0853F9F4FA105B10510F449
:1039E00080E10DC08091150690911606A0911706F2
:1039F000B09118068A8F9B8FAC8FBD8F80E28F8B22
:103A0000872DDF91CF911F910F91FF90EF90DF9065
:103A1000CF90BF90AF909F908F907F9008954F92DE
:103A20005F926F927F928F929F92AF92BF92CF924E
:103A3000DF92EF92FF920F931F93CF93DF932C01AE
:103A400024EF33E081E090E0F90145915491441670
:103A500055060CF062C0AC0141505109DA01AA0FC1
:103A6000BB1FAA0FBB1FAE50BC4FFD0165917491E7
:103A7000440F551F440F551F40515C4FFA0165908C
:103A80007490FC01EE0FFF1FEE0FFF1FEE50FC4F76
:103A9000A590B490FD0105911491F901C591D491BF
:103AA000FA0185909490882777FD8095982F0E9441
:103AB0001AB06B017C01B20166197709882777FD7E
:103AC0008095982F0E941AB02B013C01B501601B14
:103AD000710B882777FD8095982F0E941AB09B0163
:103AE000AC01C301B2010E944DB22B013C01BE01E9
:103AF00068197909882777FD8095982F0E941AB058
:103B00009B01AC01C301B2010E947FAF9B01AC01DC
:103B1000C701B6010E949FAE11C001962C5F3F4FB6
:103B20008D33910509F090CFE2EEF4E06591749148
:103B3000882777FD8095982F0E941AB0DF91CF914A
:103B40001F910F91FF90EF90DF90CF90BF90AF90BB
:103B50009F908F907F906F905F904F9008954F92BD
:103B60005F926F927F928F929F92AF92BF92CF920D
:103B7000DF92EF92FF920F931F93CF93DF932C016D
:103B8000662371F1E2ECFEE08491882341F090918C
:103B9000C00095FFFCCF8093C6003196F5CF70E052
:103BA0004AE050E08AE99DE00E94328BE9E5F2E0CC
:103BB0008491882341F09091C00095FFFCCF8093C1
:103BC000C6003196F5CF8091C00085FFFCCF8AE01A
:103BD0008093C6000E944A4660E070E0CB017EC040
:103BE00024E733E081E090E0F901459154914416D7
:103BF00055060CF062C0AC0141505109DA01AA0F20
:103C0000BB1FAA0FBB1FAE58BC4FFD01659174913D
:103C1000440F551F440F551F40595C4FFA016590E2
:103C20007490FC01EE0FFF1FEE0FFF1FEE58FC4FCC
:103C3000A590B490FD0105911491F901C591D4911D
:103C4000FA0185909490882777FD8095982F0E949F
:103C50001AB06B017C01B20166197709882777FDDC
:103C60008095982F0E941AB02B013C01B501601B72
:103C7000710B882777FD8095982F0E941AB09B01C1
:103C8000AC01C301B2010E944DB22B013C01BE0147
:103C900068197909882777FD8095982F0E941AB0B6
:103CA0009B01AC01C301B2010E947FAF9B01AC013B
:103CB000C701B6010E949FAE11C001962C5F3F4F15
:103CC0008032910509F090CFEEEEF3E065917491AA
:103CD000882777FD8095982F0E941AB0DF91CF91A9
:103CE0001F910F91FF90EF90DF90CF90BF90AF901A
:103CF0009F908F907F906F905F904F90089560E0BD
:103D000080914208909143082ADF60933E087093A7
:103D10003F08809340089093410880913C0890911F
:103D20003D087DDE609338087093390880933A0827
:103D300090933B088FB7F894109230088FBF089586
:103D400020911402309115024091160250911702F1
:103D500060E070E08FE793E40E947FAF609310080B
:103D6000709311088093120890931308089597FF99
:103D700003C08091370804C0FC01E65FF74F8081E3
:103D800090E00895CF93DF93D82FC62FC19561E0BF
:103D90000E9429A96C2F8D2F0E9462A96C2F70E0C0
:103DA0008D2FDF91CF910C941FA8CF93C1E020E01D
:103DB00030E048E452E460913E0870913F08809101
:103DC0004008909141080E947BB118160CF0C0E0A9
:103DD0006C2F88E090E0CF91D5CF2F923F924F92F9
:103DE0005F926F927F928F929F92AF92BF92CF928B
:103DF000DF92EF92FF920F931F93CF93DF93CDB794
:103E0000DEB728970FB6F894DEBF0FBECDBF809106
:103E10003008882309F4F8C172DF80903E08909042
:103E20003F08A0904008B0904108009146081091CA
:103E30004708B801882777FD8095982F0E941AB00F
:103E4000A50194010E949EAE6B017C01609318084D
:103E50007093190880931A0890931B0820E030E0B3
:103E600040E251E40E947BB1181624F481E0809373
:103E70000F08F7C020E030E040E251ECC701B60186
:103E80000E9478AF87FD02C0012B21F481E080936E
:103E90000F080CC180910F08882351F010922C0854
:103EA00010922D0810922E0810922F0810920F08D1
:103EB000209118023091190240911A0250911B0270
:103EC000C701B6010E944DB269837A838B839C83BC
:103ED0006093240870932508809326089093270800
:103EE00020912C0830912D0840912E0850912F08D8
:103EF000C701B6010E949FAE2B013C01209014081F
:103F00003090150810911608009117089101412F63
:103F1000502F0E9478AF87FD14C020901008309079
:103F2000110810911208009113089101412F502F90
:103F3000B201C3010E947BB118161CF01201162DAC
:103F4000072DC101A12FB02F80932C0890932D082D
:103F5000A0932E08B0932F082091140230911502DF
:103F60004091160250911702B101812F902F0E94AB
:103F70004DB26D837E838F83988760932008709302
:103F800021088093220890932308209128083091DB
:103F9000290840912A0850912B08C501B4010E94BC
:103FA0009EAE209110023091110240911202509168
:103FB00013020E944DB220ED3CEC4CE45DE30E9404
:103FC0004DB22B013C0123E333E343E75FE3609110
:103FD0001C0870911D0880911E0890911F080E9476
:103FE0004DB29B01AC01C301B2010E949FAE2B01F7
:103FF0003C0160931C0870931D0880931E089093E9
:104000001F082D813E814F81588569817A818B817E
:104010009C810E949FAEA30192010E949EAE2B0143
:104020003C0120E030E04FE753E40E947BB120E008
:1040300030E0A9011816E4F4C701B6010E947BB173
:1040400018167CF4A7019601B101812F902F0E94D0
:104050009EAE60932C0870932D0880932E08909349
:104060002F08412C512C9FE7692E93E4792E21C013
:10407000C301B2010E9478AF87FF1BC020E030E08F
:10408000A901C701B6010E9478AF87FF0FC0A70141
:104090009601B101812F902F0E949EAE60932C0853
:1040A00070932D0880932E0890932F08412C512C4B
:1040B00032018092280890922908A0922A08B09292
:1040C0002B086091020870910308882777FD80957E
:1040D000982F0E941AB09B01AC01C501B4010E9447
:1040E0007BB11816DCF460910802709109028827F0
:1040F00077FD8095982F0E941AB09B01AC01C501F5
:10410000B4010E9478AF87FF09C0C301B2010E94C9
:10411000E7AF7595679560930A0802C010920A0888
:104120000E9409AA0091060810910708209108082A
:1041300030910908601B710B820B930B653C794031
:104140008105910558F031DE0E9409AA60930608A6
:104150007093070880930808909309080E9409AAA1
:1041600000910B0810910C0820910D0830910E0859
:10417000601B710B820B930B6838734181059105AD
:1041800008F442C00E9409AA60930B0870930C08BF
:1041900080930D0890930E08C0903808D09039088D
:1041A000E0903A08F0903B0820E030E040E751E42E
:1041B000C701B6010E947BB118161CF520E030E063
:1041C00046E153E4C701B6010E9478AF87FF19C0EA
:1041D0006091440870914508882777FD8095982F55
:1041E0000E941AB09B01AC01C701B6010E947BB1CD
:1041F00087FD03C01092370807C08FE78093370808
:1042000003C010923708A59828960FB6F894DEBF21
:104210000FBECDBFDF91CF911F910F91FF90EF9017
:10422000DF90CF90BF90AF909F908F907F906F90D6
:104230005F904F903F902F900895CF93DF9310920F
:104240001408109215081092160810921708209161
:10425000140230911502409116025091170260E04D
:1042600070E08FE793E40E947FAF60931008709333
:10427000110880931208909313086D9A80910101A0
:104280008061809301019D9A8091010188608093F3
:10429000010187ED80937A0010927E0010927D00DC
:1042A00080917E00816080937E0080917E0082609C
:1042B00080937E0080917E00846080937E0080E801
:1042C00088BD80916E00846080936E006AEF70E01C
:1042D00080E090E00E9438AA8FE090E0909303087D
:1042E0008093020860E080910A0290910B0237DC13
:1042F00020E030E040E751E40E9478AF87FF0AC039
:1043000080910A0290910B02409790930B02809348
:104310000A02E8CF86E391E09093090280930802B5
:1043200060E0809104089091050819DC20E030E0FD
:104330004BE953E40E947BB1181654F480910408B1
:104340009091050840969093050880930408E8CF63
:10435000C0910008D0910108CE0161DB20E030E07F
:1043600046E153E40E947BB1181634F46096D09372
:104370000108C0930008ECCFDF91CF910895089514
:10438000109247081092460810924508109244086F
:1043900010920A08759810924508109244081092DD
:1043A0003708A59808952F923F924F925F926F928F
:1043B0007F928F929F92AF92BF92CF92DF92EF92B5
:1043C000FF920F931F93CF93DF93CDB7DEB7AE97D6
:1043D0000FB6F894DEBF0FBECDBF6B8F7C8F8D8F75
:1043E000292E5A8749873CA72BA70E9409AA6F8FBD
:1043F00078A389A39AA30E9409AA6FA378A789A783
:104400009AA729853A85121613061CF0E4E2F3E018
:1044100017C0E7E3F3E08191882339F09091C00061
:1044200095FFFCCF8093C600F6CF8091C00085FF3A
:10443000FCCF1BC29091C00095FFFCCF8093C600BB
:1044400081918111F7CF8091C00085FFFCCF8AE078
:104450008093C60095DF49855A858FE7452B99F1F2
:10446000809337088F8D98A1A9A1BAA1898B9A8BC7
:10447000AB8BBC8B8D879E87AF87B88B1D8290E4FA
:10448000988FACE1A98FB6E4BA8F1DA61D8A1E8A4B
:104490001F8A2FE730E040E050E029833A834B83C6
:1044A0005C83EFE74E2E512C612C712C1BA21CA2B9
:1044B0001DA21EA231E03E8F1C861B86312C00E01F
:1044C00010E01EA605C080930A08CCCF0E94737727
:1044D00080913008882309F4F6C011DC49855A859B
:1044E000452B51F0309038080091390810913A0866
:1044F00050913B085EA709C030903E0800913F08EC
:1045000010914008809141088EA7232D302F412F14
:104510005EA56DA57D898E899F890E947BB1181645
:104520002CF03DA60D8B1E8B9EA59F8B232D302F2F
:10453000412F5EA56D81788D898D9A8D0E9478AF0F
:1045400087FD05C03D82088F198FAEA5AA8F0E94F6
:1045500009AA2FA138A549A55AA5621B730B840B84
:10456000950B653C79408105910538F01EDC0E9471
:1045700009AA6FA378A789A79AA74E8D442309F4A7
:104580004FC02B8D3C8D4D8D522D632D702F812F63
:104590009EA50E947BB118160CF095C00E9409AA36
:1045A00029893A894B895C89621B730B840B950BB3
:1045B000693873418105910508F485C0D301C201B2
:1045C00029813A814B815C81821B930BA40BB50B33
:1045D00049855A85B595A79597958795452B19F0E7
:1045E0008093370802C080930A080E9409AA6D8749
:1045F0007E878F87988BDC01CB0129893A894B898B
:104600005C89821B930BA40BB50B8BA39CA3ADA35E
:10461000BEA33B8D3DA74C8D4D8B5D8D5E8B2F8A50
:104620002B8D3C8D4D8D522D632D702F812F9EA58E
:104630000E9478AF87FFEEC20E9409AA2D853E85B1
:104640004F855889621B730B840B950B6938734136
:104650008105910508F4DEC20E9409AA698B7A8B54
:104660008B8B9C8BDC01CB012D853E854F8558893A
:10467000821B930BA40BB50B4B855C85452B09F076
:1046800010C189819A81AB81BC81840D951DA61DC5
:10469000B71D29853A85B595A79597958795232BBD
:1046A00009F4B5C2809337084B855C854F5F5F4F37
:1046B0005C874B875B8D5D838C8D888F9D8D998FFB
:1046C0002A8EA1E0AE8F20E030E040EA51E46B8D0D
:1046D0007C8D8D8D922D0E949FAE9B01AC01632D30
:1046E000702F812F9EA50E947BB1181694F4EFEFD6
:1046F000F2E08491882341F09091C00095FFFCCFB7
:104700008093C6003196F5CF8091C00085FFFCCF25
:10471000ACC00E9409AA2F8D38A149A15AA1621BE1
:10472000730B840B950B613D77408105910508F46F
:104730004FC049855A85452B81F0E0903708F12C10
:10474000E9EFF2E084918823C1F09091C00095FFD9
:10475000FCCF8093C6003196F5CFE0900A08F12C8B
:10476000E3EFF2E08491882341F09091C00095FF3F
:10477000FCCF8093C6003196F5CF22E030E0432D88
:10478000502F612F7EA58AE99DE00E94088CEFEEF4
:10479000F2E08491882341F09091C00095FFFCCF16
:1047A0008093C6003196F5CF4AE050E0B7018AE920
:1047B0009DE00E94328B8091C00085FFFCCF8AE093
:1047C0008093C6000E9409AA6F8F78A389A39AA339
:1047D0000E9409AA6B017C010E9409AA89889A8813
:1047E000AB88BC882D853E854F855889820E931EE7
:1047F000A41EB51EC818D908EA08FB08C60ED71EA5
:10480000E81EF91E31E8C3163FE4D30632E1E306A1
:10481000F10490F0E2EDF2E08491882341F0909170
:10482000C00095FFFCCF8093C6003196F5CF8091F4
:10483000C00085FFFCCF19C04B855C858BA59CA56E
:10484000841795070CF042CEE6E7F2E084918823C6
:1048500041F09091C00095FFFCCF8093C600319647
:10486000F5CF8091C00085FFFCCF8AE08093C60021
:10487000AE960FB6F894DEBF0FBECDBFDF91CF91DD
:104880001F910F91FF90EF90DF90CF90BF90AF906E
:104890009F908F907F906F905F904F903F902F9060
:1048A00008958BA09CA0ADA0BEA0880E991EAA1E44
:1048B000BB1E2BA13CA14DA15EA1281B390B4A0BAD
:1048C0005B0BCA01B90129813A814B815C810E944D
:1048D00013B3A50194010E9478B3240D351D461D24
:1048E000571D243131054105510504F129013A01D3
:1048F0003CEE43165104610471042CF06BEE462E1D
:10490000512C612C712C40E844165104610471044F
:10491000DCF08EEF90E0A0E0B0E084199509A609E4
:10492000B70989839A83AB83BC8312C054E1452EB7
:10493000512C612C712C24E130E040E050E02983BF
:104940003A834B835C8304C049825A826B827C82A7
:10495000E8E6F3E08491882341F09091C00095FF50
:10496000FCCF8093C6003196F5CF2AE030E0B3014A
:10497000A2018AE99DE00E94078BE3E6F3E08491BF
:10498000882341F09091C00095FFFCCF8093C60032
:104990003196F5CF2AE030E049815A816B817C81E4
:1049A0008AE99DE00E94078BECE5F3E0849188237F
:1049B00041F09091C00095FFFCCF8093C6003196E6
:1049C000F5CF22E030E04D81588D698D7A8D8AE9EE
:1049D0009DE00E94088CE5E5F3E08491882341F096
:1049E0009091C00095FFFCCF8093C6003196F5CF23
:1049F00022E030E04DA55D896E897F898AE99DE0DE
:104A00000E94088C8091C00085FFFCCF8AE08093D3
:104A1000C6002B853C85233031050CF432CE6981EC
:104A20007A818B819C810E941AB020E030E040E8BE
:104A300050E40E944DB26B017C012D81388D498D6F
:104A40005A8D6DA57D898E899F890E949EAE20ED2D
:104A50003FE049E450E40E944DB220E030E040E005
:104A60005FE30E944DB29B01AC01C701B6010E94F9
:104A70007FAF6B017C01C501B4010E941AB020E038
:104A800030E04AE754E40E947FAF4B015C01EFE461
:104A9000F3E08491882341F09091C00095FFFCCF12
:104AA0008093C6003196F5CF22E030E0B701A60131
:104AB0008AE99DE00E94088CE9E4F3E08491882370
:104AC00041F09091C00095FFFCCF8093C6003196D5
:104AD000F5CF22E030E0B501A4018AE99DE00E9413
:104AE000088C8091C00085FFFCCF8AE08093C600CF
:104AF0002AE939E949E15FE3C701B6010E944DB2F5
:104B00006B017C019B01AC010E949FAEA501940149
:104B10000E947FAF6D837E838F839887A501940168
:104B2000C701B6010E944DB220E030E040E05EE3F4
:104B30000E944DB24B015C01EBE3F3E084918823CA
:104B400041F09091C00095FFFCCF8093C600319654
:104B5000F5CF8091C00085FFFCCF8AE08093C6002E
:104B6000E5E3F3E08491882341F09091C00095FF44
:104B7000FCCF8093C6003196F5CF22E030E0B7013C
:104B8000A6018AE99DE00E94088C8091C00085FF03
:104B9000FCCF8AE08093C600EFE2F3E084918823A3
:104BA00041F09091C00095FFFCCF8093C6003196F4
:104BB000F5CF22E030E04D815E816F8178858AE912
:104BC0009DE00E94088C8091C00085FFFCCF8AE0A8
:104BD0008093C600E9E2F3E08491882341F090914C
:104BE000C00095FFFCCF8093C6003196F5CF22E040
:104BF00030E0B501A4018AE99DE00E94088C809113
:104C0000C00085FFFCCF8AE08093C6003ACD809338
:104C10000A084ACD1E8E57CDCF93C82FB1DB0E9414
:104C2000114B811134C0E2ECFEE09491992341F0E4
:104C30008091C00085FFFCCF9093C6003196F5CFE0
:104C40006C2F70E04AE050E08AE99DE00E94328BD0
:104C50008091C00085FFFCCF8AE08093C600ECE223
:104C6000F2E08491882341F09091C00095FFFCCF41
:104C70008093C6003196F5CF8091C00085FFFCCFB0
:104C80008AE08093C6008FE192E00E94E476CF91A3
:104C90000C94D24ACF93C82F73DB0E94114B811121
:104CA00034C0E2ECFEE09491992341F08091C00081
:104CB00085FFFCCF9093C6003196F5CF6C2F70E046
:104CC0004AE050E08AE99DE00E94328B8091C0006A
:104CD00085FFFCCF8AE08093C600E2EFF1E084918B
:104CE000882341F09091C00095FFFCCF8093C600CF
:104CF0003196F5CF8091C00085FFFCCF8AE080938C
:104D0000C60085EE91E00E94E476CF910C94D24AE1
:104D1000A5980E94114B811125C0E2ECFEE0849120
:104D2000882341F09091C00095FFFCCF8093C6008E
:104D30003196F5CFEBEAF1E08491882341F0909130
:104D4000C00095FFFCCF8093C6003196F5CF8091CF
:104D5000C00085FFFCCF8AE08093C6008AE991E01D
:104D60000E94E4760C94D24A1F920F920FB60F92D3
:104D700011240BB60F920F931F932F933F934F93D2
:104D80005F936F937F938F939F93AF93BF93CF93D3
:104D9000DF93EF93FF9380910702811112C08091FE
:104DA0000A088093FF07882311F0759A01C075984F
:104DB000809137088093FE07882311F0A59A01C0DF
:104DC000A5989091FF0780910702981708F47598AD
:104DD0009091FE0780910702981708F4A59880919A
:104DE00007028F5F8F77809307028091060290E021
:104DF0008B30910508F093C0FC01EE58FF4F0C94E6
:104E000094B310927B0080E480937C0080917A00C0
:104E1000806480937A000E94ED7681E019C0209131
:104E20007800309179008091FA079091FB07A0916A
:104E3000FC07B091FD07820F931FA11DB11D809348
:104E4000FA079093FB07A093FC07B093FD0782E05D
:104E50008093060264C010927B0082E480937C0001
:104E600080917A00806480937A000E94ED7683E0DE
:104E7000EFCF20917800309179008091F6079091E2
:104E8000F707A091F807B091F907820F931FA11DB2
:104E9000B11D8093F6079093F707A093F807B0939E
:104EA000F90784E0D5CF10927B0081E480937C00E9
:104EB00080917A00806480937A000E94ED7685E08C
:104EC000C7CF20917800309179008091F2079091BE
:104ED000F307A091F407B091F507820F931FA11D6E
:104EE000B11D8093F2079093F307A093F407B0935A
:104EF000F50786E0ADCF0E94ED7687E0A9CF88E088
:104F0000A7CF0E94ED7689E0A3CF10920602809190
:104F1000F1078F5F8093F10702C010920602809123
:104F2000F107803108F463C080913008811110C00E
:104F30008091FA079091FB07909343088093420871
:104F40008091F6079091F70790933D0880933C0875
:104F500081E0809330081092F1071092FA071092C6
:104F6000FB071092FC071092FD071092F2071092B7
:104F7000F3071092F4071092F5071092ED071092C4
:104F8000EE071092EF071092F0071092F6071092BA
:104F9000F7071092F8071092F90720914208309114
:104FA000430880910408909105088217930714F034
:104FB00080E032DE209142083091430880910A025D
:104FC00090910B022817390714F080E063DE2091DE
:104FD0003C0830913D0880910008909101088217AB
:104FE00093072CF0109245081092440891DE00E0DF
:104FF00010E0E801CC0FDD1FCF5CD74F888199818D
:105000001816190644F461E0802F0E94AD9488813F
:105010009981019709C0892B49F060E0802F0E9497
:10502000AD94888199810196998388830F5F1F4F82
:1050300003301105F1F6FF91EF91DF91CF91BF9110
:10504000AF919F918F917F916F915F914F913F9120
:105050002F911F910F910F900BBE0F900FBE0F90CD
:105060001F9018952CEA35EC47E25EE30C944DB2A4
:105070002CEA35EC47E25EE30C947FAF2CEA35EC8A
:1050800047E25EE30C947FAF2CEA35EC47E25EE347
:105090000C944DB2CF93DF93EC0160E08E810E94BF
:1050A00062A981E090E00E945CAA61E08E810E948A
:1050B00062A981E090E00E945CAA60E08E810E947B
:1050C00062A984E690E0DF91CF910C945CAACF9224
:1050D000DF92EF92FF920F931F93CF93DF937C01A8
:1050E000C0E0D0E0C62ED12C87010C0F1D1F61E05F
:1050F000F80187810E9429A9B6010C2E02C075957E
:1051000067950A94E2F76170F80187810E9462A9AD
:105110002196C430D10541F7C701DF91CF911F918E
:105120000F91FF90EF90DF90CF90B4CFCF92DF92AE
:10513000EF92FF920F931F93CF93DF937C01C0E018
:10514000D0E0C62ED12C87010C0F1D1F61E0F801A5
:1051500087810E9429A9B6010C2E02C0759567951A
:105160000A94E2F76170F80187810E9462A9219692
:10517000C830D10541F7C701DF91CF911F910F9141
:10518000FF90EF90DF90CF9085CF1F93CF93DF9369
:10519000EC01162F642F8C810E9462A98D818F3FB4
:1051A00019F060E00E9462A98F85612F84FF05C01D
:1051B000CE01DF91CF911F91B9CF70E084E075955A
:1051C00067958A95E1F7CE0182DF612FCE01DF91ED
:1051D000CF911F917CCF40E0D8CF61E0FCDF80E42D
:1051E00096E00C945CAA62E0F6DF80E496E00C9412
:1051F0005CAACF93DF93CDB7DEB728970FB6F894AC
:10520000DEBF0FBECDBF28E0E7EAF2E0DE01119677
:1052100001900D922A95E1F7FC012389421710F0C5
:105220004FEF420FFE013196E40FF11DE40FF11D27
:105230002081260F2068622F28960FB6F894DEBFD3
:105240000FBECDBFDF91CF91C6CFFC016089262F65
:105250002460208B6C60BFCFCF93DF93EC01423092
:1052600018F08F8588608F874B8B1C8A222329F04A
:10527000413019F48F8584608F8780E593EC0E941C
:105280005CAA60E08C810E9462A960E08E810E942D
:1052900062A98D818F3F19F060E00E9462A96F853D
:1052A00064FD19C063E0CE0112DF84E991E10E9440
:1052B0005CAA63E0CE010BDF84E991E10E945CAA65
:1052C00063E0CE0104DF86E990E00E945CAA62E020
:1052D000CE01FDDE13C06062CE017DDF84E991E185
:1052E0000E945CAA6F856062CE0175DF86E990E05E
:1052F0000E945CAA6F856062CE016DDF6F8560627F
:10530000CE0169DF8CE390E00E945CAA84E0888B88
:10531000CE019BDF8CE390E00E945CAACE015DDFB2
:1053200088EB9BE00E945CAA82E0898B66E0CE015C
:1053300052DF8CE390E0DF91CF910C945CAA6F92E6
:105340007F928F92AF92CF92EF920F931F93CF9352
:10535000DF93CDB7DEB73C01162F842F5E854F85D6
:1053600038899989F301848325830683E782C0867F
:10537000A1868286538744873587968761E00E949D
:1053800029A9F30185818F3F19F061E00E9429A9C5
:1053900061E0F30186810E9429A9112319F0F3012C
:1053A000178603C080E1F301878720E041E060E1D8
:1053B000C301DF91CF911F910F91EF90CF90AF90EC
:1053C0008F907F906F9048CF8F92AF92CF92EF9255
:1053D0000F93DC0113961C921E921297E5E6F3E000
:1053E000ED93FC931F921F921F921F928C2CAE2C58
:1053F000C02EE22E042F2FEF462F61E0A0DF0F908A
:105400000F900F900F900F91EF90CF90AF908F90E3
:105410000895CF93DF93EC01423018F08F858860B8
:105420008F874B8B1C8A222329F0413019F48F85FA
:1054300084608F8780E593EC0E945CAA60E08C8199
:105440000E9462A960E08E810E9462A98D818F3FD7
:1054500019F060E00E9462A96F8564FD19C063E0E5
:10546000CE0135DE84E991E10E945CAA63E0CE01C1
:105470002EDE84E991E10E945CAA63E0CE0127DE82
:1054800086E990E00E945CAA62E0CE0120DE13C0B3
:105490006062CE01A0DE84E991E10E945CAA6F8582
:1054A0006062CE0198DE86E990E00E945CAA6F857A
:1054B0006062CE0190DE6F856062CE018CDE8CE38F
:1054C00090E00E945CAA84E0888BCE01BEDE8CE373
:1054D00090E00E945CAACE0186DE80E496E00E9405
:1054E0005CAA82E0898B66E0CE0175DE8CE390E0F9
:1054F0000E945CAA40E068E0CE017BDE6EE873E0CB
:10550000CE010E9496AE41E068E0CE0172DE6EE808
:1055100073E0CE010E9496AE42E066E0CE0169DE05
:105520006CE873E0CE01DF91CF910C9496AECF92F0
:10553000DF92EF92FF920F931F93CF93DF931F920F
:105540001F92CDB7DEB78C01677088E0689FB0010D
:1055500011246064C80149835A833DDE4981C42E09
:105560005A81D52EE12CF12CD6016D916D01D80117
:10557000ED91FC910190F081E02DC8011995BFEFEC
:10558000EB1AFB0AE8E0EE16F10471F70F900F90AA
:10559000DF91CF911F910F91FF90EF90DF90CF900F
:1055A000089541E0F2DD81E090E008952F923F926E
:1055B0004F925F926F927F928F929F92AF92BF9223
:1055C000CF92DF92EF92FF920F931F93CF93DF93CF
:1055D000CDB7DEB7CF54D1090FB6F894DEBF0FBEFA
:1055E000CDBF1C017E8F6D8F4A012FAB09AF28966E
:1055F000EFAE28972C96ACAEBDAECEAEDFAE2C97FC
:1056000034E0239F50011124FC01EA0DFB1D808131
:105610009181A281B381898F9A8FAB8FBC8FDA0180
:10562000AA0DBB1DBCAFABAF4D905D906D907C9053
:10563000A3019201698D7A8D8B8D9C8D0E949FAE06
:1056400021966CAF7DAF8EAF9FAF2197B4E00B9FDB
:1056500080011124F101E00FF11F2081318142818D
:1056600053812F8F38A349A35AA3A401400F511F80
:1056700023965FAF4EAF2397DA01CD90DD90ED908A
:10568000FC90A70196016F8D78A189A19AA10E9433
:105690009FAE27966CAF7DAF8EAF9FAF27972896B2
:1056A000EFAD2897B4E0EB9FC0011124F101E80FA2
:1056B000F91F20813181428153812BA33CA34DA34B
:1056C0005EA3ED8DFE8DE80FF91F608171818281EF
:1056D00093810E949EAE6FA378A789A79AA7AD8DEC
:1056E000BE8D1C968D919D910D90BC91A02D6096C4
:1056F0008CAF9DAFAEAFBFAF6097D1011C962D911F
:105700003D914D915C911F972BA73CA74DA75EA79C
:10571000A301920150582D8B3E8B4F8B588FD70190
:10572000C601B058898B9A8BAB8BBC8BED8DFE8DEF
:10573000EA0DFB1D20813181428153812FA738ABB7
:1057400049AB5AAB21962CAD3DAD4EAD5FAD219727
:105750006FA578A989A99AA90E949EAE6B017C01C8
:10576000ED8DFE8DE00FF11F80819181A281B381CB
:105770008BAB9CABADABBEAB27962CAD3DAD4EAD70
:105780005FAD2797BC01CD010E949EAE4B015C012D
:10579000A70196016D897E898F89988D0E944DB2EF
:1057A0002B013C01A501940169897A898B899C8927
:1057B0000E944DB29B01AC01C301B2010E949FAE99
:1057C0002B013C01A50194016D897E898F89988DFB
:1057D0000E944DB24B015C01A701960169897A894B
:1057E0008B899C890E944DB29B01AC01C501B4011B
:1057F0000E949EAEA30192010E9412AF6B017C0138
:1058000020E030E0A9010E9478AF87FF0AC02BEDAD
:105810003FE049EC50E4C701B6010E949FAE6B0126
:105820007C01AA968FADAA97882351F02BED3FE01B
:1058300049EC50E4C701B6010E949EAE6B017C01A9
:105840002FA538A949A95AA9698D7A8D8B8D9C8D70
:105850000E9478AF81111FC02BA93CA94DA95EA958
:105860006F8D78A189A19AA10E9478AF811113C090
:1058700020E030E0A901C701B6010E9478AF811194
:105880000AC02BED3FE049EC50E4C701B6010E948D
:105890009FAE6B017C01A9962CAD3DAD4EAD5FADC9
:1058A000A997C701B6010E944DB22FA138A549A5FD
:1058B0005AA55F770E9488B14B015C012FE632E167
:1058C00043E85AE30E9478AF87FDC8C1C501B4011F
:1058D0000E9455B00E94ECAF7A8F698FDB01AB2B31
:1058E00021F4E1E0F0E0FA8FE98F298D3A8DB901DA
:1058F00080E090E00E9418B04B015C019B01AC017C
:10590000C701B6010E947FAF2B013C01A5019401A4
:105910006FA178A589A59AA50E947FAF6FA778ABE4
:1059200089AB9AAB2BA53CA54DA55EA560966CAD49
:105930007DAD8EAD9FAD60970E949EAEA501940196
:105940000E947FAF6BAB7CAB8DAB9EAB20E030E0B9
:1059500040E05FE3C301B2010E944DB2A301920196
:105960000E944DB29B01AC0160E070E080E89FE3D3
:105970000E949EAE6FA378A789A79AA7CE01019631
:10598000FC0128964FAD289734E0439FE00DF11DB0
:1059900011242BA13CA14DA15EA120833183428320
:1059A00053832BA53CA54DA55EA52D873E874F872C
:1059B000588BB12C41E050E058A34F8F1C01BFA978
:1059C000A4E0BA9F800D911D112498AF8FAB910177
:1059D00059AD44E0549F200D311D11243AAF29AF39
:1059E000FCA7EBA74F8D58A1898D9A8D48175907B1
:1059F00008F01AC188E18B150CF444C02FA138A51A
:105A000049A55AA569897A898B899C890E944DB2DA
:105A10006B017C01A30192016D897E898F89988D2C
:105A20000E944DB2A70196010E949FAEA62E172F8D
:105A3000982E892E2FA138A549A55AA56D897E8952
:105A40008F89988D0E944DB26B017C01A301920158
:105A500069897A898B899C890E944DB29B01AC012E
:105A6000C701B6010E949EAE6D8B7E8B8F8B988F87
:105A7000B3948A2D912FA92DB82D898B9A8BAB8B3E
:105A8000BC8B6CC0AF8DB8A1BD0180E090E00E94DE
:105A900018B0A30192010E944DB26B017C010E94DB
:105AA0007CAF698B7A8B8B8B9C8BC701B6010E9474
:105AB000B0B24B015C01EBADFCADC080D180E280A7
:105AC000F380F7FAF094F7F8F0942396AEADBFADFB
:105AD00023972D913D914D915C912BA33CA34DA318
:105AE0005EA329893A894B895C89C701B6010E9466
:105AF0004DB26D8B7E8B8F8B988FA50194016BA11E
:105B00007CA18DA19EA10E944DB29B01AC016D892B
:105B10007E898F89988D0E949FAE6D8B7E8B8F8B37
:105B2000988FA5019401C701B6010E944DB26B0187
:105B30007C0129893A894B895C896BA17CA18DA163
:105B40009EA10E944DB29B01AC01C701B6010E940B
:105B50009EAE698B7A8B8B8B9C8BB12C2D893E8969
:105B60004F89588D21966CAD7DAD8EAD9FAD21973F
:105B70000E949FAEEFA9F8AD608371838283938307
:105B800029893A894B895C8927966CAD7DAD8EADAC
:105B90009FAD27970E949FAEA9ADBAAD6D937D933F
:105BA0008D939C9313972FA538A949A95AA9EBA5C2
:105BB000FCA560817181828193810E949FAEABA51B
:105BC000BCA56D937D938D939C9313972BA93CA9B2
:105BD0004DA95EA96D857E858F8598890E949FAEAF
:105BE0006D877E878F87988BC1010E949242FE014C
:105BF000E659FF4F6F012C96ECACFDAC0EAD1FAD1E
:105C00002C979E01235F3F4FAE01475F5F4FBE0160
:105C10006B5F7F4FC1010E944F9B2F8D38A12F5F7B
:105C20003F4F38A32F8FDECE2D8D3E8D245F3F4F0B
:105C30004D8D5E8D485F5F4F6D8D7E8D6C5F7F4FAC
:105C4000DE01A659BF4F6D012C96ECACFDAC0EAD3C
:105C50001FAD2C978D8D9E8D0E944F9BC15BDF4F9A
:105C60000FB6F894DEBF0FBECDBFDF91CF911F916D
:105C70000F91FF90EF90DF90CF90BF90AF909F90EB
:105C80008F907F906F905F904F903F902F900895EE
:105C9000FC01148217821382128287EB95E09183B4
:105CA0008083089527EB35E0FC0131832083278131
:105CB000222319F004960C9407140895CF92DF92D2
:105CC000EF92FF920F931F93CF93DF93EC01875BCB
:105CD0009F4FDEDFCE0186599F4FDADF7E0129E834
:105CE000E20EF11C87016E0131E4C31A3EEFD30AC4
:105CF000C801CEDF015E1F4F0C151D05C9F7FE015F
:105D0000EF53FE4F89E1818314823596178ACE01C5
:105D10008C519E4FBDDFFE01EB56FD4F108211826C
:105D200012821382389610821182128213821A8292
:105D30001B82188219826E0187E6C81A8DEFD80A75
:105D4000F6011082118212821382F80111821082F0
:105D5000FE01ED5FFD4F108286E391E0F7019C01AB
:105D6000119221503040E1F7FE01EF55FD4F81E0E7
:105D70008083C95BDF4F198218820E9409AA685785
:105D80007C4E8F4F9F4FF601608371838283938394
:105D9000DF91CF911F910F91FF90EF90DF90CF9007
:105DA0000895FC0120E03EE2DB014C91403241F0DD
:105DB000283011F430833196DB014C9140833196C9
:105DC0002F5F6F5F7F4F2B3079F7108208952F92EE
:105DD0003F924F925F926F927F928F929F92AF927B
:105DE000BF92CF92DF92EF92FF920F931F93CF93C8
:105DF000DF93CDB7DEB7CA58D1090FB6F894DEBF2E
:105E00000FBECDBF8C016B017A014901CA57DF4F2C
:105E10001882C658D04084E0E80EF11C180191E1C8
:105E2000290E311CF801EA5BFF4FC957DF4FF98398
:105E3000E883C758D0403801FEE56F1AFDEF7F0AAE
:105E400058018CE5A81A8DEFB80A80E4482E512C31
:105E50004C0E5D1E94E0490E511CA101BE016F5F06
:105E60007F4FC7010E94711218160CF03CC12C859F
:105E7000322F3871303109F09EC0F3018081918159
:105E80000197029708F497C0BE016F5F7F4FCE0164
:105E900087589F4F86DFA0961FAEA097F60180819E
:105EA000811107C069E673E0CE01815A9F4F0E94BD
:105EB000F0B6B601CE01815A9F4F0E94F0B6BE01E6
:105EC00067587F4FCE01815A9F4F0E94F0B669E616
:105ED00073E0CE01815A9F4F0E94F0B6CE01805CE4
:105EE0009F4FD6DE21E0AE0147585F4FB701C20198
:105EF0000E94FE15811139C0F30180819181892BA7
:105F0000A1F5ECEBFEE08491882341F09091C00074
:105F100095FFFCCF8093C6003196F5CFEBE6F3E01A
:105F20008191882339F09091C00095FFFCCF809338
:105F3000C600F6CF8091C00085FFFCCF8AE0809339
:105F4000C600FE01E758FF4F8191882339F09091F8
:105F5000C00095FFFCCF8093C600F6CF8091C000B3
:105F600085FFFCCF8AE08093C6008BE1FE01EC5BED
:105F7000FF4FDE01959601900D928A95E1F72496E8
:105F80008EAD9FAD24979CA38BA387EB95E09AA33E
:105F900089A320E030E0AE014F5D5F4FBE01615A42
:105FA0007F4FC80114DFCE0181967CDECE01805C7C
:105FB0009F4F78DE52CF8981882309F494C08E32B6
:105FC00009F44BCF8F3509F448CFF80181898E321F
:105FD00009F443CF8F3509F440CF23FD3ECF81E054
:105FE000303109F080E0C957DF4FE881F981C758A7
:105FF000D0408083811108C08985873409F02DCF76
:106000008A858E3709F429CF98012C5F3F4FBE0156
:106010006F5F7F4FC901C757DF4F2883C958D040F2
:10602000C657DF4F3883CA58D040BBDEF3018081AA
:106030009181C757DF4F2881C958D040C657DF4FDD
:106040003881CA58D0400097F1F4F6018191882335
:1060500039F09091C00095FFFCCF8093C600F6CF39
:10606000F9018191882339F09091C00095FFFCCF10
:106070008093C600F6CF8091C00085FFFCCF8AE0F8
:106080008093C600EACE8130910539F4F501808114
:106090009181019691838083E0CE029709F0DDCE55
:1060A0008114910439F0B901C4010E94DDB6892B35
:1060B00071F419C0CA57DF4FF881C658D0402F2F4E
:1060C00030E0F501808191812817390761F0CA57C6
:1060D000DF4FF881C658D040FF5FCA57DF4FF883C3
:1060E000C658D040BACEC657DF4F0FB6F894DEBFC1
:1060F0000FBECDBFDF91CF911F910F91FF90EF9019
:10610000DF90CF90BF90AF909F908F907F906F90D7
:106110005F904F903F902F9008950F931F93CF93D0
:10612000DF93CDB7DEB76F970FB6F894DEBF0FBE23
:10613000CDBF8C01FC01EE55FD4F1182108240E075
:1061400050E0BA01835B9F4F0E942413C801875B14
:106150009F4F2BE1FC013496DE01159601900D92C4
:106160002A95E1F7FC01828193819C838B8387EBE5
:1061700095E09A83898320E030E0AE014F5F5F4F66
:1061800062E973E0C80123DECE0101968BDD6F96D4
:106190000FB6F894DEBF0FBECDBFDF91CF911F9138
:1061A0000F9108952BE1FB013496DC0114960190C8
:1061B0000D922A95E1F7FB0122813381FC013383A3
:1061C00022830895EF92FF920F931F93CF93DF9353
:1061D000EC011B82FC01E05BFF4F8081882329F0EA
:1061E000CE01835B9F4F0E9407147E018FE3E81A64
:1061F0008EEFF80A45E360E0C7010E94E73B81119A
:106200001FC0ECEBFEE08491882341F09091C00028
:1062100095FFFCCF8093C6003196F5CFE8ECF6E011
:106220008491882341F09091C00095FFFCCF80932A
:10623000C6003196F5CF8091C00085FFFCCF77C0B6
:106240008E010A531E4F41E0B701C8010E94D51BC1
:10625000811126C040E0B701C8010E94D51B811101
:106260001FC0E2ECFEE08491882341F09091C000D1
:1062700095FFFCCF8093C6003196F5CFE5EBF6E0B5
:106280008491882341F09091C00095FFFCCF8093CA
:10629000C6003196F5CF8091C00085FFFCCF47C086
:1062A000B801CE01835B9F4F0E94141181111FC062
:1062B000E2ECFEE08491882341F09091C00095FFCC
:1062C000FCCF8093C6003196F5CFE5EAF6E08491E5
:1062D000882341F09091C00095FFFCCF8093C600C9
:1062E0003196F5CF8091C00085FFFCCF20C081E0C2
:1062F0008B83ECEBFEE08491882341F09091C00009
:1063000095FFFCCF8093C6003196F5CFEAE9F6E021
:106310008491882341F09091C00095FFFCCF809339
:10632000C6003196F5CF8091C00085FFFCCF8AE092
:106330008093C6008E01075B1F4FB801CE018659BE
:106340009F4F30DFC859DF4F19830883DF91CF910A
:106350001F910F91FF90EF900895FC01128213821C
:106360000895FC012381222311F021E02283089566
:10637000FC012281211112820895AF92BF92CF9227
:10638000DF92EF92FF920F931F93CF93DF931F92B1
:10639000CDB7DEB78C018FE2FB0181935F01D12C79
:1063A00041E07801F1E4EF1AFEEFFF0A9FE1C92E08
:1063B0002D2D30E0F7018081918128173907D8F41D
:1063C000C29EC001C39E900D112483579F4FB501FB
:1063D000800F911F49830E94BB10C50149815C0158
:1063E0000196F5012081222321F04D3810F44F5FF2
:1063F000F6CFD394DDCF47FD11C0B501C801885158
:106400009E4F0F90DF91CF911F910F91FF90EF90D2
:10641000DF90CF90BF90AF900C94BB10F50110822D
:106420000F90DF91CF911F910F91FF90EF90DF9030
:10643000CF90BF90AF9008953F924F925F926F922E
:106440007F928F929F92AF92BF92CF92DF92EF9204
:10645000FF920F931F93CF93DF93CDB7DEB7AC9727
:106460000FB6F894DEBF0FBECDBF7C015B01FC010F
:106470008381882309F408C1C70188519E4F0E9477
:106480000714F7011282CE0101966C0101DC27018D
:1064900098E6490E511CC701875B9F4FF20191831B
:1064A0008083F50180818F3209F084C06FE270E053
:1064B000C5010E94FBB68C010F5F1F4F2AE0322EF0
:1064C0000115110509F47CC06FE270E0C8010E945B
:1064D000FBB64C01009709F474C00817190708F0BF
:1064E00070C03C01601A710AA301B801CE01809608
:1064F0000E9424B7E0E2F0E0EC0FFD1FE60DF71D6F
:106500001082FE01B0968191882339F09091C000ED
:1065100095FFFCCF8093C600F6CF8091C00085FF29
:10652000FCCF3092C600F201608171816115710566
:1065300019F06C5F7F4F02C060E070E021E0AE01B7
:10654000405E5F4FCE0105960E94FE1581112BC063
:10655000EFE7F5E08491882341F09091C00095FF2A
:10656000FCCF8093C6003196F5CFFE01B0968191A5
:10657000882339F09091C00095FFFCCF8093C6002E
:10658000F6CFEDE7F5E08491882341F09091C000CB
:1065900095FFFCCF8093C6003196F5CF8091C00067
:1065A00085FFFCCF6CC0F201D182C08284010F5FF5
:1065B0001F4F86CFC70186599F4FF2019183808379
:1065C0008501F20180819181009711F0049602C04B
:1065D00080E090E0B8010E94D416882339F1EFE6FC
:1065E000F5E08491882341F09091C00095FFFCCFA5
:1065F0008093C6003196F5CFF8018191882339F058
:106600009091C00095FFFCCF8093C600F6CF80919B
:10661000C00085FFFCCF8AE08093C600F701E356F7
:10662000FD4F10821182128213822CC0E7E5F5E043
:106630008491882341F09091C00095FFFCCF809316
:10664000C6003196F5CFF8018191882339F09091F9
:10665000C00095FFFCCF8093C600F6CFE5E5F5E0DE
:106660008491882341F09091C00095FFFCCF8093E6
:10667000C6003196F5CF8091C00085FFFCCF8AE03F
:106680008093C600C6010EDBAC960FB6F894DEBF51
:106690000FBECDBFDF91CF911F910F91FF90EF9073
:1066A000DF90CF90BF90AF909F908F907F906F9032
:1066B0005F904F903F9008958F929F92AF92BF92BC
:1066C000CF92DF92EF92FF92CF93DF931F92CDB7DD
:1066D000DEB77C01FC018281882309F4AFC071968A
:1066E0008191882339F09091C00095FFFCCF809371
:1066F000C600F6CFE3E5F5E08491882341F0909160
:10670000C00095FFFCCF8093C6003196F5CFE1E441
:10671000F5E08491882341F09091C00095FFFCCF73
:106720008093C6003196F5CFF701E356FD4F4081C7
:106730005181628173812AE030E08AE99DE00E9404
:106740005E8BEFE3F5E08491882341F09091C000E7
:1067500095FFFCCF8093C6003196F5CFF701EB563D
:10676000FD4F40815181628173812AE030E08AE9E6
:106770009DE00E945E8B8091C00085FFFCCF8AE087
:106780008093C6000E9409AA30E6C32E3AEED32EAB
:10679000E12CF12CA70196010E9456B349015A0140
:1067A000609150087091510880915208909153085F
:1067B000A70196010E9456B3821A930AC4016CE3A2
:1067C00070E00E942FB36983CE0101960E94087980
:1067D000FC012191CF01222339F03091C00035FF17
:1067E000FCCF2093C600F4CF40E050E06AE38AE992
:1067F0009DE00E94168BC4016CE370E00E942FB3F1
:106800008983CE0101960E940879FC012191CF0174
:10681000222339F03091C00035FFFCCF2093C60011
:10682000F4CFEDE3F5E084918823E1F09091C0008E
:1068300095FFFCCF8093C6003196F5CFE0E3F5E0FD
:106840008491882341F09091C00095FFFCCF809304
:10685000C6003196F5CF8091C00085FFFCCF8AE05D
:106860008093C6000F90DF91CF91FF90EF90DF9063
:10687000CF90BF90AF909F908F900895AF92BF92AE
:10688000CF92DF92EF92FF920F931F93CF93DF93FC
:106890005C01EB01FB0101900020E9F78F01015041
:1068A0001109061B170B6C01F8E1CF1AFEEFDF0A86
:1068B000F60110826EE470E0CE010E94FBB67C010E
:1068C000009729F4F8013197EC0FFD1F0DC060E22D
:1068D00070E00E94FBB6EC0121966AE270E0C7010D
:1068E0000E94FBB6FC0131978DE081838AE08283B0
:1068F0001382BE01C5018C519E4F0E941B8CF60174
:106900008081882309F1E2ECFEE08491882341F044
:106910009091C00095FFFCCF8093C6003196F5CFD3
:10692000EAE1F5E08491882341F09091C00095FF61
:10693000FCCF8093C6003196F5CF8091C00085FFD3
:10694000FCCF8AE08093C600DF91CF911F910F9119
:10695000FF90EF90DF90CF90BF90AF9008952F926F
:106960003F924F925F926F927F928F929F92AF92DF
:10697000BF92CF92DF92EF92FF920F931F93CF932C
:10698000DF93CDB7DEB7CC55D1090FB6F894DEBF93
:106990000FBECDBF4C018C010F551D4F662339F042
:1069A000F8011082F401838181111DC015C0F80126
:1069B0008081882309F4AFC0F401E756FD4FC08001
:1069C000D180E280F3800E9409AAC616D706E806A5
:1069D000F90608F4A0C0E4CFC401F4DBF40183811C
:1069E000882309F498C07401F7E4EF0EF11CF70155
:1069F00081818F9380818F9381E195E09F938F9325
:106A00008E01015C1F4F1F930F930E9433B70F90AD
:106A10000F900F900F900F900F90B12CF8010190F4
:106A20000020E9F73197E01BF10BBE1684F46801F2
:106A3000CB0CD11CB7FCDA94F6018081992787FD35
:106A400090950E9470B6F6018083B394E7CFFDE481
:106A50008F0E911C40E050E0BA01C4010E94241343
:106A6000512CCE0101966C014AE0642E45E0742E53
:106A70005E0191E2A90EB11C40E050E0B601C401F4
:106A80000E9471121816DCF5412CF60101900020CD
:106A9000E9F73197EC19FD094E1674F41601240C30
:106AA000311C47FC3A94F101808190E00E9470B65D
:106AB000F10180834394E9CF8A858E37E9F245E07E
:106AC00050E0B801C6010E9416B7892BA9F61F93A2
:106AD0000F937F926F92BF92AF920E9433B7C5011E
:106AE0000E94E83E86E095E00E945B3F0F900F9089
:106AF0000F900F900F900F9055245394BDCF5110CD
:106B000004C08FEF9FEFF70104C0F70180819181EE
:106B1000019691838083C45ADF4F0FB6F894DEBF8D
:106B20000FBECDBFDF91CF911F910F91FF90EF90DE
:106B3000DF90CF90BF90AF909F908F907F906F909D
:106B40005F904F903F902F9008950F931F93CF9396
:106B5000DF93EC018C0108511E4FC8010E94BD1348
:106B6000C8010E94071418821982DF91CF911F91EA
:106B70000F910895CF92DF92EF92FF920F931F93A0
:106B8000CF93DF93CDB7DEB76F970FB6F894DEBF24
:106B90000FBECDBF8C016A017C0188E6E80EF11CB6
:106BA000C80186599F4FF70191838083E65CFD4FB2
:106BB00022E030E03183208332967183608340E0AD
:106BC00050E0BA0104960E942413F701808191815C
:106BD0002BE1FC013496DE01159601900D922A9569
:106BE000E1F7FC01828193819C838B8387EB95E0A5
:106BF0009A8389839601AE014F5F5F4F62E973E02C
:106C0000C801E5D8CE0101964DD86F960FB6F8941D
:106C1000DEBF0FBECDBFDF91CF911F910F91FF90CF
:106C2000EF90DF90CF9008952F923F924F925F9216
:106C30006F927F928F929F92AF92BF92CF92DF928C
:106C4000EF92FF920F931F93CF93DF93CDB7DEB7F1
:106C5000AC970FB6F894DEBF0FBECDBF8C016B01B1
:106C6000342EDC0113968C91882309F4EEC2F801CE
:106C7000E551FE4F8081882309F4F5C02111C1C080
:106C80007801BDEFEB1AFB0AF7018081882361F1DF
:106C9000E2ECFEE08491882341F09091C00095FFE2
:106CA000FCCF8093C6003196F5CFE7E5F6E08491FE
:106CB000882341F09091C00095FFFCCF8093C600DF
:106CC0003196F5CF4AE050E061E070E08AE99DE05E
:106CD0000E94328B8091C00085FFFCCF8AE08093B8
:106CE000C6000E944A46B1C2ECEBFEE084918823C4
:106CF00041F09091C00095FFFCCF8093C600319683
:106D0000F5CFEEE3F6E08491882341F09091C00046
:106D100095FFFCCF8093C6003196F5CFF6018191A7
:106D2000882339F09091C00095FFFCCF8093C60076
:106D3000F6CFE3E3F6E08491882341F09091C00020
:106D400095FFFCCF8093C6003196F5CFD7018C918B
:106D50006DE8B62EB801B89E600D711D1124685FF4
:106D60007D4FC8010ADBF7018081F801B89EE00D74
:106D7000F11D1124E85FFD4F8191882339F0909136
:106D8000C00095FFFCCF8093C600F6CFEDE2F6E0A1
:106D90008491882341F09091C00095FFFCCF8093AF
:106DA000C6003196F5CF5801F3E6AF1AFDEFBF0AE2
:106DB000D5014D915D916D917C912AE030E08AE999
:106DC0009DE00E945E8B8091C00085FFFCCF8AE031
:106DD0008093C600F7012081F80184E0289FE00D30
:106DE000F11D1124EC5FFD4FD5014D915D916D9129
:106DF0007C9140835183628373832F5FF7012083EB
:106E00002CC0ECEBFEE08491882341F09091C0000F
:106E100095FFFCCF8093C6003196F5CFECE1F6E00C
:106E20008491882341F09091C00095FFFCCF80931E
:106E3000C6003196F5CFF6018191882339F0909103
:106E4000C00095FFFCCF8093C600F6CF8091C000B4
:106E500085FFFCCF8AE08093C600C80188519E4F11
:106E60000E94071430C0F801ED5FFD4F1082ECEB7B
:106E7000FEE08491882341F09091C00095FFFCCF03
:106E80008093C6003196F5CFEBE0F6E0849188233D
:106E900041F09091C00095FFFCCF8093C6003196E1
:106EA000F5CFF6018191882339F09091C00095FFCC
:106EB000FCCF8093C600F6CF8091C00085FFFCCF49
:106EC0008AE08093C600D80112961C92FE0131968A
:106ED0005F01CF010E94482E2801F8E64F0E511C99
:106EE000C801875B9F4FD2018D939C93F6018081EF
:106EF0008F3209F084C06FE270E0C6010E94FBB6D9
:106F000001967C015AE0252EE114F10409F47DC0BC
:106F10006FE270E0C7010E94FBB64C01009709F4D4
:106F200075C0E816F90608F071C03C016E187F08BC
:106F3000A301B701CE0180960E9424B7E0E2F0E001
:106F4000EC0FFD1FE60DF71D1082FE01B09681913A
:106F5000882339F09091C00095FFFCCF8093C60044
:106F6000F6CF8091C00085FFFCCF2092C600D201F1
:106F70006D917C916115710519F06C5F7F4F02C0B6
:106F800060E070E021E0AE01405E5F4FCE0105960B
:106F90000E94FE1581112BC0E7EFF5E08491882354
:106FA00041F09091C00095FFFCCF8093C6003196D0
:106FB000F5CFFE01B0968191882339F09091C00001
:106FC00095FFFCCF8093C600F6CFE5EFF5E0849106
:106FD000882341F09091C00095FFFCCF8093C600BC
:106FE0003196F5CF8091C00085FFFCCF02C1F20140
:106FF000B182A0827401FFEFEF1AFF0A85CFC801AA
:1070000086599F4FD2018D939C937601F801E851E8
:10701000FE4F4F01332009F4B1C0D2016D917C9134
:107020006115710519F06C5F7F4F02C060E070E080
:1070300021E0A701C4010E94FE15882309F474C051
:10704000F40181899289A389B489F801EB56FD4F37
:1070500080839183A283B383E7EEF5E08491D80126
:10706000AB56BD4F882349F09091C00095FFFCCFEF
:107070008093C60031968491F5CFF70181918823E2
:1070800039F09091C00095FFFCCF8093C600F6CFF9
:10709000EFEDF5E08491882341F09091C00095FFD9
:1070A000FCCF8093C6003196F5CF4D915D916D91E7
:1070B0007C912AE030E08AE99DE00E945E8B80911D
:1070C000C00085FFFCCF8AE08093C600F801E3563C
:1070D000FD4F1082118212821382E1EDF5E084915E
:1070E000882341F09091C00095FFFCCF8093C600AB
:1070F0003196F5CF8091C00085FFFCCF8AE0809368
:10710000C600A70160E070E0C80134DDD8015196E7
:107110008C91882319F0C801419601C0C7010E94D3
:107120001F738EE793E08CC0EDEBF5E0849188232C
:1071300041F09091C00095FFFCCF8093C60031963E
:10714000F5CFF7018191882339F09091C00095FF28
:10715000FCCF8093C600F6CFEBEBF5E0849188235B
:1071600041F09091C00095FFFCCF8093C60031960E
:10717000F5CF8091C00085FFFCCF3BC0F20160815C
:1071800071816115710519F06C5F7F4F02C060E07D
:1071900070E026E5A701C4010E94FE1581112DC0F3
:1071A000E7EAF5E08491882341F09091C00095FFD3
:1071B000FCCF8093C6003196F5CFF70181918823EB
:1071C00039F09091C00095FFFCCF8093C600F6CFB8
:1071D000E5EAF5E08491882341F09091C00095FFA5
:1071E000FCCF8093C6003196F5CF8091C00085FF1B
:1071F000FCCF8AE08093C60025C081E0D8018C9343
:10720000E3E9F5E08491882341F09091C00095FF77
:10721000FCCF8093C6003196F5CFF601819188238B
:1072200039F09091C00095FFFCCF8093C600F6CF57
:107230008091C00085FFFCCF8AE08093C600C70123
:107240000E941F73C5010E94522EAC960FB6F8948F
:10725000DEBF0FBECDBFDF91CF911F910F91FF9089
:10726000EF90DF90CF90BF90AF909F908F907F90E6
:107270006F905F904F903F902F90089521E0FC0118
:10728000218340E0D1CCCF92DF92EF92FF920F9317
:107290001F93CF93DF93CDB7DEB76F970FB6F894F8
:1072A000DEBF0FBECDBF8C016C0128E6C20ED11C23
:1072B00086599F4FF60191838083E65CFD4F21E064
:1072C00030E0318320837801FCE5EF1AFDEFFF0AFF
:1072D000F7011182108240E050E0BA0104960E944A
:1072E0002413F601808191812BE1FC013496DE01AB
:1072F000159601900D922A95E1F7FC018281938108
:107300009C838B8387EB95E09A83898320E030E030
:10731000AE014F5F5F4F62E973E0C8010E94E72E44
:10732000CE0101960E94522EF701808191816F96C5
:107330000FB6F894DEBF0FBECDBFDF91CF911F9186
:107340000F91FF90EF90DF90CF900895AF92BF9292
:10735000CF92DF92EF92FF920F931F93CF93DF9321
:10736000CDB7DEB76F970FB6F894DEBF0FBECDBFB7
:107370008C017B01CE0101960E94482EF801EF5846
:10738000FF4F80816801811104C029E4C20ED11C25
:1073900003C08AE6C80ED11C21E0A701B6016C5FCC
:1073A0007F4FCE0105960E94FE1581112DC0ECEB9A
:1073B000FEE08491882341F09091C00095FFFCCFBE
:1073C0008093C6003196F5CFE0EFF4E084918823F6
:1073D00041F09091C00095FFFCCF8093C60031969C
:1073E000F5CFF7018191882339F09091C00095FF86
:1073F000FCCF8093C600F6CF8091C00085FFFCCF04
:107400008AE08093C60036C0F801E154FE4F8081C7
:1074100091818A30910530F59C012F5F3F4F318378
:1074200020832FE1289F7001299FF00C112429E867
:10743000E20EF11CE00EF11E5C01B701C7014F9690
:107440000E94D23081E0A81AB1082FE1E21AF108B7
:107450008FEFA816B80689F7B601C80187579F4F66
:107460000E94D230BE016F5F7F4FC80186599F4F87
:107470000E94D230CE0101960E94522E6F960FB616
:10748000F894DEBF0FBECDBFDF91CF911F910F915A
:10749000FF90EF90DF90CF90BF90AF900895EF9264
:1074A000FF920F931F93CF93DF93EC01C154DE4FF4
:1074B0002881398121153105F9F0215031093983AD
:1074C00028838C0107571F4FB80186599F4F0E9490
:1074D000D230C80100E010E07C012FE1E20EF11C87
:1074E000288139810217130738F40F5F1F4FB70146
:1074F0000E94D230C701F0CFDF91CF911F910F9141
:10750000FF90EF900895EF92FF920F931F93CF9308
:10751000DF93EC010E9415948E010D5F1D4FF80161
:1075200080819E0128513E4F79018823A1F1C90134
:107530000E940714F801808181508083BE01FDE81C
:107540008F9F600D711D1124685F7D4F21E041E028
:10755000CE016ADBF8018081FE0124E0829FE00D0C
:10756000F11D1124EC5FFD4F4081518162817381D7
:10757000FE01E356FD4F4083518362837383C7014D
:107580000E942413CE01DF91CF911F910F91FF90A4
:10759000EF900C94B1310E948B94C7010E940714A4
:1075A0001A8284EE94E0DF91CF911F910F91FF90AA
:1075B000EF9081C48FEF8EBD0DB407FEFDCF8EB569
:1075C00008958EBD0DB407FEFDCF089561E0FC0166
:1075D00080810C9462A9FC012281322F306A369599
:1075E0003CBD20FD06C031E0263009F430E0232FF9
:1075F00001C020E02DBD60E0FC0180810C9462A9F7
:10760000CF92DF92EF92FF920F931F93CF93DF936E
:10761000EC018B017A010E9409AA6B01CBDF8B83FD
:107620008F3F49F40E9409AA6C197D096D3271409F
:10763000A8F381E144C08E3F11F08FE040C0E11417
:10764000F104D9F0C70101972FEF2EBDF8014FEFDC
:107650009F01201B310B2817390738F40DB407FEA2
:10766000FDCF2EB521934EBDF3CF0DB407FEFDCF58
:107670002EB5F801E80FF91F2083D801E00EF11EA6
:10768000C12CD12CAE15BF0579F08D91ED2DFF27C2
:10769000E827EE0FFF1FEB52F94F85919491DC2CF8
:1076A000CC24C826D926EECF85DF082F10E0102F76
:1076B000002780DF082BC016D10631F080E28983D5
:1076C000CE0184DF80E003C0CE0180DF81E0DF9166
:1076D000CF911F910F91FF90EF90DF90CF90089581
:1076E0000F931F93CF93DF93EB010E9409AA8B01A5
:1076F00061DF8F3F49F00E9409AA601B710B6C1774
:107700007D07B0F380E001C081E0DF91CF911F9150
:107710000F910895CF92DF92FF920F931F93CF9313
:10772000DF9300D01F92CDB7DEB76C01F62E298310
:107730003A834B835C834FDF6CE271E0C601D0DF9C
:107740008F2D80643EDF08E110E05C814B813A813F
:107750002981DA01C901002E04C0B695A795979535
:1077600087950A94D2F729833A834B835C8329DF78
:107770000850110929813A814B815C81083F8FEFC4
:10778000180739F7FF2029F0E8E0FE1621F08FEF07
:1077900003C085E901C087E814DFFCE0FF1201C0E7
:1077A00009DF10E007DFF601838387FF04C01F3F76
:1077B00011F01F5FF7CF0F900F900F900F90DF9198
:1077C000CF911F910F91FF90DF90CF900895BF92BE
:1077D000CF92DF92EF92FF920F931F93CF93DF939D
:1077E000EC01B62E1C82198248830E9409AA8B01E3
:1077F00061E088810E9429A9CE01E8DE60E082E391
:107800000E9429A961E083E30E9429A961E084E341
:107810000E9429A961E085E30E9429A961E085E32E
:107820000E9462A985E08A8382E58CBD1DBC6AE066
:10783000F62E8FEFC6DEFA94E1F720E030E0A901E2
:1078400060E0CE0167DFF82E8B8381E0F81649F007
:107850000E9409AA601B710B613D774070F381E0C3
:1078600046C02AEA31E040E050E068E0CE0152DF55
:1078700082FF02C0FC820CC054E0F52E9BDE8B839D
:10788000FA94E1F78A3A11F082E031C082E08C8309
:107890008C81823031F4C12CD12CE12C40E4F42EC7
:1078A00003C0C12CD12C760120E030E0A90167E3B0
:1078B000CE0130DFA701960169E2CE012BDF8B8379
:1078C000882349F00E9409AA601B710B613D774033
:1078D00058F38AE00CC08C818230B1F420E030E0B3
:1078E000A9016AE3CE0116DF882329F088E08983A5
:1078F000CE016CDE14C05EDE807C803C11F483E03F
:107900008C8358DE57DE56DECE0160DE86E08B15B6
:1079100018F488E1898303C0BA8281E001C080E065
:10792000DF91CF911F910F91FF90EF90DF90CF905B
:10793000BF900895AF92BF92CF92DF92EF92FF92E5
:107940000F931F93CF93DF93EC016A017B018901B1
:107950008C81833039F0F9E0CC0CDD1CEE1CFF1C6F
:10796000FA95D1F773E0B72EE4E0AE2EBA94A701F2
:10797000960161E1CE01CEDE882311F0A98207C015
:1079800040E052E0B801CE013BDE81110EC0CE01D5
:10799000BB2049F01BDE20E030E0A9016CE0CE0105
:1079A000B9DE1982E3CF12DE80E0DF91CF911F9123
:1079B0000F91FF90EF90DF90CF90BF90AF90089520
:1079C000CF93DF93EC016EBD20E030E00DB407FEF5
:1079D000FDCFFA01E20FF31F80818EBD0DB407FECB
:1079E000FDCF81818EBD2E5F3F4F211582E038078C
:1079F00069F70DB407FEFDCF8FEFE3DD8FEFE1DD1B
:107A0000D9DD8B838F71853031F083E18983CE019D
:107A1000DDDD80E001C081E0DF91CF9108950F931B
:107A20001F93CF93DF93EC0189018C81833039F070
:107A3000B9E0440F551F661F771FBA95D1F79A0119
:107A4000AB0168E1CE0166DE882311F086E01EC03E
:107A5000A8016EEFCE01B4DF8823C9F068E572E0BB
:107A6000CE013EDE182F811102C087E10FC020E059
:107A700030E0A9016DE0CE014DDE811106C09ADD36
:107A8000811103C0CE01A2DD05C086E18983CE014C
:107A90009DDD10E0812FDF91CF911F910F9108950F
:107AA000FC01659175918591949108952F923F9273
:107AB0004F925F926F927F928F929F92AF92BF92FE
:107AC000CF92DF92EF92FF920F931F93CF93DF93AA
:107AD00000D000D0CDB7DEB71C01FC01E358F14F58
:107AE00014919C01220F331F220F331F3E832D83DD
:107AF0002E5B354F4901F9011082118212821382E7
:107B00002EE43AE04AE45AE066E47AE082E49AE05D
:107B10000E9416A58D819E818457914FC1DF6B0114
:107B20007C01612F772767FD7095872F972F0E9423
:107B30001AB02B013C012D813E81235F354F590145
:107B400020E030E040EC5FE3C701B6010E944DB297
:107B5000A30192010E944DB2F5016083718382837B
:107B600093832D813E81215A3D4F3C832B83F90124
:107B700060817181828193816093210270932202DE
:107B8000809323029093240220E030E040E752E407
:107B90000E947FAF2EE2C22E2AE0D22E7B018C0102
:107BA00029E13AE045E15AE061E17AE08DE09AE0CE
:107BB0000E944F9B0E941594F40110821182128240
:107BC00013822EE43AE04AE45AE066E47AE082E482
:107BD0009AE00E9416A52D813E812058314F3A83AC
:107BE0002983C9015DDF9058A30192010E944DB223
:107BF000F501608371838283938320E030E040E766
:107C000052E46091210270912202809123029091AE
:107C100024020E947FAF7B018C0129E13AE045E11B
:107C20005AE061E17AE08DE09AE00E944F9B0E9469
:107C3000159489819A8134DF9B01AC010E949FAE2B
:107C4000A30192010E944DB2F5016083718382838A
:107C5000938320E030E040E05FE3EB81FC816081D2
:107C60007181828193810E944DB260932102709351
:107C70002202809323029093240220E030E040E728
:107C800052E40E947FAF7B018C0129E13AE045E19B
:107C90005AE061E17AE08DE09AE00E944F9B0E94F9
:107CA00015948D819E818856914FFADE0D811E813B
:107CB0000A5C154FF80120813181428153810E9475
:107CC0009FAEF40160837183828393838D819E8153
:107CD0008055914FE5DE2D813E812D5B3D4F790131
:107CE000F80120813181428153810E949FAEF701CA
:107CF00060837183828393838D819E818C55914FA4
:107D0000CFDE2D813E81295C3D4F7901F801208134
:107D10003181428153810E949FAEF701608371835C
:107D200082839383F40180819181A281B381F501E3
:107D300080839183A283B383109221021092220246
:107D400010922302109224020E94C28CF101ED5C79
:107D5000F54F81E0808326960FB6F894DEBF0FBE04
:107D6000CDBFDF91CF911F910F91FF90EF90DF90EA
:107D7000CF90BF90AF909F908F907F906F905F90CB
:107D80004F903F902F900895FC012491222341F0C1
:107D90003091C00035FFFCCF2093C6000196F4CF90
:107DA00022E030E08AE99DE00C94088CFC012491EB
:107DB000222341F03091C00035FFFCCF2093C60054
:107DC0000196F4CF2AE030E08AE99DE00C945E8BC6
:107DD0002091620830916308243031050CF06AC0AC
:107DE000409164085091650860E6649F9001659F2A
:107DF000300D1124BC01C9018459974F0E940FB75F
:107E0000ECEBFEE08491882341F09091C00095FF57
:107E1000FCCF8093C6003196F5CFE2E7FEE0849177
:107E2000882341F09091C00095FFFCCF8093C6005D
:107E30003196F5CF809164089091650820E6289FDF
:107E4000F001299FF00D1124E459F74F8191882307
:107E500039F09091C00095FFFCCF8093C600F6CF1B
:107E6000E0E7FEE08491882341F09091C00095FF07
:107E7000FCCF8093C6003196F5CF8091C00085FF7E
:107E8000FCCF8AE08093C6008091640890916508D9
:107E9000019664E070E00E9443B39093650880937C
:107EA000640880916208909163080196909363083A
:107EB000809362080895209162083091630824300D
:107EC00031050CF06AC0409164085091650860E685
:107ED000649F9001659F300D1124BC01C901845934
:107EE000974F0E9478B6ECEBFEE08491882341F036
:107EF0009091C00095FFFCCF8093C6003196F5CFDE
:107F0000E5E6FEE08491882341F09091C00095FF62
:107F1000FCCF8093C6003196F5CF80916408909194
:107F2000650820E6289FF001299FF00D1124E459EF
:107F3000F74F8191882339F09091C00095FFFCCFD5
:107F40008093C600F6CFE3E6FEE08491882341F0FB
:107F50009091C00095FFFCCF8093C6003196F5CF7D
:107F60008091C00085FFFCCF8AE08093C60080919D
:107F7000640890916508019664E070E00E9443B344
:107F800090936508809364088091620890916308DB
:107F90000196909363088093620808959B9AA39832
:107FA0000895FCDF40E052EC61E070E08AE99DE07A
:107FB0000E94168AEDE5FEE08491882341F09091BD
:107FC000C00095FFFCCF8093C6003196F5CF80911D
:107FD000C00085FFFCCF8AE08093C6008CEB9EE05A
:107FE000FC012491222341F03091C00035FFFCCFE9
:107FF0002093C6003196F5CF24B720FF14C0E5E5E5
:10800000FEE03491332341F04091C00045FFFCCFA6
:108010003093C6003196F5CF3091C00035FFFCCFCC
:108020003AE03093C60021FF14C0E5E4FEE034914D
:10803000332341F04091C00045FFFCCF3093C60090
:108040003196F5CF3091C00035FFFCCF3AE0309348
:10805000C60022FF14C0E4E3FEE03491332341F074
:108060004091C00045FFFCCF3093C6003196F5CF5C
:108070003091C00035FFFCCF3AE03093C60023FFBB
:1080800014C0E4E2FEE03491332341F04091C0009B
:1080900045FFFCCF3093C6003196F5CF3091C0003C
:1080A00035FFFCCF3AE03093C60025FF14C0E4E171
:1080B000FEE02491222341F03091C00035FFFCCF37
:1080C0002093C6003196F5CF2091C00025FFFCCF4C
:1080D0002AE02093C60014BEEDE0FEE024912223A6
:1080E00041F03091C00035FFFCCF2093C60031969F
:1080F000F5CFE7E0FEE02491222341F03091C0006B
:1081000035FFFCCF2093C6003196F5CF2091C000FB
:1081100025FFFCCF2AE02093C600FC012491ECEB64
:10812000FEE0222349F03091C00035FFFCCF2093C0
:10813000C60031962491F5CFE7EFFDE0249122238C
:1081400041F03091C00035FFFCCF2093C60031963E
:10815000F5CFE2EEFDE02491222341F03091C00002
:1081600035FFFCCF2093C6003196F5CFE6EDFDE05C
:108170002491222341F03091C00035FFFCCF2093A1
:10818000C6003196F5CFEFEBFDE02491222341F0BC
:108190003091C00035FFFCCF2093C6003196F5CF5B
:1081A0002091C00025FFFCCF2AE02093C600E4EB1D
:1081B000FDE02491222341F03091C00035FFFCCF37
:1081C0002093C6003196F5CFE8EAFDE02491222302
:1081D00041F03091C00035FFFCCF2093C6003196AE
:1081E000F5CF2091C00025FFFCCF2AE02093C600E8
:1081F000FC018491ECEBFEE0882349F09091C000F3
:1082000095FFFCCF8093C60031968491F5CFE9E9C4
:10821000FDE08491882341F09091C00095FFFCCF50
:108220008093C6003196F5CF0E9430974AE050E027
:10823000BC018AE99DE00E94328BE2E8FDE0849176
:10824000882341F09091C00095FFFCCF8093C60039
:108250003196F5CF4AE050E060ED74E08AE99DE0A8
:108260000E94328B8091C00085FFFCCF8AE0809312
:10827000C600109268081092690810926A0810925D
:108280006B080E9439880E940B840E941D210E9465
:10829000FF9A0E941E960E944777FFEF23ED80E32E
:1082A000F15020408040E1F700C000000895809127
:1082B0005C0890915D0860E070E001960C94CFB38B
:1082C00080915C0890915D084AE050E060E070E0C9
:1082D00001960C9437B5682F772767FD709520912C
:1082E00066083091670840E6429FC001439F900DA9
:1082F00011248459974F0E94FBB690935D08809398
:108300005C0821E0892B09F420E0822F08950E9467
:1083100009AA609358087093590880935A0890935B
:108320005B0808950E9409AA609358087093590841
:1083300080935A0890935B08E0916608F091670873
:10834000E859F74F8081811114C0EDE7F9E084917D
:10835000882341F09091C00095FFFCCF8093C60028
:108360003196F5CF8091C00085FFFCCF8AE08093E5
:10837000C60008958AE99DE00E94688AE0E8F9E075
:108380008491882341F09091C00095FFFCCF8093A9
:10839000C6003196F5CF4091F1095091F2096091F4
:1083A000F3097091F4094F5F5F4F6F4F7F4F2AE0E1
:1083B00030E08AE99DE00E94078B8091C00085FF34
:1083C000FCCF8AE08093C600ADCF8F929F92AF9290
:1083D000BF92CF92DF92EF92FF920F931F93CF93B2
:1083E000DF9337ECE32E34E0F32E02E41AE0CDE025
:1083F000DAE047E5C42E4AE0D42EF70181917F01EF
:108400006ADF882311F153DF4B015C01F6018081A3
:10841000811103C06091EC0901C061E070E080E06F
:1084200090E00E941AB0F80120813181428153818D
:108430000E944DB29B01AC01C501B4010E949FAEE8
:10844000688379838A839B8309C0F8018081918145
:10845000A281B38188839983AA83BB830C5F1F4F5A
:108460002496FFEFCF1ADF0A8BECE81684E0F806BB
:1084700021F686E430DF8823D1F019DF6B017C011F
:108480006093FD097093FE098093FF099093000AA1
:1084900020E030E0A9010E947BB1181644F4C0929C
:1084A0002102D0922202E0922302F0922402DF9174
:1084B000CF911F910F91FF90EF90DF90CF90BF90E1
:1084C000AF909F908F90089580DF89E404DF882328
:1084D00051F0EDDE6093010A7093020A8093030A63
:1084E0009093040A08C01092010A1092020A109296
:1084F000030A1092040A8AE4EEDE882351F0D7DEE4
:108500006093050A7093060A8093070A9093080AFD
:1085100008951092050A1092060A1092070A109206
:10852000080A0895CF92DF92EF92FF92CF93DF93E4
:10853000EC01C0904302D0904402E0904502F090DC
:108540004602A7019601688179818A819B810E94F8
:1085500078AF87FF04C0C882D982EA82FB82C090CC
:108560004702D0904802E0904902F0904A02A701E9
:1085700096016C817D818E819F810E9478AF87FFFB
:1085800004C0CC82DD82EE82FF8220E030E0A901CF
:1085900060914B0270914C0280914D0290914E027D
:1085A0000E949FAE6B017C019B01AC0168857985BF
:1085B0008A859B850E9478AF87FF04C0C886D986CC
:1085C000EA86FB86C0903702D0903802E0903902EC
:1085D000F0903A02A7019601688179818A819B8196
:1085E0000E947BB1181624F4C882D982EA82FB82E9
:1085F000C0903B02D0903C02E0903D02F0903E02E1
:10860000A70196016C817D818E819F810E947BB143
:10861000181624F4CC82DD82EE82FF82C0903F02E5
:10862000D0904002E0904102F0904202A7019601F2
:10863000688579858A859B850E947BB1181624F40C
:10864000C886D986EA86FB86DF91CF91FF90EF90AE
:10865000DF90CF900895CF92DF92EF92FF920F9329
:108660001F938DE09AE05EDF0E9409AA609358088C
:108670007093590880935A0890935B0820910D0AD3
:1086800030910E0A40910F0A5091100A6091420AEF
:108690007091430A8091440A9091450A0E9478AFF4
:1086A000811179C02091110A3091120A4091130A68
:1086B0005091140A6091460A7091470A8091480AC5
:1086C0009091490A0E9478AF811165C020E030E0A6
:1086D00040E752E4609121027091220280912302CE
:1086E000909124020E947FAF5EE2C52E5AE0D52E03
:1086F0007B018C0129E13AE045E15AE061E17AE051
:108700008DE09AE00E944F9B80910D0A90910E0A95
:10871000A0910F0AB091100A8093420A9093430AE5
:10872000A093440AB093450A8091110A9091120ACD
:10873000A091130AB091140A8093460A9093470AB5
:10874000A093480AB093490A8091150A9091160A9D
:10875000A091170AB091180A80934A0A90934B0A85
:10876000A0934C0AB0934D0A8091190A90911A0A6D
:10877000A0911B0AB0911C0A80934E0A90934F0A55
:10878000A093500AB093510A1F910F91FF90EF9060
:10879000DF90CF90089560915D0270915E0288270E
:1087A00077FD8095982F0E941AB020912102309178
:1087B000220240912302509124020E944DB220E0F7
:1087C00030E040E752E40E947FAF20E030E048EC28
:1087D00052E488CFCF92DF92EF92FF92CF93C62FD1
:1087E000E0912E0AF0E0882309F4C2C0DF01A65D03
:1087F000B54F8C91811196C18091420A9091430AA4
:10880000A091440AB091450A80930D0A90930E0AF4
:10881000A0930F0AB093100A8091460A9091470ADC
:10882000A091480AB091490A8093110A9093120AC4
:10883000A093130AB093140A80914A0A90914B0AAC
:10884000A0914C0AB0914D0A8093150A9093160A94
:10885000A093170AB093180AC0904E0AD0904F0AFE
:10886000E090500AF090510AC092190AD0921A0A68
:10887000E0921B0AF0921C0AEE0FFF1FEE0FFF1F83
:10888000E15BFD4F2081318142815381CC2349F04E
:1088900060912F02709130028091310290913202EA
:1088A00008C060913302709134028091350290913A
:1088B00036020E947FAF9B01AC01C701B6010E9446
:1088C0009FAE60934E0A70934F0A8093500A909324
:1088D000510A8EE49AE00E94BBA5C0902102D0907C
:1088E0002202E0902302F090240220E030E040E7F2
:1088F00052E460912B0270912C0280912D02909194
:108900002E020E944DB26093210270932202809346
:10891000230290932402E0912E0AF0E0E65DF54FE9
:1089200081E0808398DE2091260A3091270A4091C9
:10893000280A5091290A60914A0A70914B0A809145
:108940004C0A90914D0A0E949EAE60934A0A709321
:108950004B0A80934C0A90934D0A2EE43AE04AE485
:108960005AE066E47AE082E49AE00E9416A5D1C05B
:10897000E65DF54F8081882309F4D4C08091420AD6
:108980009091430AA091440AB091450A80930D0A40
:1089900090930E0AA0930F0AB093100A8091460A92
:1089A0009091470AA091480AB091490A8093110A10
:1089B0009093120AA093130AB093140A60914A0A82
:1089C00070914B0A80914C0A90914D0A6093150A60
:1089D0007093160A8093170A9093180AC0904E0A53
:1089E000D0904F0AE090500AF090510AC092190AB4
:1089F000D0921A0AE0921B0AF0921C0A2091260AD1
:108A00003091270A4091280A5091290A0E949FAE6E
:108A100060934A0A70934B0A80934C0A90934D0AD4
:108A20002EE43AE04AE45AE066E47AE082E49AE02E
:108A30000E9416A5F0902E0ACC2389F020911E0AE0
:108A400030911F0A4091200A5091210A60912F0213
:108A500070913002809131029091320210C02091C9
:108A6000220A3091230A4091240A5091250A6091EC
:108A700033027091340280913502909136020E9447
:108A80009FAE24E0F29EF0011124E15BFD4F2081B6
:108A90003181428153810E947FAF9B01AC01609183
:108AA0004E0A70914F0A8091500A9091510A0E948B
:108AB0009EAE60934E0A70934F0A8093500A909333
:108AC000510A8EE49AE00E94BBA5C0902102D0908A
:108AD0002202E0902302F090240220E030E040E700
:108AE00052E46091270270912802809129029091AE
:108AF0002A020E944DB26093210270932202809359
:108B0000230290932402E0912E0AF0E0E65DF54FF7
:108B10001082A1DDC0922102D0922202E0922302B3
:108B2000F0922402CF91FF90EF90DF90CF900895C4
:108B3000AF92BF92CF92DF92EF92FF920F931F936B
:108B4000CF93DF93D82F2091050A3091060A4091E8
:108B5000070A5091080A6091010A7091020A8091F7
:108B6000030A9091040A0E9488B1C62F172F082F7C
:108B7000F92E60915D0270915E02882777FD8095E5
:108B8000982F0E941AB02091210230912202409128
:108B90002302509124020E944DB220E030E040E7D1
:108BA00052E40E947FAF20E030E048EC52E40E94A3
:108BB0007FAF20912E0A2F93DF93FF920F931F9385
:108BC000CF935B016C0172E0E72E01E020E041E011
:108BD0005AE06DE07AE082E49AE00E94D62A809121
:108BE0000D0A90910E0AA0910F0AB091100A80937D
:108BF000420A9093430AA093440AB093450A809195
:108C0000110A9091120AA091130AB091140A80934C
:108C1000460A9093470AA093480AB093490A809164
:108C2000150A9091160AA091170AB091180A80931C
:108C30004A0A90934B0AA0934C0AB0934D0A809134
:108C4000190A90911A0AA0911B0AB0911C0A8093EC
:108C50004E0A90934F0AA093500AB093510A0E9473
:108C600009AA609358087093590880935A08909302
:108C70005B080F900F900F900F900F900F90DF9167
:108C8000CF911F910F91FF90EF90DF90CF90BF9009
:108C9000AF900895F8940E94C021179A1092330A59
:108CA000169A1092340A159A1092350A149A60E0B6
:108CB00087E40E9429A9E2ECFEE08491882341F038
:108CC0009091C00095FFFCCF8093C6003196F5CF00
:108CD000EEE5F9E08491882341F09091C00095FF82
:108CE000FCCF8093C6003196F5CF8091C00085FF00
:108CF000FCCF8AE08093C60085E599E00E94E47687
:108D00007894C6E0D0E02197209749F068EC70E0B5
:108D100080E090E00E9438AA0E947377F4CFF89424
:108D2000FFCF2F923F924F925F926F927F928F92DE
:108D30009F92AF92BF92CF92DF92EF92FF920F93EA
:108D40001F93CF93DF93CDB7DEB76E970FB6F8942E
:108D5000DEBF0FBECDBFB0E6BB2E14E0E12EF12C7E
:108D600008E4C02E0CE0D02E8AE0A82E992493941B
:108D700080911B0E90911C0E20911D0E30911E0EA5
:108D8000821B930B8F779927892B09F41AC2809144
:108D900062089091630804970CF013C28AE99DE081
:108DA0000E944C8A8093610820915F08309160088E
:108DB0008A3061F08D3051F08A3321F490915E0851
:108DC000992321F02F3531050CF41DC121153105F2
:108DD00009F437C18091640890916508B89E30010C
:108DE000B99E700C1124F301E20FF31FE459F74F01
:108DF000108220915E08211101C110925E08FC01D1
:108E0000E859F74F108283010459174F6EE470E060
:108E1000C8010E94FBB60097F1F190935D08809322
:108E20005C08801B910B860D971D4AE050E060E0C6
:108E300070E08359974F0E9437B56093F50970939E
:108E4000F6098093F7099093F8094090F109509042
:108E5000F2096090F3097090F4092FEF421A520A58
:108E6000620A720A0091640810916508641575051C
:108E70008605970509F4E8C0B09EC001B19E900D2B
:108E8000112464E67DE08459974F0E94A6B6892B91
:108E900009F0DAC069C16AE270E0C8010E94FBB65D
:108EA000892B09F444C0E2ECFEE08491882341F070
:108EB0009091C00095FFFCCF8093C6003196F5CF0E
:108EC000EEEBFCE08491882341F09091C00095FF87
:108ED000FCCF8093C6003196F5CF4091F1095091B7
:108EE000F2096091F3097091F4092AE030E08AE90F
:108EF0009DE00E94078B8091C00085FFFCCF8AE037
:108F00008093C6001092600810925F08C0C28091E2
:108F1000F5099091F609A091F709B091F8098093AD
:108F2000F1099093F209A093F309B093F4098091A9
:108F3000640890916508B89E8001B99E100D1124B7
:108F4000C8018459974F3C0167E470E00E94FBB66A
:108F5000009781F190935D0880935C0886199709CA
:108F6000800F911F60E070E08359974F0E94CFB34C
:108F70000E94E7AF64307105E8F480914A088823C5
:108F8000C9F0F6018491E8E4FCE0882349F090916F
:108F9000C00095FFFCCF8093C60031968491F5CF39
:108FA0008091C00085FFFCCFA092C6008EE39CE0BC
:108FB0000E94D7760091640810916508B09EC001A8
:108FC000B19E900D112463E973E08459974F0E947C
:108FD00006B7892B09F45EDEC8010196B7010E942D
:108FE00043B39093650880936408809162089091E0
:108FF000630801969093630880936208109260085A
:1090000010925F08B5CE8B3311F490925E08909168
:109010005E089111ADCE4091640850916508B90188
:109020006F5F7F4F7093600860935F08B49EF0019C
:10903000B59EF00D1124E20FF31FE459F74F808322
:1090400097CE10925E0823C2B09E3001B19E700C84
:109050001124C3018459974F1C016AE270E00E94F9
:10906000FBB6009789F5E2ECFEE08491882341F09D
:109070009091C00095FFFCCF8093C6003196F5CF4C
:10908000E8EEFCE08491882341F09091C00095FFC8
:10909000FCCF8093C6003196F5CF4091F1095091F5
:1090A000F2096091F3097091F4092AE030E08AE94D
:1090B0009DE00E94078B8091C00085FFFCCF8AE075
:1090C0008093C60057D91ECF20E010E0F301E20FD5
:1090D000F11DE459F74F30813A3219F02F5F132711
:1090E000F5CF90935D0880935C0882199309860DF3
:1090F000971D60E070E08359974F0E94CFB30E94A4
:10910000E7AF212F30E02617370709F400CFE2EC54
:10911000FEE08491882341F09091C00095FFFCCF40
:109120008093C6003196F5CFE2E1FDE0849188237B
:1091300041F09091C00095FFFCCF8093C60031961E
:10914000F5CF4091F1095091F2096091F3097091C6
:10915000F4092AE030E08AE99DE00E94078B8091C3
:10916000C00085FFFCCFABCFE2ECFEE0849188230A
:1091700041F09091C00095FFFCCF8093C6003196DE
:10918000F5CFE1E3FDE08491882341F09091C000A8
:1091900095FFFCCF8093C6003196F5CF4091F10941
:1091A0005091F2096091F3097091F4092AE030E0DE
:1091B0008AE99DE00E94078B8091C00085FFFCCF6B
:1091C0007ECF80915D0A882309F461C180915F0898
:1091D00090916008892B09F05AC1809162089091A2
:1091E0006308892B11F410924808F8EE2F2EF3E053
:1091F0003F2E412C512CACE3CA2ED12CE12CF12C6A
:109200008E010F5F1F4FE0E66E2E7724739440911E
:10921000F80C5091F90C6091FA0C7091FB0C809154
:10922000F00C9091F10CA091F20CB091F30C481756
:1092300059076A077B0708F02AC18091620890915C
:10924000630804970CF023C18091480881111FC165
:1092500080914B0C90914C0CA0914D0CB0914E0C08
:109260008093F80C9093F90CA093FA0CB093FB0C3C
:1092700083E49CE00E945B12482F809361088A304F
:10928000B9F04D30A9F0433229F420915E08222331
:1092900079F002C04A33C9F320915F083091600829
:1092A0002F3531052CF48F3FFFEF9F0709F0D1C018
:1092B0004091F80C5091F90C6091FA0C7091FB0CF4
:1092C0008091F00C9091F10CA091F20CB091F30C04
:1092D000481759076A077B0708F481C0EBE2FCE0F6
:1092E0008491882341F09091C00095FFFCCF80933A
:1092F000C6003196F5CF8091C00085FFFCCFFAE023
:10930000F093C6000E9409AA60934C0870934D0820
:1093100080934E0890934F08809050089090510889
:10932000A0905208B0905308681979098A099B09DE
:10933000A20191010E9456B349015A01CA01B90123
:10934000A70196010E9456B3CA01B901A70196016F
:109350000E9456B37F936F93C501B40120E13EE0B4
:1093600040E050E00E9456B33F932F93A7E1BCE04A
:10937000BF93AF931F930F930E9433B7ECEBFEE0C4
:1093800084910FB6F894DEBF0FBECDBF882349F09D
:109390009091C00095FFFCCF8093C60031968491D8
:1093A000F5CFF8018191882339F09091C00095FFA5
:1093B000FCCF8093C600F6CF8091C00085FFFCCF24
:1093C0003AE03093C600C8010E941F738BE59AE013
:1093D0000E94833A61E08BE59AE00E94AF3480916D
:1093E0006108833211F47092480820915F0830912F
:1093F00060082115310509F424CE8091640890910C
:109400006508689EF001699EF00D1124E20FF31FBC
:10941000E459F74F1082FC01E859F74F7082209110
:109420006208309163082F5F3F4F309363082093A9
:109430006208019664E070E00E9443B3909365086F
:109440008093640810925E081092600810925F0882
:10945000DECE4B3311F470925E0840915E084111EC
:10946000D2CE4091640850916508B9016F5F7F4F7B
:109470007093600860935F08649EF001659EF00D34
:109480001124E20FF31FE459F74F8083C0CE6E968C
:109490000FB6F894DEBF0FBECDBFDF91CF911F9105
:1094A0000F91FF90EF90DF90CF90BF90AF909F9083
:1094B0008F907F906F905F904F903F902F90089586
:1094C000CF92DF92EF92FF920F931F93CF93C82F0B
:1094D000809162089091630803970CF422DC0E944B
:1094E00009AA00915408109155082091560830910E
:1094F0005708C0905808D0905908E0905A08F0904A
:109500005B086C197D098E099F0906171707280744
:10951000390728F4012B022B032B09F0BBDB409108
:109520001D0250911E0260911F0270912002452B76
:10953000462B472B19F10E9409AA00915808109157
:10954000590820915A0830915B08601B710B820BFF
:10955000930B00911D0210911E0220911F02309169
:109560002002061717072807390740F490916B0E61
:1095700080916A0E981302C0CC2349F0CF911F91BD
:109580000F91FF90EF90DF90CF900C94339B179A40
:109590001092330A169A1092340A159A1092350ACC
:1095A000149AECCF0E94C02180914A08811138C0E2
:1095B00081E080934A088091F1099091F209A0918D
:1095C000F309B091F4098093ED099093EE09A0930B
:1095D000EF09B093F009E2ECFEE08491882341F0BA
:1095E0009091C00095FFFCCF8093C6003196F5CFD7
:1095F000EFEDF8E08491882341F09091C00095FF51
:10960000FCCF8093C6003196F5CF8091C00085FFD6
:10961000FCCF8AE08093C60085ED98E00C94D77665
:10962000089580914A080895CF93DF93EC018091CB
:109630002E0A80934B0884E50E946B41811102C081
:1096400080E075C00E9457410E94ECAF60934B08C8
:109650006623B1F3ECEBFEE08491882341F0909116
:10966000C00095FFFCCF8093C6003196F5CFCD3674
:10967000D105B9F054F4C836D105B1F0C936D105D9
:1096800009F045C0EDEDF3E021C0CA3DD10531F050
:10969000CD3DD105E1F5E8E9F3E036C0EFEAF3E0CE
:1096A00029C0E6ECF3E01CC0E4EFF3E081918823ED
:1096B00071F19091C00095FFFCCF8093C600F6CF6A
:1096C0009091C00095FFFCCF8093C60081918111DD
:1096D000F7CF1DC09091C00095FFFCCF8093C600CE
:1096E00081918111F7CF13C09091C00095FFFCCFFD
:1096F0008093C60081918111F7CF09C09091C0007D
:1097000095FFFCCF8093C60081918111F7CF40E097
:1097100050E060914B088AE99DE00E94698B80913E
:10972000C00085FFFCCF8AE08093C60081E0DF9116
:10973000CF910895CF92DF92EF92FF922091520A3B
:109740002223F1F020E030E040E05FE30E944DB2E0
:109750006B017C0120E030E0A9010E9478AF8823F2
:1097600079F0A7019601C701B6010E944DB22BED19
:109770003FE049E450E40E944DB29B01AC0104C0BB
:1097800020E030E040E85FE360E070E080E89FE3E5
:109790000E947FAFFF90EF90DF90CF90089560918F
:1097A0005302709154028091550290915602C2DF8B
:1097B00060934F0270935002809351029093520233
:1097C00008953F924F925F926F927F928F929F92F5
:1097D000AF92BF92CF92DF92EF92FF920F931F93BF
:1097E000CF93DF93CDB7DEB7E9970FB6F894DEBF1E
:1097F0000FBECDBF81E40E946B418823B1F182E7A7
:109800000E946B418823A9F0EAE1F4E0819188236A
:1098100039F09091C00095FFFCCF8093C600F6CF41
:109820008091C00085FFFCCF8AE08093C6000C9435
:10983000046286E70E946B41882311F40C94046251
:10984000E0E2F4E08191882339F09091C00095FF27
:10985000FCCF8093C600F6CF8091C00085FFFCCF7F
:109860008AE08093C6000C94046287E40E946B41F6
:10987000882309F44CC20E9457410E94E7AF6A3026
:10988000710509F4AFC09CF46230710509F44CC055
:1098900024F477FF25C00C9404626330710509F449
:1098A0004EC06430710509F455C00C9404626A35E9
:1098B000710509F4D8C154F46B30710509F498C0EE
:1098C0006C31710509F49AC00C9404626B35710512
:1098D00009F4CDC16C35710509F4CEC10C94046254
:1098E00080914A0881110C9404620E94E5418091A4
:1098F0002B0A8823A9F088E50E946B41811110C0D2
:1099000089E50E946B4181110BC08AE50E946B4181
:10991000811106C085E40E946B4181110C9407629D
:109920000E942B430C94046280914A0881110C948C
:1099300004620E94644281E0FBD80C94046280912E
:109940004A0881110C9404620E94644280E0F0D8BD
:109950000C9404628EE09CE00E94D77680E50E9421
:109960006B41882339F00E9457410E94ECAF4B01B4
:109970005C0103C0812C912C540183E50E946B4152
:10998000882361F00E94574120E030E04AE754E428
:109990000E944DB20E94ECAF4B015C010E941594F5
:1099A0000E9409AA6B017C01C80CD91CEA1CFB1C93
:1099B0000E9409AA609358087093590880935A0826
:1099C00090935B080E9409AA6C157D058E059F0582
:1099D00010F00C9404620E94ED1E80E071DD0E9484
:1099E0007377F0CF60E081E00E94EA430C94046258
:1099F00060E080E00E94EA430C94046280912102BE
:109A000090912202A0912302B09124028093F9093F
:109A10009093FA09A093FB09B093FC0980915D0231
:109A200090915E029093560A8093550A84E690E0E6
:109A300090935E0280935D020E9409AA6093580889
:109A40007093590880935A0890935B0881E00E94B4
:109A5000C98C8091420A9091430AA091440AB09126
:109A6000450A80930D0A90930E0AA0930F0AB093B3
:109A7000100A8091460A9091470AA091480AB09135
:109A8000490A8093110A9093120AA093130AB09383
:109A9000140A80914A0A90914B0AA0914C0AB09105
:109AA0004D0A8093150A9093160AA093170AB09353
:109AB000180A80914E0A90914F0AA091500AB091D5
:109AC000510A8093190A90931A0AA0931B0AB09323
:109AD0001C0A10922102109222021092230210926C
:109AE000240288E50E946B41882311F090E00AC0AF
:109AF00089E50E946B418111F9CF8AE50E946B4193
:109B000091E098279093250291110C94366288E594
:109B10000E946B4181110C94366280912502811163
:109B20000C943C6289E50E946B4181110C943C626B
:109B300088E50E946B418823D1F00E946041672B29
:109B4000682B692BA1F00E9457412091360A309171
:109B5000370A4091380A5091390A0E949FAE6093AB
:109B6000420A7093430A8093440A9093450A89E518
:109B70000E946B418823D1F00E946041672B682BC3
:109B8000692BA1F00E94574120913A0A30913B0A7B
:109B900040913C0A50913D0A0E949FAE6093460A54
:109BA0007093470A8093480A9093490A809125024E
:109BB00081110C9442628AE50E946B4181110C94E0
:109BC00042628AE50E946B418823D1F00E94604185
:109BD000672B682B692BA1F00E94574120913E0A08
:109BE00030913F0A4091400A5091410A0E949FAE35
:109BF00060934A0A70934B0A80934C0A90934D0AE3
:109C00002EE43AE04AE45AE066E47AE082E49AE03C
:109C10000E9416A580E00E94C98C8091F90990915C
:109C2000FA09A091FB09B091FC098093210290935D
:109C30002202A0932302B09324028091550A9091AE
:109C4000560A90935E0280935D020E9409AA609377
:109C500058087093590880935A0890935B080E94A3
:109C6000C28C0C9404621092EC090C94046281E0A2
:109C70008093EC090C94046285E40E946B4181118D
:109C800002C00E94159457ECC52E54E0D52E66E311
:109C9000E62E6AE0F62E02E41AE0B12CF60181917C
:109CA0006F010E946B41882339F1F3E0BF120CC0B1
:109CB0000E945741F80160837183828393838EE40D
:109CC0009AE00E94BBA518C00E945741F70120816D
:109CD0003181428153810E949FAEF801608371837C
:109CE000828393832EE43AE04AE45AE066E47AE021
:109CF00082E49AE00E9416A5B394F4E0EF0EF11C02
:109D00000C5F1F4F24E0B212C9CF0C9404628DE4A3
:109D10000E946B41882311F40C9433610E945741D7
:109D20000E94E7AF6537710511F40C94F1560CF001
:109D3000A6C06032710509F4F0C20CF056C067315C
:109D4000710509F445C254F56231710509F468C71B
:109D5000BCF477FF02C00C940462623071050CF40D
:109D600061C16131710511F00C94046281ED9BE0D9
:109D70000E94D77617981698159814980C94046238
:109D80006531710509F418C20CF01CC2643171050B
:109D900011F00C940462E1ECFBE0EAC16B31710557
:109DA00009F442C2B4F46931710509F429C20CF016
:109DB0002DC28BE59AE00E94B1310E9409AA6093FE
:109DC00050087093510880935208909353080C9454
:109DD00004626E31710509F462C20CF03AC36C3151
:109DE000710509F427C20C9404626C35710509F4FD
:109DF0006AC7ECF46235710509F409C764F460358B
:109E0000710509F4DAC60CF0E5C66A32710509F489
:109E10007EC30C9404626435710509F401C70CF427
:109E2000FAC66535710509F433C70C9404626B36C4
:109E3000710509F4BCC664F46936710509F4DEC322
:109E40000CF085C66836710509F4A8C30C94046249
:109E50006037710509F4BFC334F46D36710509F438
:109E6000D9C40C9404626237710509F4CEC7633714
:109E7000710511F00C940462EFE3FAE0ADC76D3D9B
:109E8000710511F40C94F95A0CF04DC06B3C71053E
:109E900011F40C94755944F56C38710509F49DC39F
:109EA0009CF46837710511F40C94E5576937710516
:109EB00011F40C94EA576737710511F00C940462A1
:109EC000E7E2F4E00C94F557683C710511F40C944A
:109ED000DF58693C710511F40C9454596E3B7105BF
:109EE00011F00C94046220C56F3C710511F40C94C0
:109EF0002F5A54F46D3C710511F40C94B45914F4B8
:109F00000C9492590C94125A613D710511F40C9401
:109F10008A5A14F40C94645A6C3D710511F40C9433
:109F2000EA5A0C940462603931E0730711F40C941E
:109F3000BC5C54F56E3291E0790711F40C94765CB8
:109F400084F46C32F1E07F0711F40C947A5B14F026
:109F50000C94B05B623E710511F40C941F5B0C9481
:109F600004626E3531E0730711F40C94A0606F3514
:109F700081E0780711F40C94D7606F32714011F0D2
:109F80000C9404620C94845C6835E2E07E0711F462
:109F90000C949A5DBCF4663F21E0720711F40C94B6
:109FA000BF5C673F31E0730711F40C94C25C653FFE
:109FB000714011F00C9404620E9439880E940B8455
:109FC0000C9404626B3893E0790711F40C947A6076
:109FD0003CF46335734011F40C94C55C0C9404623A
:109FE000603A23E0720709F401C2673E734011F042
:109FF0000C94046210924A080E94EA768091ED095E
:10A000009091EE09A091EF09B091F0098093F109C8
:10A010009093F209A093F309B093F4090E94BA4116
:10A020000C94046200915C0810915D080E5F1F4F54
:10A0300080E50E946B41882379F00E9457410E947D
:10A04000ECAF6B017C01BB24B394611571058105F4
:10A05000910531F4B12C04C0B12CC12CD12C760166
:10A0600083E50E946B41882399F00E94574120E0CC
:10A0700030E04AE754E40E944DB20E94ECAF6B011D
:10A080007C01AA24A394611571058105910509F449
:10A09000A12C6AE270E0C8010E94FBB6009711F0A3
:10A0A000FC011082F801CF0121912032E1F3B110BF
:10A0B00007C0A11005C0222319F00E941F7304C01D
:10A0C0008DEF9BE00E94D77681E00E94FF720E9494
:10A0D00015940E9409AA60935808709359088093B8
:10A0E0005A0890935B08C114D104E104F104A9F06B
:10A0F0000E9409AA4B015C018C0C9D1CAE1CBF1C6C
:10A100000E9409AA681579058A059B05B8F40E9482
:10A110003978811113C00C9448620E9437788823E3
:10A1200011F40C9404620E94397881110AC00E94D3
:10A13000ED1E80E0C5D90E947377F5CF80E00E94C4
:10A14000FF7280915D0A882331F08EEE9BE00E94C1
:10A15000D7760C9404628AED9BE00E94D7760C942B
:10A1600004629091C00095FFFCCF8093C6003196A9
:10A1700084918111F6CF8091C00085FFFCCF8AE0E9
:10A180008093C6008BE59AE00E948D30E3EBFBE004
:10A190008491882341F09091C00095FFFCCF80937B
:10A1A000C6003196F5CF8091C00085FFFCCF8AE0D4
:10A1B0008093C6000C9404628BE59AE00E94E23022
:10A1C0000C9404628BE59AE00E94AD310C94046219
:10A1D00000915C0810915D080C5F1F4F6AE270E00F
:10A1E000C8010E94FBB6009711F0FC01108221E02B
:10A1F00041E0B8018BE59AE00E9414360C940462A9
:10A200008BE59AE00E94B8310C94046280915E0A5A
:10A21000882311F40C94046283E50E946B41811140
:10A220000C9451620C9404628BE59AE00E945C33BA
:10A230000C94046280915C0890915D086AE270E081
:10A2400004960E94FBB68C010097D9F02091660815
:10A250003091670840E6429FC001439F900D112452
:10A260006EE470E08459974F0E94FBB660E270E0A4
:10A270000E94FBB6019690935D0880935C08F801FC
:10A28000108260915C0870915D086C5F7F4F21E0E7
:10A2900040E08BE59AE00E9414360C9404628091B1
:10A2A0005E0A882311F40C94046260E08BE59AE066
:10A2B0000E94A53580915C0890915D086AE270E08B
:10A2C00004960E94FBB68C010097D9F02091660895
:10A2D0003091670840E6429FC001439F900D1124D2
:10A2E0006EE470E08459974F0E94FBB660E270E024
:10A2F0000E94FBB6019690935D0880935C08F8017C
:10A30000108260915C0870915D086C5F7F4F8BE5F7
:10A310009AE00E941C320C94046280915D0A8111C3
:10A320000E94159400915C0810915D080C5F1F4F0E
:10A330006AE270E0C8010E94FBB67C0161E270E055
:10A34000C8010E94FBB6009719F08C010F5F1F4FE8
:10A35000E114F10411F0F701108280E50E946B41D5
:10A36000F82E20915C0830915D080217130708F45D
:10A37000F12C80915E0A882311F40C94046221E090
:10A380002F2541E0B8018BE59AE00E94143683E561
:10A390000E946B418823B9F020915C0830915D08E0
:10A3A0002017310780F40E946041AB01BC0140934B
:10A3B000F80C5093F90C6093FA0C7093FB0C83E447
:10A3C0009CE00E9424138BE59AE00E94B131F110C9
:10A3D0000C9404620E9409AA60935008709351087B
:10A3E00080935208909353080C94046280915C0807
:10A3F00090915D086AE270E005960E94FBB68C01C0
:10A400000097D9F0209166083091670840E6429F96
:10A41000C001439F900D11246EE470E08459974F62
:10A420000E94FBB660E270E00E94FBB6019690933A
:10A430005D0880935C08F801108260915C0870915F
:10A440005D086B5F7F4F8BE59AE00E943E390C946C
:10A4500004620E9409AA60934C0870934D0880938F
:10A460004E0890934F080091500810915108209188
:10A47000520830915308601B710B820B930B28EE2E
:10A4800033E040E050E00E9456B3CA01B9012CE32A
:10A4900030E040E050E00E9456B37F936F933F93CB
:10A4A0002F9384EA9BE09F938F93CE0101969F9315
:10A4B0008F930E9433B7ECEBFEE084910FB6F894D3
:10A4C000DEBF0FBECDBF882349F09091C00095FF3D
:10A4D000FCCF8093C60031968491F5CFFE01319672
:10A4E0008191882339F09091C00095FFFCCF809333
:10A4F000C600F6CF8091C00085FFFCCF8AE0809334
:10A50000C600CE0101960E941F730C94046283E57D
:10A510000E946B41882311F40C9404620E945741FD
:10A520000E94E7AFF62EE72E862F9E2D8C0180E548
:10A530000E946B41882331F00F3F110509F010F4A0
:10A540000C9462620DE010E0EFE8F4E081919191EB
:10A550008017910711F40C94046234E0E73CF30790
:10A56000A9F70630110539F48F2D9E2D90932D0AF1
:10A5700080932C0A04C017FF02C00C94046261E0AF
:10A58000802F0E9429A96F2D802F0E9462A96F2D14
:10A590007E2D802F0E941FA80C94046288E690E014
:10A5A00043D881110C94046283E50E946B41882397
:10A5B00071F000914B080E94574110E0000F111FED
:10A5C0000A5B174F0E94E7AFF801718360830E9416
:10A5D000BF210C9404620E944A4683E50E946B41AD
:10A5E000882311F40C9404620E9457410E94E7AF43
:10A5F00070934508609344080C94046289E690E0E7
:10A6000013D881110C940462EEE9FBE08491882355
:10A6100041F09091C00095FFFCCF8093C600319629
:10A62000F5CFE0914B0824E0E29FF0011124E25CB9
:10A63000F74F408151816281738121E030E08AE9E6
:10A640009DE00E94088CEBE9FBE08491882341F0B7
:10A650009091C00095FFFCCF8093C6003196F5CF56
:10A66000E0914B08F0E0EE0FFF1FEA5BF74F6081CF
:10A670007181882777FD8095982F0E941AB0AB01D1
:10A68000BC0121E030E08AE99DE00E94088CE7E906
:10A69000FBE08491882341F09091C00095FFFCCFAE
:10A6A0008093C6003196F5CF409138085091390813
:10A6B00060913A0870913B0821E030E08AE99DE022
:10A6C0000E94088CE4E9FBE08491882341F090919A
:10A6D000C00095FFFCCF8093C6003196F5CF609106
:10A6E000440870914508882777FD8095982F0E942F
:10A6F0001AB0AB01BC0121E030E08AE99DE00E9484
:10A70000088CE1E9FBE08491882341F09091C0003E
:10A7100095FFFCCF8093C6003196F5CF4AE050E01C
:10A7200060E070E08AE99DE00E94328BEFE8FBE098
:10A730008491882341F09091C00095FFFCCF8093D5
:10A74000C6003196F5CF40913E0850913F08609188
:10A7500040087091410821E030E08AE99DE00E94C4
:10A76000088CECE8FBE08491882341F09091C000D4
:10A7700095FFFCCF8093C6003196F5CF60914608D7
:10A7800070914708882777FD8095982F0E941AB00E
:10A79000AB01BC0121E030E08AE99DE00E94088C19
:10A7A000E8E8FBE08491882341F09091C00095FF98
:10A7B000FCCF8093C6003196F5CF80914B0890E096
:10A7C0000E94B71E4AE050E0BC018AE99DE00E9469
:10A7D000328BE3E8FBE08491882341F09091C00044
:10A7E00095FFFCCF8093C6003196F5CF8FEF9FEF9A
:10A7F0000E94B71E4AE050E0BC018AE99DE00E9439
:10A80000328B8091C00085FFFCCF8AE08093C60028
:10A810000C94C0638DE690E00E94144B81110C945F
:10A82000046286E79BE00E94D77683E50E946B4135
:10A83000882391F000914B080E94574110E0000FCF
:10A84000111F0A5B174F0E94E7AFF8017183608305
:10A8500081E080931C0215C082E50E946B41882331
:10A8600081F000914B080E94574110E0000F111F2A
:10A870000A5B174F0E94E7AFF80171836083109263
:10A880001C020E94BF210E9409AA4B015C01009199
:10A890004B0810E0F801EE0FFF1FEA5BF74F6081F5
:10A8A0007181882777FD8095982F0E941AB0F80152
:10A8B000EE0FFF1FEE0FFF1FE25CF74F11E020814C
:10A8C0003181428153810E947BB118160CF010E057
:10A8D0001093490810921D0ACC24CA94DC2C7601EE
:10A8E00048EE442E43E0542E612C712C5AE0352E54
:10A8F00080911D0A81110C947D63FFEFCF16DF0656
:10A90000EF06FF0611F40C946962F7FE02C00C9486
:10A910007D630E9409AA6C197D09683B7B4010F495
:10A920000C9469620C947D638CE49BE00E94D77662
:10A9300083E50E946B41882361F00E9457410E9489
:10A94000E7AF709345086093440881E080931C0250
:10A950000FC082E50E946B41882351F00E9457414D
:10A960000E94E7AF709345086093440810921C0260
:10A970000E9409AA4B015C0110921D0A60914408D3
:10A9800070914508882777FD8095982F0E941AB00E
:10A9900011E0209138083091390840913A085091DF
:10A9A0003B080E947BB118160CF010E01093490888
:10A9B00009E41BE0E5E4EE2EEBE0FE2EF1E4CF2E01
:10A9C000FBE0DF2EAAE07A2E8091490860914408CE
:10A9D00070914508882309F48BC080911D0A81116C
:10A9E00087C0882777FD8095982F0E941AB0209104
:10A9F00038083091390840913A0850913B080E943C
:10AA00007BB118160CF08BC00E9409AA681979094D
:10AA10008A099B09693E73408105910508F460C06D
:10AA2000E0912E0A84E0E89FF0011124E25CF74FE8
:10AA30004081518162817381F8018491E9E4FBE0F6
:10AA4000882349F09091C00095FFFCCF8093C60009
:10AA500031968491F5CF22E030E08AE99DE00E94B2
:10AA6000088CF7018491E5E4FBE0882349F090919C
:10AA7000C00095FFFCCF8093C60031968491F5CF3E
:10AA800060912E0A70E04AE050E08AE99DE00E9461
:10AA9000328BF6018491E1E4FBE0882349F0909148
:10AAA000C00095FFFCCF8093C60031968491F5CF0E
:10AAB000409138085091390860913A0870913B08EC
:10AAC00021E030E08AE99DE00E94088C8091C0007E
:10AAD00085FFFCCF7092C6000E9409AA4B015C0161
:10AAE0000E94ED1E80E00E94604A0E9473776CCF46
:10AAF000882777FD8095982F0E941AB020913808FA
:10AB00003091390840913A0850913B080E9478AF43
:10AB100087FF05C080911C02882309F475CF89E363
:10AB20009BE00E94D77680915D0A882321F08EE712
:10AB300093E00E941F730E9409AA609358087093C3
:10AB4000590880935A0890935B080C94046283E53B
:10AB50000E946B41882319F10E94574120E030E0A8
:10AB6000A9010E9478AF87FD0FC00E94574120E0E5
:10AB700030E04FE753E40E947BB1181644F00E9486
:10AB800057410E94E7AF05C060E070E002C06FEF80
:10AB900070E070932D0A60932C0A0C9404628FEF7E
:10ABA00090E090932D0A80932C0A0C9404621092EA
:10ABB0002D0A10922C0A0C9404629B9AA39881E0AF
:10ABC0008093260285E29BE00E94D7760E947377ED
:10ABD0000C9404620E94C0210E941594149A0E9451
:10ABE0007F9410922D0A10922C0A68EE73E080E098
:10ABF00090E00E9438AA9B9AA39A1092260287E1BD
:10AC00009BE00E94D7760E9473770C9404621092A6
:10AC10005A0A0C94046281E080935A0A0C940462EC
:10AC200083E50E946B418823A1F00E94574120E0F8
:10AC300030E04AE754E40E944DB20E94ECAF6093CA
:10AC40001D0270931E0280931F02909320020C94A9
:10AC5000046288E50E946B4181110C949E6389E532
:10AC60000E946B4181110C949E638AE50E946B41A6
:10AC700081110C949E6385E40E946B4181110C94B8
:10AC80009E630E941594149A0E947F940C9404620F
:10AC900083E50E946B41882311F40C9404620E94A6
:10ACA000574120E030E04AE754E40E944DB20E9450
:10ACB000ECAF6093540870935508809356089093B6
:10ACC00057080C94046227EC34E039AF28AF0FE941
:10ACD00013E16FEA862E63E1962E73E6A72E73E1E9
:10ACE000B72E312CE8ADF9AD8191F9AFE8AF0E94F4
:10ACF0006B41882309F45BC0F3E03F1251C00E940E
:10AD000057416B017C0120E030E040EA51E40E94B1
:10AD100078AF87FF3FC0A7019601F801608171817C
:10AD2000828193810E947FAF2B013C019B01AC018A
:10AD300060917713709178138091791390917A13C1
:10AD40000E944DB2609377137093781380937913B8
:10AD500090937A13A3019201F40160817181828141
:10AD600093810E944DB2F401608371838283938347
:10AD7000F50160817181828193810E9418B0A301E5
:10AD800092010E944DB20E94ECAFF5016083718385
:10AD900082839383F801C082D182E282F38207C06A
:10ADA0000E945741F80160837183828393833394B7
:10ADB0000C5F1F4FF4E08F0E911C24E0A20EB11C1B
:10ADC00034E033128FCF0C9404629091C00095FF51
:10ADD000FCCF8093C600319684918111F6CF0C94FC
:10ADE000046200915C0810915D080B5F1F4F6AE2DE
:10ADF00070E0C8010E94FBB6009711F0FC011082C0
:10AE0000C8010E941F730C940462ECE3FAE0849181
:10AE1000882341F09091C00095FFFCCF8093C6003D
:10AE20003196F5CF4091420A5091430A6091440A0D
:10AE30007091450A22E030E08AE99DE00E94088C8A
:10AE4000E8E3FAE08491882341F09091C00095FFF7
:10AE5000FCCF8093C6003196F5CF4091460A5091C1
:10AE6000470A6091480A7091490A22E030E08AE975
:10AE70009DE00E94088CE4E3FAE08491882341F08D
:10AE80009091C00095FFFCCF8093C6003196F5CF1E
:10AE900040914A0A50914B0A60914C0A70914D0AB8
:10AEA00022E030E08AE99DE00E94088CE0E3FAE0CD
:10AEB0008491882341F09091C00095FFFCCF80934E
:10AEC000C6003196F5CF40914E0A50914F0A6091DD
:10AED000500A7091510A22E030E08AE99DE00E9418
:10AEE000088CE5E2FAE08491882341F09091C0005B
:10AEF00095FFFCCF8093C6003196F5CF0E947194E8
:10AF00000E941AB020919F133091A0134091A11379
:10AF10005091A2130E947FAFAB01BC0122E030E050
:10AF20008AE99DE00E94088CE1E2FAE0849188239E
:10AF300041F09091C00095FFFCCF8093C600319600
:10AF4000F5CF81E00E9471940E941AB02091A31362
:10AF50003091A4134091A5135091A6130E947FAF86
:10AF6000AB01BC0122E030E08AE99DE00E94088C40
:10AF7000EDE1FAE08491882341F09091C00095FFC3
:10AF8000FCCF8093C6003196F5CF82E00E94719489
:10AF90000E941AB02091A7133091A8134091A913D1
:10AFA0005091AA130E947FAFAB01BC0122E030E0B8
:10AFB0008AE99DE00E94088C8091C00085FFFCCF4B
:10AFC0008AE08093C6000C94046280E00E94C98CE1
:10AFD0000C94046281E00E94C98C0C9404629091EC
:10AFE000C00095FFFCCF8093C60081918111F7CFFF
:10AFF0008091C00085FFFCCF8AE08093C600E5E128
:10B00000FAE08491882341F09091C00095FFFCCF35
:10B010008093C6003196F5CF1E9B03C0EBE0F4E0B1
:10B0200009C0E5E1F4E006C09091C00095FFFCCFB7
:10B030008093C60081918111F7CF8091C00085FF78
:10B04000FCCF8AE08093C600EDE0FAE0849188238B
:10B0500041F09091C00095FFFCCF8093C6003196DF
:10B06000F5CF029903C0EBE0F4E009C0E5E1F4E0BC
:10B0700006C09091C00095FFFCCF8093C6008191DF
:10B080008111F7CF8091C00085FFFCCF8AE08093CB
:10B09000C600E5E0FAE08491882341F09091C00079
:10B0A00095FFFCCF8093C6003196F5CF1D9B03C062
:10B0B000EBE0F4E009C0E5E1F4E006C09091C000E7
:10B0C00095FFFCCF8093C60081918111F7CF8091CD
:10B0D000C00085FFFCCF8AE08093C600EDEFF9E069
:10B0E0008491882341F09091C00095FFFCCF80931C
:10B0F000C6003196F5CF019903C0EBE0F4E009C03A
:10B10000E5E1F4E006C09091C00095FFFCCF80938C
:10B11000C60081918111F7CF8091C00085FFFCCFDF
:10B120008AE08093C600E5EFF9E08491882341F03E
:10B130009091C00095FFFCCF8093C6003196F5CF6B
:10B140001C9B03C0EBE0F4E009C0E5E1F4E006C0BD
:10B150009091C00095FFFCCF8093C6008191811132
:10B16000F7CF8091C00085FFFCCF8AE08093C600B6
:10B17000EDEEF9E08491882341F09091C00095FFB5
:10B18000FCCF8093C6003196F5CF379903C0EBE032
:10B19000F4E009C0E5E1F4E006C09091C00095FF3D
:10B1A000FCCF8093C60081918111F7CF8091C000C0
:10B1B00085FFFCCF8AE08093C6000C9404628091E6
:10B1C0002E0A80934B0884E50E946B41882319F175
:10B1D0000E9457410E94ECAF60934B086623D9F060
:10B1E000ECEBFEE08491882341F09091C00095FF44
:10B1F000FCCF8093C6003196F5CFE0E4F4E0819176
:10B20000882311F40C9404629091C00095FFFCCF48
:10B210008093C600F4CF84E40E946B41882311F42C
:10B220000C9404620E94574120E030E0A9010E9482
:10B2300078AF811103C01092520A32C000914B08BE
:10B2400010E00E945741F801EE0FFF1FEE0FFF1FA5
:10B25000ED5AFD4F6083718382839383E0905302A4
:10B26000F0905402009155021091560220E030E017
:10B27000A901B701C8010E9478AF811104C0E12C77
:10B28000F12C00E410E4C701D8018093530290939D
:10B290005402A0935502B093560281E08093520A63
:10B2A0000E94CF4B0C94046207EC14E04FE8E42EAC
:10B2B00043E1F42EF80181918F010E946B418823B4
:10B2C00049F00E9457410E94ECAFF70160837183FF
:10B2D00082839383F4E0EF0EF11C24E00B3C120711
:10B2E00049F70E94E8A50C94046207EC14E03FEAD9
:10B2F000E32E33E1F32EF80181918F010E946B411F
:10B30000882339F00E945741F7016083718382835B
:10B310009383F4E0EF0EF11C24E00B3C120759F785
:10B320000C94046283E50E946B41882351F00E94D3
:10B330005741609387137093881380938913909378
:10B340008A1384E50E946B41882311F40C940462F3
:10B350000E945741609383137093841380938513E5
:10B36000909386130C94046283E50E946B418823BA
:10B3700051F00E94574160938B1370938C1380930C
:10B380008D1390938E1384E50E946B41882351F0B6
:10B390000E945741609373137093741380937513D5
:10B3A0009093761382E40E946B41882361F00E949F
:10B3B00057410E94ECAF6093BF137093C01380930A
:10B3C000C1139093C21388E50E946B41882351F00A
:10B3D0000E94574160937F13709380138093811371
:10B3E000909382138AE50E946B41882351F00E945A
:10B3F000574160937B1370937C1380937D139093DC
:10B400007E1385E40E946B41882309F4FDC70E94E6
:10B4100057416093771370937813809379139093C7
:10B420007A13F2C707EC14E026E3E22E2AE0F22EAC
:10B43000F80181918F010E946B41882339F00E94AD
:10B440005741F7016083718382839383F4E0EF0EA9
:10B45000F11C24E00A3C120709F4D6C7E9CF83E5C2
:10B460000E946B41882351F00E9457416093330240
:10B4700070933402809335029093360286E40E94E2
:10B480006B41882381F00E94574120E030E040E783
:10B4900052E40E947FAF60932B0270932C02809342
:10B4A0002D0290932E028AE50E946B41882309F4B5
:10B4B000ABC70E9457416093260A7093270A809376
:10B4C000280A9093290AA0C783E50E946B4188232C
:10B4D00051F00E9457416093220A7093230A80938F
:10B4E000240A9093250A86E40E946B41882309F47C
:10B4F0008BC70E94574120E030E040E752E40E94B1
:10B500007FAF609327027093280280932902909363
:10B510002A027AC783E50E946B41882309F474C725
:10B520000E9457410E94E7AF6115710549F06130F3
:10B53000710559F481E080932B0A10922A0A64C79E
:10B5400010922B0A10922A0A5FC7ECEBFEE084915E
:10B55000882341F09091C00095FFFCCF8093C600F6
:10B560003196F5CFEAEDF9E08491882341F090918E
:10B57000C00095FFFCCF8093C6003196F5CF809137
:10B5800066089091670820E6289FF001299FF00D3A
:10B590001124E459F74F8191882339F09091C0002C
:10B5A00095FFFCCF8093C600F6CFE8EDF9E08491DB
:10B5B000882341F09091C00095FFFCCF8093C60096
:10B5C0003196F5CF8091C00085FFFCCF8AE0809353
:10B5D000C6001AC783E50E946B41882309F414C78B
:10B5E0000E9457410E94E7AF70935E0260935D0234
:10B5F0000BC783E50E946B41882309F405C70E94AD
:10B6000057410E94E7AF6B017C0184E50E946B41CA
:10B61000882381F08DED90E00E94144B8111F4C6D7
:10B62000E0914B08F0E0EE0FFF1FE75AFD4FD1828B
:10B63000C082EAC6D0925C02C0925B02E5C680E599
:10B640000E946B41882309F4DFC60E9457410E9483
:10B65000E7AFD62E062F172F83E50E946B41882374
:10B6600031F00E9457410E94E7AF7B0103C0EE24F6
:10B67000EA94FE2CC7010196039708F0C5C6EFE8CF
:10B68000F4E0819191918017910709F4BDC634E0EF
:10B69000E73CF307B1F717FDB7C60E941594CD2C10
:10B6A00060E08D2D0E9429A98FEFE816F80631F091
:10B6B000EA94EF2871F000E010E00DC08D2D0E949B
:10B6C00097A931E020E0892B09F030E0032F122FF9
:10B6D00002C001E010E08C2D0E9497A9801791070D
:10B6E00009F492C60E94ED1E80E00E94604A0E940A
:10B6F0007377F1CF83E50E946B41882331F00E947C
:10B7000057410E94E7AF8B0102C00EE610E080E5D2
:10B710000E946B41882331F00E9457410E94E7AF9D
:10B72000CB0102C088EE93E06C01EE24D7FCE094DC
:10B73000FE2C101611067CF420E030E0A901B801BF
:10B740008EE40E94D5AAC701B6010E9438AA8EE4F1
:10B750000E94E6AD59C6C701B6010E9438AA54C678
:10B7600080E50E946B41882351F00E94574160930D
:10B7700018027093190280931A0290931B0289E4B5
:10B780000E946B41882361F00E9457410E94322839
:10B79000609314027093150280931602909317021F
:10B7A00084E40E946B41882361F00E9457410E940B
:10B7B0003E286093100270931102809312029093BE
:10B7C000130283E40E946B41882351F00E94574189
:10B7D00060930C0270930D0280930E0290930F02FF
:10B7E0000E94A01EE7E5F4E08191882339F0909152
:10B7F000C00095FFFCCF8093C600F6CFEAE5F4E0E9
:10B800008191882339F09091C00095FFFCCF8093FF
:10B81000C600F6CF409118025091190260911A02A9
:10B8200070911B0222E030E08AE99DE00E94088CC2
:10B83000EEE5F4E08191882339F09091C00095FF06
:10B84000FCCF8093C600F6CF609114027091150270
:10B8500080911602909117020E943828AB01BC011A
:10B8600022E030E08AE99DE00E94088CE2E6F4E004
:10B870008191882339F09091C00095FFFCCF80938F
:10B88000C600F6CF609110027091110280911202F1
:10B89000909113020E944428AB01BC0122E030E0E9
:10B8A0008AE99DE00E94088CE6E6F4E08191882315
:10B8B00039F09091C00095FFFCCF8093C600F6CF81
:10B8C00040910C0250910D0260910E0270910F0296
:10B8D00022E030E08AE99DE00E94088C8091C0005F
:10B8E00085FFFCCF8AE08093C6008EC583E50E9469
:10B8F0006B41882319F00E94574103C060E070E05B
:10B90000CB010E94DFA580C585E40E946B4188239E
:10B9100041F00E9457410E94E7AF8B0177FF03C0BF
:10B9200009C000E010E0C12CD12CB6E1EB2EB3E44D
:10B93000FB2E06C0C12CD12CACE8EA2EA2E4FA2ED4
:10B9400083E50E946B41882321F00E9457416B01DF
:10B950007C0183E40E946B41882331F00E945741AF
:10B960000E94E7AF9B0102C025E030E0A801C701BB
:10B97000B6010E94D32148C50E94159445C50E9476
:10B98000398842C50E940B843FC58AE50E946B41FD
:10B99000882309F497C00E9457416B017C0120E085
:10B9A00030E040E751EC0E947BB187FD3FC020E0D2
:10B9B00030E040EA50ECC701B6010E9478AF18169B
:10B9C000ACF1F7FAF094F7F8F094C0922F0AD09205
:10B9D000300AE092310AF092320AECEBFEE08491F8
:10B9E000882341F09091C00095FFFCCF8093C60062
:10B9F0003196F5CFECECF9E08491882341F09091F9
:10BA0000C00095FFFCCF8093C6003196F5CF8091A2
:10BA1000C00085FFFCCF8AE08093C6008091C00003
:10BA200085FFFCCF8AE08093C600EEC4ECEBFEE01D
:10BA30008491882341F09091C00095FFFCCF8093C2
:10BA4000C6003196F5CFE3ECF9E08491882341F00C
:10BA50009091C00095FFFCCF8093C6003196F5CF42
:10BA6000EBEBF9E08491882341F09091C00095FFC1
:10BA7000FCCF8093C6003196F5CF4AE050E061EFED
:10BA80007FEF8AE99DE00E94328BE3EBF9E084913D
:10BA9000882341F09091C00095FFFCCF8093C600B1
:10BAA0003196F5CF4AE050E06BEF7FEF8AE99DE0F9
:10BAB0000E94328B8091C00085FFFCCF8AE080938A
:10BAC000C600A2C4ECEBFEE08491882341F0909183
:10BAD000C00095FFFCCF8093C6003196F5CFE7EA12
:10BAE000F9E08491882341F09091C00095FFFCCF4C
:10BAF0008093C6003196F5CF8091C00085FFFCCFC2
:10BB00008AE08093C60040912F0A5091300A6091DC
:10BB1000310A7091320A705822E030E08AE99DE0E3
:10BB20000E94088C8091C00085FFFCCF8AE0809342
:10BB3000C6006AC480915D0290915E0290935802A3
:10BB400080935702C090420AD090430AE090440A82
:10BB5000F090450ACF8ED8A2E9A2FAA20091460A37
:10BB60001091470A2091480A3091490A0BA31CA35F
:10BB70002DA33EA340914A0A50914B0A60914C0A72
:10BB800070914D0A4FA358A769A77AA780914E0AD2
:10BB900090914F0AA091500AB091510A8BA79CA78F
:10BBA000ADA7BEA7C982DA82EB82FC820D831E8319
:10BBB0002F83388749875A876B877C878D879E8735
:10BBC000AF87B88B85E40E946B41882359F00E94AF
:10BBD00057419B01AC016BA57CA58DA59EA50E943C
:10BBE0009FAE0AC020E030E040E050E46BA57CA5A9
:10BBF0008DA59EA50E949EAE6BA77CA78DA79EA734
:10BC0000EEE2CE2EEAE0DE2EE12CF12C08EC13E47D
:10BC10009E01255D3F4FAE01495D5F4FBE016D5DE9
:10BC20007F4FCE014F960E944F9B8AE50E946B4149
:10BC3000882349F00E9457419B01AC016FA178A570
:10BC400089A59AA51EC020E030E040E050E46FA135
:10BC500078A589A59AA50E949FAE6B017C016FA370
:10BC600078A789A79AA720E030E040E251E40E943B
:10BC700078AF87FF0CC020E030E040E251E4C7011C
:10BC8000B6010E949FAE6FA378A789A79AA76EE21C
:10BC9000C62E6AE0D62EE12CF12C06E913E49E01B3
:10BCA000255D3F4FAE01495D5F4FBE016D5D7F4F2A
:10BCB000CE014F960E944F9B88E50E946B418823DE
:10BCC00079F00E9457419B01AC016F8D78A189A149
:10BCD0009AA10E949FAE6F8F78A389A39AA308C0F0
:10BCE00080E090E0A3E5B3E48F8F98A3A9A3BAA363
:10BCF00089E50E946B41882339F00E9457416BA36C
:10BD00007CA38DA39EA304C01BA21CA21DA21EA2E5
:10BD10004EE2C42E4AE0D42EE12CF12C0CE812E4C1
:10BD20009E01255D3F4FAE01495D5F4FBE016D5DD8
:10BD30007F4FCE014F960E944F9B8CE40E946B4137
:10BD4000882359F00E9457419B01AC016BA57CA54B
:10BD50008DA59EA50E949FAE0AC020E030E040EA7B
:10BD600052E46BA57CA58DA59EA50E949EAE6BA7F7
:10BD70007CA78DA79EA72EE2C22E2AE0D22EE12C10
:10BD8000F12C00EA11E49E01255D3F4FAE01495DB3
:10BD90005F4FBE016D5D7F4FCE014F960E944F9B5E
:10BDA0000E941594149A64E670E080E090E00E948E
:10BDB00038AA0E94597200E010E0F12C0E943978F4
:10BDC00081111BC0F3940E94ED1E81E00E94604A25
:10BDD000F110F4CF043FE1E01E0711F400E010E0A1
:10BDE0006A9A0115110511F4729A04C00431110503
:10BDF00009F472980F5F1F4FE1CF729820E030E096
:10BE00004CE852E46BA57CA58DA59EA50E949FAE33
:10BE10006BA77CA78DA79EA71EE2C12E1AE0D12E8C
:10BE2000E12CF12C00EA11E49E01255D3F4FAE01AB
:10BE3000495D5F4FBE016D5D7F4FCE014F960E9401
:10BE40004F9B20E030E048E452E46BA57CA58DA533
:10BE50009EA50E949FAE6BA77CA78DA79EA7E12CF5
:10BE6000F12C00E010E49E01255D3F4FAE01495DDD
:10BE70005F4FBE016D5D7F4FCE014F960E944F9B7D
:10BE80001092540A1092530A0E94BF728091530A72
:10BE90009091540A019709F47CC01092540A1092B0
:10BEA000530A0E943F788091530A9091540A82303D
:10BEB000910549F1039709F069C020E030E048E4BA
:10BEC00052E46BA57CA58DA59EA50E949FAE6BA795
:10BED0007CA78DA79EA77EE2C72E7AE0D72EE12C05
:10BEE000F12C00E010E49E01255D3F4FAE01495D5D
:10BEF0005F4FBE016D5D7F4FCE014F960E944F9BFD
:10BF00000E947F72C3CF20E030E04CE852E46BA582
:10BF10007CA58DA59EA50E949FAE6BA77CA78DA733
:10BF20009EA7FEE2CF2EFAE0DF2EE12CF12C00EAF4
:10BF300011E49E01255D3F4FAE01495D5F4FBE019B
:10BF40006D5D7F4FCE014F960E944F9B20E030E009
:10BF500048E452E46BA57CA58DA59EA50E949FAEEA
:10BF60006BA77CA78DA79EA7E12CF12C00E010E425
:10BF70009E01255D3F4FAE01495D5F4FBE016D5D86
:10BF80007F4FCE014F960E944F9B7ECF0E947272D0
:10BF90007DCF20E030E040EA50E46BA57CA58DA584
:10BFA0009EA50E949FAE6BA77CA78DA79EA79EE231
:10BFB000C92E9AE0D92EE12CF12C00E010E49E016C
:10BFC000255D3F4FAE01495D5F4FBE016D5D7F4F07
:10BFD000CE014F960E944F9BA80197016BA57CA5AF
:10BFE0008DA59EA50E949EAE6BA77CA78DA79EA740
:10BFF000E12CF12C08EC13E49E01255D3F4FAE01CE
:10C00000495D5F4FBE016D5D7F4FCE014F960E942F
:10C010004F9BE12CF12C0CE812E49E01255D3F4F73
:10C02000AE01495D5F4FBE016D5D7F4FCE014F9602
:10C030000E944F9B9E01255D3F4FAE01495D5F4FC2
:10C04000BE016B5F7F4FCE0101960E944F9BE12C9A
:10C05000F12C08E413E49E01255D3F4FAE01475FDC
:10C060005F4FBE016B5F7F4FCE0101960E944F9BD9
:10C0700020E030E040E050E46BA57CA58DA59EA5B6
:10C080000E949FAE6BA77CA78DA79EA7E12CF12CE9
:10C0900000EA10E49E01255D3F4FAE01475F5F4F10
:10C0A000BE016B5F7F4FCE0101960E944F9BCE0178
:10C0B0000D960E94BBA580915702909158028093E3
:10C0C0005D0290935E029F938F938EE999E09F9318
:10C0D0008F938E01015D1F4F1F930F930E9433B703
:10C0E000C8010E94E83E0F900F900F900F900F90A4
:10C0F0000F908AC188E50E946B41882339F00E9425
:10C1000057410E94E7AF80E00E941D958AE50E949A
:10C110006B41882339F00E9457410E94E7AF81E0CC
:10C120000E941D9585E40E946B41882309F46CC12F
:10C130000E9457410E94E7AF82E00E941D9564C1B2
:10C1400083E50E946B41811104C007EC14E0F12CDF
:10C1500010C010E00E9457410E94ECAF812F0E9456
:10C16000BC951F5F1530B1F7F0CFF394F4E0FF16E4
:10C1700079F0F80181918F010E946B418823A9F326
:10C180000E9457410E94ECAF8F2D0E94BC95EDCFCD
:10C1900082E40E946B41882339F00E9457410E943B
:10C1A000ECAF84E00E94BC950E9482962DC183E58D
:10C1B0000E946B41882309F453C00E9457410E949A
:10C1C000E7AF6130710541F06230710509F048C098
:10C1D00007EC14E0F12C25C007EC14E0F12CF80179
:10C1E00081918F010E946B41882341F00E94574149
:10C1F0000E94E7AF4FEF8F2D0E947E95F394F4E0FD
:10C20000FF12EDCF82E40E946B41882349F10E9426
:10C2100057410E94E7AF4FEF20C0F394F4E0FF16C0
:10C2200089F0F80181918F010E946B418823A9F365
:10C230000E9457410E94E7AF462F6FEF8F2D0E945B
:10C240007E95EBCF82E40E946B41882349F00E94E7
:10C2500057410E94E7AF462F6FEF84E00E947E9522
:10C260000E948296D1C084E50E946B41882309F424
:10C2700087C00E9457410E94ECAF60934B08662331
:10C28000A9F1ECEBFEE08491882341F09091C0008D
:10C2900095FFFCCF8093C6003196F5CFEAE6F4E037
:10C2A0008191882339F09091C00095FFFCCF809355
:10C2B000C600F6CF40E050E060914B088AE99DE06F
:10C2C0000E94698BECE6F4E08191882339F090912B
:10C2D000C00095FFFCCF8093C600F6CF8091C000D0
:10C2E00085FFFCCF8AE08093C6008EC086E40E9462
:10C2F0006B418823D9F00E9457416B017C01609308
:10C30000FD097093FE098093FF099093000A20E0D5
:10C3100030E0A9010E947BB1181644F4C0922102BA
:10C32000D0922202E0922302F0922402ECEBFEE093
:10C330008491882341F09091C00095FFFCCF8093B9
:10C34000C6003196F5CFEDE7F4E08191882339F00E
:10C350009091C00095FFFCCF8093C600F6CF60910E
:10C360002E0A70E04AE050E08AE99DE00E94328B9C
:10C370008091C00085FFFCCF8AE08093C60044C056
:10C38000ECEBFEE08491882341F09091C00095FF92
:10C39000FCCF8093C6003196F5CFEBE8F9E08491AD
:10C3A000882341F09091C00095FFFCCF8093C60098
:10C3B0003196F5CF809166089091670820E6289F16
:10C3C000F001299FF00D1124E459F74F8191882342
:10C3D00039F09091C00095FFFCCF8093C600F6CF56
:10C3E000E9E8F9E08491882341F09091C00095FF3D
:10C3F000FCCF8093C6003196F5CF8091C00085FFB9
:10C40000FCCF8AE08093C6000E949241B9C1C090DF
:10C41000190AD0901A0AE0901B0AF0901C0A209189
:10C420004E0A30914F0A4091500A5091510AC7016B
:10C43000B6010E949EAE2DEC3CEC4CEC5DE30E94FC
:10C440007BB1181614F00C94904CC0924E0AD09206
:10C450004F0AE092500AF092510A8EE49AE00E944C
:10C46000BBA560E080E00E94EA438AC180E090E0E2
:10C470000E94563D0C948D4D81E090E00E94563D07
:10C480000C94984D82E090E00E94563D0C94E14D52
:10C490000E94ED1E80E00E94604A0E9473770C9417
:10C4A00080500E946041AB01BC014093F80C509356
:10C4B000F90C6093FA0C7093FB0C83E49CE00E94EF
:10C4C0002413A2CF0E9457410E94E7AF8B010C9426
:10C4D000A4520E9409AA681979098A099B09693E30
:10C4E00073408105910508F479C0E3E7FBE084918E
:10C4F000882341F09091C00095FFFCCF8093C60047
:10C500003196F5CFE0914B0824E0E29FF001112431
:10C51000E25CF74F408151816281738121E030E01C
:10C520008AE99DE00E94088CEFE6FBE08491882375
:10C5300041F09091C00095FFFCCF8093C6003196EA
:10C54000F5CF60914B0870E04AE050E08AE99DE049
:10C550000E94328BEBE6FBE08491882341F09091BE
:10C56000C00095FFFCCF8093C6003196F5CFF7FE53
:10C5700003C0E3E7F5E025C00E9409AA8B019C01F6
:10C58000C701B6016854744F8F4F9F4F601B710BEA
:10C59000820B930BA30192010E9456B3BA01A90129
:10C5A0002AE030E08AE99DE00E945E8B8091C00025
:10C5B00085FFFCCF0DC09091C00095FFFCCF80930C
:10C5C000C60081918111F7CF8091C00085FFFCCF1B
:10C5D0003092C6000E9409AA4B015C010E94ED1E28
:10C5E00080E00E94604A0E947377FFEFCF16DF065B
:10C5F000EF06FF0609F046C080914908E0914B081C
:10C60000F0E08F01000F111F000F111F025C174F88
:10C61000EE0FFF1FEA5BF74F608171818823C9F03D
:10C62000882777FD8095982F0E941AB020E030E08F
:10C6300040E85FE30E949EAE9B01AC01F80160817F
:10C640007181828193810E947BB187FF50C00C94DD
:10C650007854882777FD8095982F0E941AB020E0A3
:10C6600030E040E85FE30E949FAE9B01AC01F8011F
:10C6700060817181828193810E9478AF1816BCF528
:10C680000C947854F7FE02C00C947854E0914B0857
:10C69000F0E08F01000F111F000F111F025C174FF8
:10C6A000EE0FFF1FEA5BF74F60817181882777FDEE
:10C6B0008095982F0E941AB09B01AC01F80160810F
:10C6C0007181828193810E949EAE0E94E7AF97FFA5
:10C6D00007C090958095709561957F4F8F4F9F4FC4
:10C6E000663071058105910514F40C9478540E940C
:10C6F00009AA6B017C010C9478548DE59BE00E94A3
:10C70000D77680915D0A882321F08EE793E00E941E
:10C710001F730E9409AA6093500870935108809378
:10C720005208909353080E9409AA60935808709386
:10C73000590880935A0890935B0866CE0E9415941E
:10C7400088E50E946B41882319F0179A1092330AEA
:10C7500089E50E946B41882319F0169A1092340AD9
:10C760008AE50E946B41882319F0159A1092350AC8
:10C7700085E40E946B41882309F446CE149A44CE86
:10C78000E9960FB6F894DEBF0FBECDBFDF91CF9113
:10C790001F910F91FF90EF90DF90CF90BF90AF90DF
:10C7A0009F908F907F906F905F904F903F900895F3
:10C7B000CF93DF938091620890916308039714F4FC
:10C7C0000E94914660E08BE59AE00E94AF34809130
:10C7D000620890916308892B09F464C080915B0A18
:10C7E0008823E1F0809166089091670820E6289FF1
:10C7F000E001299FD00D1124C459D74F6EE77DE089
:10C80000CE010E94A6B6892BF1F4BE018BE59AE019
:10C810000E943E3480915C0A882319F00E94E14B0B
:10C820002BC0EBE7FDE08491882341F09091C0009C
:10C8300095FFFCCF8093C6003196F5CF8091C00064
:10C8400085FFFCCF16C060E08BE59AE00E94A5351D
:10C85000E9E6FDE08491882341F09091C00095FFC6
:10C86000FCCF8093C6003196F5CF8091C00085FF44
:10C87000FCCF8AE08093C6008091620890916308A3
:10C880000197909363088093620880916608909165
:10C890006708019664E070E00E9443B390936708D4
:10C8A000809366080E94ED1E80E00E94604A0E940C
:10C8B000278CDF91CF910C9473778F929F92AF92D8
:10C8C000BF92CF92DF92EF92FF920F931F93CF937D
:10C8D000DF938C018C519E4F0E94522E680189E893
:10C8E000C80ED11C21F1780181E4E81A8EEFF80A14
:10C8F000E70157018FE1A81AB10877EB872E75E0A1
:10C90000972ECC15DD0599F0FE01EE19FF09EA0D11
:10C91000FB1D91828082FE0178978081811102C087
:10C920006F97EFCFCE014B970E940714F9CFC80144
:10C9300086599F4F0E94522EC801875B9F4FDF91FF
:10C94000CF911F910F91FF90EF90DF90CF90BF900C
:10C95000AF909F908F900C94522E8BE59AE00C94A0
:10C960005E2E8BE59AE0A9CFFB0160917002709179
:10C97000710270932A0D6093290D6091330D7091AF
:10C98000340D7093280D6093270D62E060936F0261
:10C9900066E97FE770937102609370029093260DB1
:10C9A0008093250DF093240DE093230D662757FD0A
:10C9B0006095762F40931F0D5093200D6093210DAD
:10C9C0007093220DC901AA2797FDA095BA2F841B49
:10C9D000950BA60BB70B80931B0D90931C0DA0938A
:10C9E0001D0DB0931E0D80819181AA2797FDA09502
:10C9F000BA2F841B950BA60BB70B8093330D909326
:10CA0000340DA093350DB093360D08950F931F93F9
:10CA1000CF93DF93EB01142F022F482F60E08EE3BA
:10CA20009DE00E94F928612F8EE39DE00E9497AE61
:10CA300011E1FE016491662311F0111117C0112359
:10CA400039F060E28EE39DE00E9497AE1150F7CF7F
:10CA5000602F8EE39DE00E9497AE60E28EE39DE042
:10CA6000DF91CF911F910F910C9497AE8EE39DE0D3
:10CA70000E9497AE21961150DCCFEF92FF920F9358
:10CA80001F93CF93DF93EB01E42E8901F90101900D
:10CA90000020E9F7F22EFE1A92E1F90E482F60E02D
:10CAA0008EE39DE00E94F9286E2D8EE39DE00E94AA
:10CAB00097AEFE016491662311F0F11019C06AE38C
:10CAC0008EE39DE00E9497AEFF2039F060E28EE396
:10CAD0009DE00E9497AEFA94F7CFB8018EE39DE0F7
:10CAE000DF91CF911F910F91FF90EF900C9496AE34
:10CAF0008EE39DE00E9497AE2196FA94DACF1092D1
:10CB0000970D8BE59AE00E944F3A10923C0D0895E4
:10CB10008BE59AE00C94B1318BE59AE00C94B83136
:10CB2000CF93DF93CDB7DEB7C054D1090FB6F894D9
:10CB3000DEBF0FBECDBF88E0EFEAF2E0DE01D9969E
:10CB400001900D928A95E1F788E0E7EBF2E0DE01D3
:10CB5000D19601900D928A95E1F788E0EFEBF2E033
:10CB6000DE01999601900D928A95E1F788E0E7EC55
:10CB7000F2E0DE01919601900D928A95E1F788E04E
:10CB8000EFECF2E0DE01599601900D928A95E1F703
:10CB900088E0E7EDF2E0DE01519601900D928A9572
:10CBA000E1F788E0EFEDF2E0DE01199601900D92D9
:10CBB0008A95E1F788E0E7EEF2E0DE011196019058
:10CBC0000D928A95E1F7AE01475C5F4F60E08EE31E
:10CBD0009DE00E94972AAE014F5C5F4F61E08EE3BB
:10CBE0009DE00E94972AAE01475D5F4F62E08EE3B1
:10CBF0009DE00E94972AAE014F5D5F4F63E08EE398
:10CC00009DE00E94972AAE01475E5F4F64E08EE38D
:10CC10009DE00E94972AAE014F5E5F4F65E08EE374
:10CC20009DE00E94972AAE01475F5F4F66E08EE36A
:10CC30009DE00E94972AAE014F5F5F4F67E08EE351
:10CC40009DE00E94972AC05CDF4F0FB6F894DEBFCC
:10CC50000FBECDBFDF91CF910895CF9382E0809337
:10CC60006F020E9409AA6C507E4F8F4F9F4F6093B6
:10CC7000380D7093390D80933A0D90933B0D6A9A5D
:10CC8000CAE0729A84E690E00E945CAA729884E6F8
:10CC900090E00E945CAAC150A1F7CF910895E09165
:10CCA0007002F0917102E817F90771F09093710228
:10CCB000809370024093330D5093340D6093350D83
:10CCC0007093360D2111C9CF089521E040E050E066
:10CCD000BA01E5CF21E040E050E0BA01E0CF8F9209
:10CCE0009F92AF92BF92CF92DF92EF92FF920F93FB
:10CCF0001F93CF93DF938091330D9091340DA091CA
:10CD0000350DB091360D81309048A105B10540F048
:10CD10001092330D1092340D1092350D1092360D85
:10CD20006091330D7091340D8091350D9091360DD9
:10CD300025E030E040E050E00E9456B380913C0D89
:10CD400090E0A0E0B0E0281739074A075B0710F42D
:10CD500020933C0DD0913C0D10913D0D12FB1127FD
:10CD600010F9C0E085E0C82ED12CE12CF12C9DE11A
:10CD7000892E912CA12CB12C01E06091330D709182
:10CD8000340D8091350D9091360DD11131C0209127
:10CD90006F02222369F023E065307105810591055A
:10CDA00010F443E001C040E267E671E18C2F2EDE13
:10CDB000112309F400C18091330D9091340DA0919D
:10CDC000350DB091360D0597A105B10508F0F3C0FA
:10CDD00044DF83E493E7DF91CF911F910F91FF90A0
:10CDE000EF90DF90CF90BF90AF909F908F906DCFDE
:10CDF000D13061F520916F02222391F0A7019601B5
:10CE00000E9456B3213031054105510519F423E044
:10CE100043E002C023E040E266E571E18C2FF6DDDD
:10CE2000112309F4C8C06091330D7091340D8091C5
:10CE3000350D9091360DA70196010E9456B3213011
:10CE400031054105510509F0B6C0C2CFD23061F5B8
:10CE500020916F02222391F0A70196010E9456B300
:10CE6000223031054105510519F423E043E002C0A9
:10CE700023E040E26AE471E18C2FC8DD112309F45C
:10CE80009AC06091330D7091340D8091350D909161
:10CE9000360DA70196010E9456B322303105410597
:10CEA000510509F088C094CFD33061F520916F020D
:10CEB000222391F0A70196010E9456B32330310539
:10CEC0004105510519F423E043E002C023E040E2AC
:10CED00068E371E18C2F9ADD112309F46CC0609135
:10CEE000330D7091340D8091350D9091360DA70161
:10CEF00096010E9456B3233031054105510509F0D2
:10CF00005AC066CFD43059F520916F02222391F098
:10CF1000A70196010E9456B3243031054105510501
:10CF200019F423E043E002C023E040E266E271E14D
:10CF30008C2F6CDD112309F43EC06091330D70918C
:10CF4000340D8091350D9091360DA70196010E9408
:10CF500056B3243031054105510569F539CFD53037
:10CF600051F520916F02222391F0A70196010E94B2
:10CF700056B3253031054105510519F423E043E04E
:10CF800002C023E040E26AE171E18C2F3FDD112312
:10CF900091F06091330D7091340D8091350D909129
:10CFA000360DA70196010E9456B325303105410583
:10CFB000510509F40DCF8091330D9091340DA0915E
:10CFC000350DB091360D4E97A105B10540F0809218
:10CFD000330D9092340DA092350DB092360D6091C4
:10CFE000330D7091340D8091350D9091360DA70160
:10CFF00096010E9456B380913C0D90E00396422F1B
:10D0000050E0841795074CF48DEF820F80933C0D10
:10D0100000936F02DCEFD20FCFEFCF5FDF5FC43042
:10D0200008F4ABCEDF91CF911F910F91FF90EF905D
:10D03000DF90CF90BF90AF909F908F9008958F9288
:10D040009F92AF92BF92CF92DF92EF92FF920F9397
:10D050001F93CF93DF938091330D9091340DA09166
:10D06000350DB091360D81309048A105B10540F0E5
:10D070001092330D1092340D1092350D1092360D22
:10D080006091330D7091340D8091350D9091360D76
:10D0900025E030E040E050E00E9456B380913C0D26
:10D0A00090E0A0E0B0E0281739074A075B0710F4CA
:10D0B00020933C0DD0913C0D10913D0D12FB11279A
:10D0C00010F9C0E025E0C22ED12CE12CF12C3DE17D
:10D0D000832E912CA12CB12C01E06091330D709125
:10D0E000340D8091350D9091360DD11131C02091C4
:10D0F0006F02222369F023E06530710581059105F7
:10D1000010F443E001C040E26BE071E18C2F7EDC63
:10D11000112309F429C18091330D9091340DA09110
:10D12000350DB091360D0597A105B10508F01CC16C
:10D1300094DD83E493E7DF91CF911F910F91FF90EE
:10D14000EF90DF90CF90BF90AF909F908F90BDCD2C
:10D15000D13079F520916F02222391F0A701960139
:10D160000E9456B3213031054105510519F42EE7CF
:10D170004EE302C02EE740E263E071E18C2F46DC13
:10D18000112309F4F1C06091330D7091340D809139
:10D19000350D9091360DA70196010E9456B32130AE
:10D1A00031054105510509F0DFC057DD8DE79AE7EC
:10D1B00030C0D230D9F520916F02222391F0A7011F
:10D1C00096010E9456B3223031054105510519F4EC
:10D1D0002EE74EE302C02EE740E266EF70E18C2FAF
:10D1E00015DC112309F4C0C06091330D7091340D2A
:10D1F0008091350D9091360DA70196010E9456B38E
:10D20000223031054105510509F0AEC026DD8DEA19
:10D210009BE6DF91CF911F910F91FF90EF90DF90F0
:10D22000CF90BF90AF909F908F9054CDD33079F531
:10D2300020916F02222391F0A70196010E9456B31C
:10D24000233031054105510519F420E24EE302C0B7
:10D2500020E240E269EE70E18C2FD8DB112309F463
:10D2600083C06091330D7091340D8091350D909194
:10D27000360DA70196010E9456B3233031054105B2
:10D28000510509F071C0E9DC83EE90E15FC0D43054
:10D2900079F520916F02222391F0A70196010E9457
:10D2A00056B3243031054105510519F420E24EE30F
:10D2B00002C020E240E264ED70E18C2FA7DB112375
:10D2C00009F452C06091330D7091340D8091350D89
:10D2D0009091360DA70196010E9456B32430310576
:10D2E0004105510509F040C0B8DC80ED90E12EC049
:10D2F000D530D1F520916F02222391F0A70196013C
:10D300000E9456B3253031054105510519F420E23C
:10D310004EE302C020E240E266EC70E18C2F76DB47
:10D32000112311F16091330D7091340D8091350D01
:10D330009091360DA70196010E9456B32530310514
:10D340004105510589F489DC82EC90E1DF91CF91B0
:10D350001F910F91FF90EF90DF90CF90BF90AF9013
:10D360009F908F900C945B3F8091330D9091340D82
:10D37000A091350DB091360D4E97A105B10540F045
:10D380008092330D9092340DA092350DB092360DEF
:10D390006091330D7091340D8091350D9091360D63
:10D3A000A70196010E9456B380913C0D90E0039630
:10D3B000422F50E0841795074CF48DEF820F809335
:10D3C0003C0D00936F02DCEFD20FCFEFCF5FDF5F3A
:10D3D000C43008F482CEDF91CF911F910F91FF905E
:10D3E000EF90DF90CF90BF90AF909F908F90089577
:10D3F000BF92CF92DF92EF92FF920F931F93CF9342
:10D40000DF938091330D9091340DA091350DB09143
:10D41000360D81309048A105B10540F01092330DD2
:10D420001092340D1092350D1092360D6091330D1F
:10D430007091340D8091350D9091360D25E030E0DE
:10D4400040E050E00E9456B380913C0D90E0A0E097
:10D45000B0E0281739074A075B0710F420933C0D0A
:10D46000D0913C0D10913D0D12FB112710F9C0E039
:10D4700065E0C62ED12CE12CF12C01E06091330D3A
:10D480007091340D8091350D9091360DD1112EC0D3
:10D4900020916F02222369F023E065307105810538
:10D4A000910510F443E001C040E268EB70E18C2F7D
:10D4B000ADDA112309F479C08091330D9091340DC8
:10D4C000A091350DB091360D0597A105B10508F075
:10D4D0006CC0C3DB8FE198E6DF91CF911F910F9174
:10D4E000FF90EF90DF90CF90BF90EFCBD13071F5F0
:10D4F00020916F02222391F0A70196010E9456B35A
:10D50000213031054105510519F42EE74EE302C0E3
:10D510002EE740E26DEA70E18C2F78DA112309F4EE
:10D5200044C06091330D7091340D8091350D909110
:10D53000360DA70196010E9456B3213031054105F1
:10D54000510599F58ADB81EE90E8A8C0D23069F5E3
:10D5500020916F02222391F0A70196010E9456B3F9
:10D56000223031054105510519F42EE74EE302C082
:10D570002EE740E262EA70E18C2F48DA1123A9F02D
:10D580006091330D7091340D8091350D9091360D71
:10D59000A70196010E9456B322303105410551057D
:10D5A00021F45BDB88EE90E879C020E030E040E2D7
:10D5B00051E460910F0D7091100D8091110D9091BB
:10D5C000120D0E9478AF87FF73C06091330D709188
:10D5D000340D8091350D9091360DD33081F5209129
:10D5E0006F02222391F0A70196010E9456B32330C7
:10D5F00031054105510519F42EE74EE302C02EE72F
:10D6000040E267E970E18C2F01DA111103C055E0A7
:10D61000B52E50C06091330D7091340D8091350D51
:10D620009091360DA70196010E9456B32330310523
:10D630004105510561F711DB8FEE90E82FC0D43022
:10D6400031F720916F02222391F0A70196010E94E9
:10D6500056B3243031054105510519F42EE74EE348
:10D6600002C02EE740E26EE870E18C2FCFD9112383
:10D6700071F26091330D7091340D8091350D909160
:10D68000360DA70196010E9456B32430310541059D
:10D69000510509F0BCCFE1DA8DE19FE7DF91CF9131
:10D6A0001F910F91FF90EF90DF90CF90BF9012CB22
:10D6B00043E0B42E6091330D7091340D8091350D9F
:10D6C0009091360DA70196010E9456B38B2D90E0E4
:10D6D000A0E0B0E0281739074A075B0788F025E08B
:10D6E000B29EC00111240197AA2797FDA095BA2FD9
:10D6F0008093330D9093340DA093350DB093360D78
:10D700006091330D7091340D8091350D9091360DEF
:10D71000A70196010E9456B380913C0D90E00396BC
:10D72000422F50E0841795074CF48DEF820F8093C1
:10D730003C0D00936F02DCEFD20FCFEFCF5FDF5FC6
:10D74000C43008F49BCEDF91CF911F910F91FF90D1
:10D75000EF90DF90CF90BF90089580E090E0A0E838
:10D76000BFE380930F0D9093100DA093110DB09314
:10D77000120D3ECE20E044E064E18EE39DE00E9485
:10D780002C29CED98EE39DE00C94ED28F3DF20E028
:10D7900040E050E0BA0186EF90E881CA1092470855
:10D7A00010924608109245081092440810922D0AD3
:10D7B00010922C0AEBCF8EE39DE00C94ED2820E034
:10D7C00030E04EE353E460913E0870913F08809151
:10D7D0004008909141080E947BB118164CF48EE0ED
:10D7E0009FE00E945B3F81E09FE00E945B3F20C082
:10D7F000E2DF40E060E08EE39DE00E94F9286BEC00
:10D8000074E08EE39DE00E9496AE42E060E08EE31D
:10D810009DE00E94F92862ED74E08EE39DE00E9495
:10D8200096AE60ED77E080E090E00E9438AAC3DF1A
:10D83000ADCF20E030E04EE353E460913E087091BC
:10D840003F0880914008909141080E947BB11816D2
:10D850006CF48DEF9EE00E945B3F81EF9EE00E94A2
:10D860005B3F85EE9EE00E945B3F20C0A4DF40E06E
:10D8700060E08EE39DE00E94F9286BEC74E08EE39B
:10D880009DE00E9496AE42E060E08EE39DE00E9443
:10D89000F92862ED74E08EE39DE00E9496AE60EDA3
:10D8A00077E080E090E00E9438AA85DF6FCF80911A
:10D8B000950D9091960D909347088093460880911E
:10D8C000930D9091940D9093450880934408109285
:10D8D0002D0A10922C0A5ADF0C94BF2180918F0DD3
:10D8E0009091900D909347088093460880918D0DFC
:10D8F00090918E0D909345088093440810922D0AC4
:10D9000010922C0A43DF0C94BF21809195029091D4
:10D9100096029093470880934608809193029091D5
:10D920009402909345088093440810922D0A109217
:10D930002C0A2CDF0C94BF218091910290919202CD
:10D94000909347088093460880918F0290919002AF
:10D95000909345088093440810922D0A10922C0A47
:10D9600015DF0C94BF2180918D0290918E029093CF
:10D9700047088093460880918B0290918C02909387
:10D9800045088093440810922D0A10922C0AFEDE5E
:10D990000C94BF218091890290918A02909347084C
:10D9A0008093460880918702909188029093450861
:10D9B0008093440810922D0A10922C0AE7DE0C94F2
:10D9C000BF212F923F924F925F926F927F928F92E0
:10D9D0009F92AF92BF92CF92DF92EF92FF920F93FE
:10D9E0001F93CF93DF93CDB7DEB7A6970FB6F8940A
:10D9F000DEBF0FBECDBF80916F02811104C0809148
:10DA00003D0D82FFC4C28BE59AE00E9443398C0130
:10DA10008091330D9091340DA091350DB091360D5C
:10DA200081309048A105B10540F01092330D10925D
:10DA3000340D1092350D1092360D6091330D7091AA
:10DA4000340D8091350D9091360D25E030E040E0A9
:10DA500050E00E9456B380913C0D90E0A0E0B0E011
:10DA6000281739074A075B0710F420933C0D2090D4
:10DA70003C0D80913D0D82FB882780F98F8F312CE2
:10DA800085E0C82ED12CE12CF12CC80101979BA375
:10DA90008AA321102DC080916F028823A9F0809164
:10DAA000330D9091340DA091350DB091360D23E0DA
:10DAB0000597A105B10510F443E001C040E262E31F
:10DAC00070E1832D0E9406659F8D992389F08091D6
:10DAD000330D9091340DA091350DB091360D059711
:10DAE000A105B10528F4B9D883E493E7EED84FC275
:10DAF0006FE57AE089EC9AE00E94BB1080915F0AA2
:10DB00008F3229F0E1E02E1669F012E001C011E039
:10DB1000AAA0BBA0422C512C612C712CF1E0F20D7B
:10DB2000F8A351C080916F028823D9F06091330D22
:10DB30007091340D8091350D9091360DA7019601AD
:10DB40000E9456B3213031054105510519F420E2F8
:10DB50004EE302C020E240E26EE270E1832D0E94BB
:10DB600006652F8D222389F26091330D7091340D5B
:10DB70008091350D9091360DA70196010E9456B304
:10DB8000213031054105510509F0BFCF66D80E940B
:10DB90007F65FDC1121163C140E050E0B5018BE526
:10DBA0009AE00E94BA359091A10A80916F02992360
:10DBB00009F49EC081110CC08F8D811176C018A10F
:10DBC000F1E0AF1AB1082FEFA216B20619F749C15A
:10DBD0006091330D7091340D8091350D9091360D1B
:10DBE000A70196010E9456B3241535054605570531
:10DBF00071F5432D60E08EE39DE00E94F9286EE30D
:10DC00008EE39DE00E9497AE65E08EE39DE00E946A
:10DC100097AE80916C0A882329F010927E0A0CE658
:10DC20001AE002C00FE51AE0B2E19B2EF801619103
:10DC30008F01662311F0911062C1992009F4BCCFC5
:10DC400060E28EE39DE00E9497AE9A94F6CF432D5A
:10DC500060E08EE39DE00E94F92860E28EE39DE0A3
:10DC60000E9497AE65E08EE39DE00E9497AE8091A2
:10DC70006C0A882329F010927E0A0CE61AE002C092
:10DC80000FE51AE0A2E19A2EF80161918F01662357
:10DC900011F091103AC1992009F48ECF60E28EE321
:10DCA0009DE00E9497AE9A94F6CF6091330D7091EB
:10DCB000340D8091350D9091360DA70196010E948B
:10DCC00056B3241535054605570509F078CF0E944F
:10DCD0002D666FE57AE08BE59AE00E94A6391092F6
:10DCE000330D1092340D1092350D1092360D4FC138
:10DCF000811104C0FF8DF1116FC061CF6091330DB0
:10DD00007091340D8091350D9091360DA7019601DB
:10DD10000E9456B32415350546055705A1F52091F7
:10DD2000990D29A310E0412F60E08EE39DE00E9451
:10DD3000F92860E28EE39DE00E9497AE1F5F1430E9
:10DD400091F7432D60E08EE39DE00E94F9286EE399
:10DD50008EE39DE00E9497AE2DE63AE0FCE68F2E22
:10DD6000FAE09F2E01E010E0F40151914F015111B2
:10DD7000D2C014E1101B60E28EE39DE00E9497AEDA
:10DD80001150C9F7B7CF432D60E08EE39DE00E94AC
:10DD9000F92860E28EE39DE00E9497AE80916C0AC4
:10DDA000882329F010927F0A0CE61AE002C00FE5E2
:10DDB0001AE0E3E19E2EF80161918F01662311F0D4
:10DDC0009110DFC0992009F495CF60E28EE39DE0C9
:10DDD0000E9497AE9A94F6CF6091330D7091340DF6
:10DDE0008091350D9091360DA70196010E9456B392
:10DDF000241535054605570509F0E1CE0E942D662C
:10DE00008FE59AE09F938F9387E290E19F938F93A2
:10DE10008E010F5F1F4F1F930F930E9433B70F9018
:10DE20000F900F900F900F900F907E01F5E0EF0E86
:10DE3000F11CF7018081882349F0992787FD90958F
:10DE40000E9470B6F70181937F01F3CFC8010E9451
:10DE5000E83E83E290E10E945B3F98DC98C01F5F40
:10DE6000AFCE6091330D7091340D8091350D90914E
:10DE7000360DA70196010E9456B3812F90E0A0E0D5
:10DE8000B0E0281739074A075B0788F0E5E01E9FD6
:10DE9000C00111240197AA2797FDA095BA2F80935E
:10DEA000330D9093340DA093350DB093360D6091E2
:10DEB000330D7091340D8091350D9091360DA70181
:10DEC00096010E9456B380913C0D90E00396422F3C
:10DED00050E08417950764F48DEF820F80933C0D1A
:10DEE00081E080936F027CEF272E220E33243A9438
:10DEF00033942394F3E0F31508F0CBCD48C08EE3C0
:10DF00009DE00E9497AE9A9491CE8EE39DE00E9490
:10DF100097AE9A94B9CE432D602F8EE39DE02DA34A
:10DF20003EA35CA30E94F9285CA1652F8EE39DE0CF
:10DF30000E9497AE0F5F1F4F2DA13EA10431110526
:10DF400009F012CF49010CE211E080913D0D82FDF4
:10DF500005C08091990D99A1981741F001501109C0
:10DF60000115110591F72F5F3F4FFCCE61E070E086
:10DF700080E090E02DA33EA30E9438AA2DA13EA1EF
:10DF8000EDCF8EE39DE00E9497AE9A9414CFA696B3
:10DF90000FB6F894DEBF0FBECDBFDF91CF911F91BA
:10DFA0000F91FF90EF90DF90CF90BF90AF909F9038
:10DFB0008F907F906F905F904F903F902F9008953B
:10DFC0008F929F92AF92BF92CF92DF92EF92FF9289
:10DFD0000F931F93CF93DF938091330D9091340D66
:10DFE000A091350DB091360D81309048A105B10555
:10DFF00040F01092330D1092340D1092350D1092A6
:10E00000360D6091330D7091340D8091350D9091E6
:10E01000360D25E030E040E050E00E9456B380919C
:10E020003C0D90E0A0E0B0E0281739074A075B07F5
:10E0300010F420933C0DD0913C0D10913D0D12FB3E
:10E04000112710F9C0E095E0C92ED12CE12CF12C5C
:10E0500027E2822E912CA12CB12C01E06091330D8E
:10E060007091340D8091350D9091360DD11134C0E1
:10E0700020916F02222371F023E065307105810544
:10E08000910510F443E001C040E264E070E18C2FA0
:10E090000E940665112309F4C8C18091330D909147
:10E0A000340DA091350DB091360D0597A105B10540
:10E0B00008F0BBC10E942D6683E493E7DF91CF9106
:10E0C0001F910F91FF90EF90DF90CF90BF90AF9096
:10E0D0009F908F900C946566D130D9F520916F0296
:10E0E000222399F0A70196010E9456B321303105F1
:10E0F0004105510519F420E24EE302C020E240E25E
:10E1000064EF7FE08C2F0E940665112309F48DC116
:10E110006091330D7091340D8091350D9091360DD5
:10E12000A70196010E9456B32130310541055105E2
:10E1300009F07BC10E942D66DF91CF911F910F9155
:10E14000FF90EF90DF90CF90BF90AF909F908F9017
:10E15000C5CBD230D9F520916F02222399F0A701C7
:10E1600096010E9456B3223031054105510519F43C
:10E1700020E24EE302C020E240E265EE7FE08C2F19
:10E180000E940665112309F450C16091330D70910E
:10E19000340D8091350D9091360DA70196010E94A6
:10E1A00056B3223031054105510509F03EC10E94A8
:10E1B0002D66DF91CF911F910F91FF90EF90DF902F
:10E1C000CF90BF90AF909F908F9071CBD330D9F507
:10E1D00020916F02222399F0A70196010E9456B365
:10E1E000233031054105510519F420E24EE302C008
:10E1F00020E240E266ED7FE08C2F0E94066511234D
:10E2000009F413C16091330D7091340D8091350D77
:10E210009091360DA70196010E9456B32330310527
:10E220004105510509F001C10E942D66DF91CF9192
:10E230001F910F91FF90EF90DF90CF90BF90AF9024
:10E240009F908F9079CBD430D9F520916F02222303
:10E2500099F0A70196010E9456B32430310541057B
:10E26000510519F420E24EE302C020E240E266ECE0
:10E270007FE08C2F0E940665112309F4D6C06091BF
:10E28000330D7091340D8091350D9091360DA701AD
:10E2900096010E9456B3243031054105510509F01D
:10E2A000C4C00E942D66DF91CF911F910F91FF9006
:10E2B000EF90DF90CF90BF90AF909F908F9053CB17
:10E2C000D530D9F520916F02222399F0A70196014C
:10E2D0000E9456B3253031054105510519F420E25D
:10E2E0004EE302C020E240E266EB7FE08C2F0E940A
:10E2F0000665112309F499C06091330D7091340DB6
:10E300008091350D9091360DA70196010E9456B36C
:10E31000253031054105510509F087C00E942D6661
:10E32000DF91CF911F910F91FF90EF90DF90CF90F1
:10E33000BF90AF909F908F90E8CAD630D9F52091CA
:10E340006F02222399F0A70196010E9456B326304E
:10E3500031054105510519F420E24EE302C020E2E7
:10E3600040E267EA7FE08C2F0E940665112309F4E2
:10E370005CC06091330D7091340D8091350D90919A
:10E38000360DA70196010E9456B32630310541058E
:10E39000510509F04AC00E942D66DF91CF911F916F
:10E3A0000F91FF90EF90DF90CF90BF90AF909F9034
:10E3B0008F90F0CAD730C9F520916F02222399F0CF
:10E3C000A70196010E9456B327303105410551053A
:10E3D00019F420E24EE302C020E240E26EE97FE061
:10E3E0008C2F0E940665112301F16091330D70910D
:10E3F000340D8091350D9091360DA70196010E9444
:10E4000056B3273031054105510579F40E942D6638
:10E41000DF91CF911F910F91FF90EF90DF90CF9000
:10E42000BF90AF909F908F90B9C98091330D90911C
:10E43000340DA091350DB091360D8897A105B10529
:10E4400040F08092330D9092340DA092350DB09231
:10E45000360D6091330D7091340D8091350D909192
:10E46000360DA70196010E9456B380913C0D90E0B5
:10E470000396422F50E0841795074CF48DEF820FDE
:10E4800080933C0D00936F02DCEFD20FCFEFCF5F94
:10E49000DF5FC43008F4E2CDDF91CF911F910F917F
:10E4A000FF90EF90DF90CF90BF90AF909F908F90B4
:10E4B000089581D941E060E08EE39DE00E94F92853
:10E4C00068EF74E08EE39DE00E9496AE42E060E06B
:10E4D0008EE39DE00E94F92868E075E08EE39DE000
:10E4E0000C9496AE68D942E060E08EE39DE00E9415
:10E4F000F9286DE175E08EE39DE00C9496AE1F93D4
:10E50000CF93DF9358D940E060E08EE39DE00E9416
:10E51000F9286CE275E08EE39DE00E9496AE42E041
:10E5200060E08EE39DE00E94F9286AE375E08EE3E7
:10E530009DE00E9496AE10E043E0612F8EE39DE0E7
:10E540000E94F9286FE573E08EE39DE00E9496AE8D
:10E55000CAE0D0E00E94ED1E81E00E94604A65E5BD
:10E5600070E080E090E00E9438AA2197209791F710
:10E570001F5F143109F7DF91CF911F9108951F9309
:10E58000CF93DF9318D940E060E08EE39DE00E94D6
:10E59000F92869E475E08EE39DE00E9496AE42E0C2
:10E5A00060E08EE39DE00E94F9286AE375E08EE367
:10E5B0009DE00E9496AE10E043E0612F8EE39DE067
:10E5C0000E94F9286FE573E08EE39DE00E9496AE0D
:10E5D000CAE0D0E00E94ED1E81E00E94604A6EE633
:10E5E00070E080E090E00E9438AA2197209791F790
:10E5F0001F5F143109F7DF91CF911F910895809328
:10E600002C0D10922B0D0895E2E7F2E0019000200E
:10E61000E9F73197E257F2401E161F0634F01092C8
:10E62000860282E080936F02089580E2E431F10572
:10E63000B4F7DF01AE58BD4F8C933196F7CF2091E0
:10E640008A0D211108C044E150E0BC0182E792E04C
:10E650000E9424B7D9CF089510925D0A60E08BE53F
:10E660009AE00E94A5350E948B9487E190E10E9478
:10E670005B3F81E080931D0A8CE595E0E0DF83E15C
:10E6800090E10C945B3FAF92BF92CF92DF92EF92FA
:10E69000FF920F931F93CF93DF931092970D80916A
:10E6A000330D9091340DA091350DB091360D813020
:10E6B0009048A105B10540F01092330D1092340D31
:10E6C0001092350D1092360D6091330D7091340D0E
:10E6D0008091350D9091360D25E030E040E050E01E
:10E6E0000E9456B380913C0D90E0A0E0B0E0281766
:10E6F00039074A075B0710F420933C0DD0913C0D7D
:10E7000010913D0D12FB112710F9C0E045E0C42E19
:10E71000D12CE12CF12CAA24A394D11137C08091E3
:10E720006F028823A9F08091330D9091340DA09150
:10E73000350DB091360D23E00597A105B10510F414
:10E7400043E001C040E26BEF71E18C2F0E9406654F
:10E750001123E1F08091330D9091340DA091350D8E
:10E76000B091360D0597A105B10580F40E942D6684
:10E7700086EF90E8DF91CF911F910F91FF90EF907E
:10E78000DF90CF90BF90AF900C9465660E94D8A5A3
:10E790004091330D5091340D6091350D7091360DCF
:10E7A000811104C080915D0A882399F1D130C9F5A7
:10E7B00080916F028823A9F0CB01BA01A7019601CD
:10E7C0000E9456B3213031054105510519F42EE759
:10E7D0004EE302C02EE740E265EF71E18C2F0E940C
:10E7E00006651123F1F06091330D7091340D809125
:10E7F000350D9091360DA70196010E9456B3213038
:10E8000031054105510569F40E942D6684E39CE7BA
:10E810003EC2D13031F480916F0281119BC211113F
:10E82000AFC220915E0A6091330D7091340D8091DA
:10E83000350D9091360D222309F4F1C02091460C3C
:10E84000222309F4B9C020915D0A2223E9F1D230D4
:10E8500009F076C020916F02222399F0A70196015A
:10E860000E9456B3223031054105510519F420E2CA
:10E870004EE302C020E240E26BED71E18C2F0E947A
:10E880000665112309F4E2C06091330D7091340DD7
:10E890008091350D9091360DA70196010E9456B3D7
:10E8A000223031054105510509F0D0C00E942D6686
:10E8B000DF91CF911F910F91FF90EF90DF90CF905C
:10E8C000BF90AF900C948C65D230D1F520916F023F
:10E8D000222399F0A70196010E9456B322303105F8
:10E8E0004105510519F420E24EE302C020E240E266
:10E8F00060ED71E18C2F0E940665112309F4A6C01A
:10E900006091330D7091340D8091350D9091360DDD
:10E91000A70196010E9456B32230310541055105E9
:10E9200009F094C00E942D66DF91CF911F910F9145
:10E93000FF90EF90DF90CF90BF90AF900C948865E0
:10E94000D33009F083C020916F02222399F0A701F0
:10E9500096010E9456B3233031054105510519F443
:10E9600020E24EE302C020E240E262EC71E18C2F33
:10E970000E940665112309F469C06091330D7091FE
:10E98000340D8091350D9091360DA70196010E94AE
:10E9900056B3233031054105510509F057C00E9497
:10E9A0002D66DF91CF911F910F91FF90EF90DF9037
:10E9B000CF90BF90AF9050CED23011F003E047C05F
:10E9C00020916F02222399F0A70196010E9456B36D
:10E9D000223031054105510519F42EE74EE302C0FE
:10E9E0002EE740E268EB71E18C2F0E94066511234F
:10E9F00029F36091330D7091340D8091350D909114
:10EA0000360DA70196010E9456B32230310541050B
:10EA10005105A1F60E942D6681EE9CE638C1D230E8
:10EA200069F620916F02222311F3A70196010E943B
:10EA300056B3223031054105510519F42EE74EE356
:10EA400002C02EE740E269EA71E1CECF04E0809196
:10EA50005D0A8111DCC00D1348C080916F028823CC
:10EA6000F9F06091330D7091340D8091350D9091D6
:10EA7000360DA70196010E9456B3802F90E0A0E0CA
:10EA8000B0E0281739074A075B0719F420E24EE384
:10EA900002C020E240E269E971E18C2F0E94066524
:10EAA000112319F16091330D7091340D8091350D62
:10EAB0009091360DA70196010E9456B3802F90E0E9
:10EAC000A0E0B0E0281739074A075B0771F40E94FD
:10EAD0002D66DF91CF911F910F91FF90EF90DF9006
:10EAE000CF90BF90AF900C94196CBB24B394B00E30
:10EAF000BD1248C080916F028823F9F06091330DF8
:10EB00007091340D8091350D9091360DA7019601CD
:10EB10000E9456B38D2F90E0A0E0B0E0281739078F
:10EB20004A075B0719F420E24EE302C020E240E20C
:10EB300068E871E18C2F0E940665112319F160913C
:10EB4000330D7091340D8091350D9091360DA701E4
:10EB500096010E9456B38B2D90E0A0E0B0E02817FC
:10EB600039074A075B0771F40E942D66DF91CF9148
:10EB70001F910F91FF90EF90DF90CF90BF90AF90DB
:10EB80000C94DF6B32E0B32EB00EBD123FC080910B
:10EB90006F028823F9F06091330D7091340D8091EC
:10EBA000350D9091360DA70196010E9456B38D2F19
:10EBB00090E0A0E0B0E0281739074A075B0719F496
:10EBC0002EE74EE302C02EE740E26EE771E18C2FA4
:10EBD0000E9406651123D1F06091330D7091340DC0
:10EBE0008091350D9091360DA70196010E9456B384
:10EBF0008B2D90E0A0E0B0E0281739074A075B07AB
:10EC000029F40E942D668FE198E641C00D5F0D1337
:10EC10004AC080916F028823F9F06091330D7091A2
:10EC2000340D8091350D9091360DA70196010E940B
:10EC300056B3802F90E0A0E0B0E0281739074A07CC
:10EC40005B0719F42EE74EE302C02EE740E266E7C9
:10EC500071E18C2F0E940665112329F16091330D1B
:10EC60007091340D8091350D9091360DA70196016C
:10EC70000E9456B3802F90E0A0E0B0E0281739073B
:10EC80004A075B0781F40E942D668FE696E6DF91C6
:10EC9000CF911F910F91FF90EF90DF90CF90BF9099
:10ECA000AF900C946A66BB24B394B00E6091330DA0
:10ECB0007091340D8091350D9091360DA70196011C
:10ECC0000E9456B38B2D90E0A0E0B0E028173907E2
:10ECD0004A075B0788F025E0B29EC0011124019726
:10ECE000AA2797FDA095BA2F8093330D9093340DEA
:10ECF000A093350DB093360D6091330D7091340DA6
:10ED00008091350D9091360DA70196010E9456B362
:10ED100080913C0D90E00396422F50E084179507B8
:10ED20004CF48DEF820F80933C0DA0926F02DCEFCC
:10ED3000D20FCFEFCF5FDF5FC43008F4EECCDF91AE
:10ED4000CF911F910F91FF90EF90DF90CF90BF90E8
:10ED5000AF900895CB01BA01A70196010E9456B366
:10ED6000213031054105510519F42EE74EE302C06B
:10ED70002EE740E26BEE71E18C2F0E9406654FCDCD
:10ED80006091330D7091340D8091350D9091360D59
:10ED9000A70196010E9456B3213031054105510566
:10EDA00009F03FCD0E942D6680EE9FE670CF209146
:10EDB0008A0D211108C044E150E0BC0182E792E0D5
:10EDC0000E9497B621CC0895F2DF81E080938A0DEE
:10EDD0000C94C66B10928A0D0895CF92DF92EF9239
:10EDE000FF92CF93CCB1C095CC1FCC27CC1F809184
:10EDF000030183FFC260C090380DD090390DE090C0
:10EE00003A0DF0903B0D0E9409AAC616D706E806F7
:10EE1000F90610F4489B39C0C0933D0D80913D0D1B
:10EE2000817090913D0D91FD82609091370D891711
:10EE300021F18130F1F028F0823089F08330A1F0A7
:10EE40001CC0913021F49091990D9F5F05C09230C4
:10EE5000A1F49091990D91509093990D0EC0992322
:10EE600091F3933051F4F5CF923069F3913029F456
:10EE7000F0CF933041F3992361F38093370DCF9115
:10EE8000FF90EF90DF90CF900895C460C5CF0E94AF
:10EE9000BA6B6F98E4E0F1E08081877F8083779A96
:10EEA0009FB7F894E5E0F1E08081886080839FBFA0
:10EEB0005098589A60E088E40E9429A99FB7F89476
:10EEC000E5E0F1E08081846080839FBF8091030151
:10EED00082FB882780F991E089278093320D7DDFBE
:10EEE0001092990D0895CF92DF92EF92FF9275DF05
:10EEF0008091030191E082FB882780F98927209186
:10EF0000320D8217C9F082E080936F028091030175
:10EF100082FB882780F989278093320D0E94BA6B83
:10EF20008091320D882309F490C08BE59AE00E940D
:10EF3000E23087ED9EE03BDFC0902E0DD0902F0D8C
:10EF4000E090300DF090310D0E9409AAC616D70648
:10EF5000E806F90608F086C04091990D442361F156
:10EF600081E080936F02552747FD5095652F752FDF
:10EF70008091330D9091340DA091350DB091360DE7
:10EF8000840F951FA61FB71F8093330D9093340DE8
:10EF9000A093350DB093360D1092990D0E9409AAD9
:10EFA0006856754C8F4F9F4F6093030D7093040DFF
:10EFB0008093050D9093060D80913D0D82FF0EC04C
:10EFC0000E9409AA6856754C8F4F9F4F6093030D9E
:10EFD0007093040D8093050D9093060DE0917002DF
:10EFE000F09171021995C090030DD090040DE0903E
:10EFF000050DF090060D0E9409AAC616D706E80670
:10F00000F90638F48091700290917102865F904801
:10F0100019F580916F02823011F40E94DB6B8091B0
:10F020006F02882319F0815080936F020E9409AA11
:10F030006C597F4F8F4F9F4F60932E0D70932F0D04
:10F040008093300D9093310D0DC08BE59AE00E94B6
:10F05000AD3189EC9EE06FCF0E94C66B82E0809359
:10F060006F02D7CFFF90EF90DF90CF90089581E0AF
:10F07000089580913D0D82FB882780F908950F93B4
:10F080001F93CF93DF930E94DB6B40E060E08EE341
:10F090009DE00E94F9286AE675E08EE39DE00E94FB
:10F0A00096AE41E061E08EE39DE00E94F92865E7BD
:10F0B00075E08EE39DE00E9496AE42E061E08EE353
:10F0C0009DE00E94F92869E775E08EE39DE00E94CB
:10F0D00096AE43E061E08EE39DE00E94F9286CE883
:10F0E00075E08EE39DE00E9496AE41E060E08EE325
:10F0F0009DE00E94F9286DE975E08EE39DE00E9495
:10F1000096AE0091990D112707FD1095C1E0D0E052
:10F110008091530A9091540A892B09F071C00E9482
:10F12000ED1E81E00E94604A2091990D332727FD52
:10F130003095C801821B930B97FF03C09195819571
:10F14000910905970CF44DC0201731070CF4219755
:10F15000021713070CF42196C430D1052CF4209724
:10F1600029F4C1E0D0E002C0C3E0D0E041E060E0BB
:10F170008EE39DE00E94F92861E973E08EE39DE053
:10F180000E9496AE42E060E08EE39DE00E94F92886
:10F1900061E973E08EE39DE00E9496AE43E060E09B
:10F1A0008EE39DE00E94F92861E973E08EE39DE023
:10F1B0000E9496AE4C2F60E08EE39DE00E94F928FD
:10F1C0006DE975E08EE39DE00E9496AE0091990D89
:10F1D000112707FD109564E670E080E090E00E9442
:10F1E00038AA47DF882309F493CFD093540AC093F9
:10F1F000530A64EF71E080E090E00E9438AA88CF63
:10F200000E94DB6BDF91CF911F910F910C94C66B25
:10F21000FC01808190E02AE030E0B9010E9443B314
:10F22000482FCB01B9010E9443B3805D8093070D45
:10F23000405D4093080D1092090D87E09DE0089510
:10F2400020E030E040E251E4FC0160817181828184
:10F2500093810E944DB20E94E7AF77FD02C02BE27E
:10F2600001C02DE22093070D9B0177FF04C02227E8
:10F270003327261B370BC90168EE73E00E9443B3A6
:10F28000CB01EAE0F0E0BF010E9443B3805D8093D0
:10F29000080DC90164E670E00E9443B3CB01BF01D1
:10F2A0000E9443B3805D8093090DC901BF010E9494
:10F2B00043B3282FCB01BF010E9443B3805D8093ED
:10F2C0000A0D8EE280930B0D205D20930C0D1092A1
:10F2D0000D0D87E09DE008958F929F92AF92BF92AF
:10F2E000CF92DF92EF92FF92FC0180809180A2800A
:10F2F000B38020E030E048EC52E4C501B4010E9444
:10F300004DB26B017C0120E030E0A9010E947BB18D
:10F3100018161CF4C701B60103C0C701B601905806
:10F320000E94E7AF6B017C0120E030E0A901C5013C
:10F33000B4010E9478AF87FF12C08DE28093070D61
:10F34000C701B60128EE33E040E050E00E9478B3F8
:10F35000CA01B9012AE030E040E050E036C0C70100
:10F36000B60120E137E240E050E00E9478B3AAE025
:10F370008A2E912CA12CB12CCA01B901A5019401AE
:10F380000E9478B3662391F0605D6093070DC7011A
:10F39000B60128EE33E040E050E00E9478B3CA01A5
:10F3A000B901A50194010E9478B313C080E2809353
:10F3B000070DC701B60128EE33E040E050E00E949F
:10F3C00078B3CA01B901A50194010E9478B36623FC
:10F3D00011F0605D01C060E26093080DC701B601E5
:10F3E00024E630E040E050E00E9478B3FAE08F2E4F
:10F3F000912CA12CB12CCA01B901A50194010E9444
:10F4000078B3605D6093090DC701B601A501940151
:10F410000E9478B3662381F0605D60930C0DCA0191
:10F42000B901A50194010E9478B3605D60930B0D52
:10F430008EE280930A0D15C0CA01B901A50194019D
:10F440000E9478B3662329F0605D60930B0D8EE215
:10F4500003C080E280930B0D80930A0D80E28093BD
:10F460000C0D10920D0D87E09DE0FF90EF90DF9066
:10F47000CF90BF90AF909F908F900895FC01208116
:10F48000318137FF07C08DE28093070D31952195BB
:10F49000310914C02436310574F0C90164E670E006
:10F4A0000E9443B3CB016AE070E00E9443B3805DE9
:10F4B0008093070D06C080E28093070D2A30310546
:10F4C00064F0EAE0F0E0C901BF010E9443B3CB0160
:10F4D000BF010E9443B3805D01C080E28093080DAC
:10F4E000C9016AE070E00E9443B3805D8093090D1A
:10F4F00010920A0D87E09DE008958F929F92AF923F
:10F50000BF92CF92DF92EF92FF920F931F93CF9310
:10F51000DF93609114027091150280911602909110
:10F5200017020E9438286093170D7093180D80936E
:10F53000190D90931A0D6091100270911102809133
:10F540001202909113020E9444286093130D70934D
:10F55000140D8093150D9093160D8091330D90919D
:10F56000340DA091350DB091360D81309048A10534
:10F57000B10540F01092330D1092340D1092350DFC
:10F580001092360D6091330D7091340D8091350DD0
:10F590009091360D25E030E040E050E00E9456B3F7
:10F5A00080913C0D90E0A0E0B0E0281739074A07B1
:10F5B0005B0710F420933C0DD0913C0D10913D0D54
:10F5C00012FB112710F9C0E0B5E0CB2ED12CE12CB5
:10F5D000F12C03E1802E912CA12CB12C01E0609143
:10F5E000330D7091340D8091350D9091360DD11100
:10F5F00034C020916F02222371F023E06530710541
:10F600008105910510F443E001C040E265E770E137
:10F610008C2F0E940665112309F4E2C08091330DFE
:10F620009091340DA091350DB091360D0597A1053F
:10F63000B10508F0D5C00E942D668FE198E6DF91F4
:10F64000CF911F910F91FF90EF90DF90CF90BF90DF
:10F65000AF909F908F900C946566D130D9F5209132
:10F660006F022223B9F0A70196010E9456B386E4E7
:10F6700098E0213031054105510521F4FFDE9C0160
:10F680004EE303C0FBDE9C0140E26EE670E18C2F8E
:10F690000E943D65112309F4A3C06091330D709160
:10F6A000340D8091350D9091360DA70196010E9481
:10F6B00056B3213031054105510509F091C00E9432
:10F6C0002D6623E331E040E050E066E478E087E631
:10F6D00090E178C0D230D9F520916F022223B9F0A1
:10F6E000A70196010E9456B384E498E022303105C8
:10F6F0004105510521F4C2DE9C014EE303C0BEDE8C
:10F700009C0140E263E670E18C2F0E943D6511236D
:10F7100009F466C06091330D7091340D8091350D00
:10F720009091360DA70196010E9456B32230310503
:10F730004105510509F054C00E942D6623E930E0CF
:10F7400040E050E064E478E08FE590E13BC0D330E6
:10F7500009F046C020916F022223B9F0A70196015B
:10F760000E9456B38CE29AE02330310541055105E1
:10F7700021F484DE9C014EE303C080DE9C0140E264
:10F7800060E570E18C2F0E943D65112349F1609185
:10F79000330D7091340D8091350D9091360DA70188
:10F7A00096010E9456B32330310541055105C1F43D
:10F7B0000E942D662FEF30E040E050E06CE27AE0EE
:10F7C00081E490E1DF91CF911F910F91FF90EF9035
:10F7D000DF90CF90BF90AF909F908F900C94B464C7
:10F7E0008091330D9091340DA091350DB091360D6F
:10F7F0004497A105B10540F08092330D9092340DED
:10F80000A092350DB092360D6091330D7091340D8C
:10F810008091350D9091360DA70196010E9456B347
:10F8200080913C0D90E00396422F50E0841795079D
:10F830004CF48DEF820F80933C0D00936F02DCEF50
:10F84000D20FCFEFCF5FDF5FC43008F4C8CEDF91B7
:10F85000CF911F910F91FF90EF90DF90CF90BF90CD
:10F86000AF909F908F9008958F929F92AF92BF928A
:10F87000CF92DF92EF92FF920F931F93CF93DF937C
:10F880008091330D9091340DA091350DB091360DCE
:10F8900081309048A105B10540F01092330D1092CF
:10F8A000340D1092350D1092360D6091330D70911C
:10F8B000340D8091350D9091360D25E030E040E01B
:10F8C00050E00E9456B380913C0D90E0A0E0B0E083
:10F8D000281739074A075B0710F420933C0DD09195
:10F8E0003C0D10913D0D12FB112710F9C0E085E091
:10F8F000C82ED12CE12CF12C92E2892E912CA12C36
:10F90000B12C01E06091330D7091340D8091350D73
:10F910009091360DD11134C020916F02222371F0E5
:10F9200023E0653071058105910510F443E001C0C5
:10F9300040E26FE87FE08C2F0E940665112309F4F6
:10F940009CC18091330D9091340DA091350DB091F3
:10F95000360D0597A105B10508F08FC10E942D66EF
:10F9600083E493E7DF91CF911F910F91FF90EF9088
:10F97000DF90CF90BF90AF909F908F900C94656672
:10F98000D130D9F520916F022223B9F0A701960159
:10F990000E9456B38DE592E02130310541055105B5
:10F9A00021F46CDD9C014EE303C068DD9C0140E264
:10F9B00066E87FE08C2F0E943D65112309F45DC14C
:10F9C0006091330D7091340D8091350D9091360D0D
:10F9D000A70196010E9456B321303105410551051A
:10F9E00009F04BC10E942D6627EE33E04AE050E05B
:10F9F0006DE572E08DE79FE03DC0D23009F048C070
:10FA000020916F022223B9F0A70196010E9456B3FC
:10FA100086E498E0223031054105510521F42EDDC0
:10FA20009C014EE303C02ADD9C0140E266E77FE0D3
:10FA30008C2F0E943D65112309F41FC16091330D85
:10FA40007091340D8091350D9091360DA70196017E
:10FA50000E9456B3223031054105510509F00DC110
:10FA60000E942D6623E331E040E050E066E478E058
:10FA70008FE69FE0DF91CF911F910F91FF90EF9064
:10FA8000DF90CF90BF90AF909F908F900C94B46414
:10FA9000D330D9F520916F022223B9F0A701960146
:10FAA0000E9456B384E498E02330310541055105A6
:10FAB00021F4E4DC9C014EE303C0E0DC9C0140E265
:10FAC0006BE67FE08C2F0E943D65112309F4D5C0C1
:10FAD0006091330D7091340D8091350D9091360DFC
:10FAE000A70196010E9456B3233031054105510507
:10FAF00009F0C3C00E942D6623E930E040E050E0E9
:10FB000064E478E087E69FE0B5CFD430D9F5209162
:10FB10006F022223B9F0A70196010E9456B38CE22E
:10FB20009AE0243031054105510521F4A7DC9C0100
:10FB30004EE303C0A3DC9C0140E268E57FE08C2F2C
:10FB40000E943D65112309F498C06091330D7091B6
:10FB5000340D8091350D9091360DA70196010E94CC
:10FB600056B3243031054105510509F086C00E9485
:10FB70002D662FEF30E040E050E06CE27AE089E45F
:10FB80009FE078CFD530D9F520916F022223B9F0CC
:10FB9000A70196010E9456B38BE592E0253031050E
:10FBA0004105510521F46ADC9C014EE303C066DC8B
:10FBB0009C0140E262E47FE08C2F0E943D651123AE
:10FBC00009F45BC06091330D7091340D8091350D57
:10FBD0009091360DA70196010E9456B3253031054C
:10FBE0004105510509F049C00E942D6627EE33E01A
:10FBF0004AE050E06BE572E08BE39FE03BCFD6300C
:10FC0000E1F520916F02222399F0A70196010E944D
:10FC100056B3263031054105510519F420E24EE373
:10FC200002C020E240E26AE27FE08C2F0E9406657B
:10FC3000112319F16091330D7091340D8091350DC0
:10FC40009091360DA70196010E9456B326303105DA
:10FC50004105510591F40E942D6685E29FE0DF91F8
:10FC6000CF911F910F91FF90EF90DF90CF90BF90B9
:10FC7000AF909F908F900C945B3F8091330D90914B
:10FC8000340DA091350DB091360D8397A105B105C6
:10FC900040F08092330D9092340DA092350DB092C9
:10FCA000360D6091330D7091340D8091350D90912A
:10FCB000360DA70196010E9456B380913C0D90E04D
:10FCC0000396422F50E0841795074CF48DEF820F76
:10FCD00080933C0D00936F02DCEFD20FCFEFCF5F2C
:10FCE000DF5FC43008F40ECEDF91CF911F910F91EA
:10FCF000FF90EF90DF90CF90BF90AF909F908F904C
:10FD00000895FC01808191818436910524F164E697
:10FD100070E00E9443B3CB012AE030E0B9010E94B9
:10FD200043B3805D8093070D80819181B9010E946A
:10FD300043B3CB01B9010E9443B3805D8093080DAA
:10FD400080819181B9010E9443B3805D8093090D48
:10FD500010920A0D23C08A309105BCF02AE030E0F1
:10FD6000B9010E9443B3CB01B9010E9443B3805D46
:10FD70008093070D80819181B9010E9443B3805D1A
:10FD80008093080D1092090D09C06AE070E00E948E
:10FD900043B3805D8093070D1092080D87E09DE0CE
:10FDA0000895CF92EF920F93EFE1CE2EF0E2EF2E77
:10FDB0000FE02EE045E066E28EE39DE00E94E4293C
:10FDC0000F91EF90CF900895CF93DF93FC01649152
:10FDD000EC012196662331F08EE39DE00E94D12A4A
:10FDE000CE01F4CFDF91CF9108950F931F93CF935E
:10FDF000DF938C01EB0141E061E08EE39DE00E9426
:10FE0000F928C801E1DF6AE38EE39DE00E9497AE26
:10FE1000FE0101900020E9F76C2F6E1B6C5E41E043
:10FE20008EE39DE00E94F928BE018EE39DE0DF9104
:10FE3000CF911F910F910C9496AECF92DF92EF92DB
:10FE4000FF920F931F938091330D9091340DA091E9
:10FE5000350DB091360D0097A105B10509F442C0EA
:10FE6000BC01882777FD8095982F0E941AB02091B9
:10FE70000F0D3091100D4091110D5091120D0E94F7
:10FE80004DB29B01AC0160914E0A70914F0A809176
:10FE9000500A9091510A0E949FAE60934E0A70934F
:10FEA0004F0A8093500A9093510A1092330D10928A
:10FEB000340D1092350D1092360DAEE2CA2EAAE026
:10FEC000DA2EE12CF12C00E81FE32EE43AE04AE4BC
:10FED0005AE066E47AE082E49AE00E944F9B81E077
:10FEE00080936F0280916F02882339F08EE49AE04C
:10FEF000A7D9BC0185E890E178DF80913D0D82FFB4
:10FF00000EC021E040E050E0BA0188EF99E61F9171
:10FF10000F91FF90EF90DF90CF900C944F661F9160
:10FF20000F91FF90EF90DF90CF900895CF93DF93E4
:10FF30001F921F92CDB7DEB78091330D9091340D93
:10FF4000A091350DB091360DB7FF08C01092330D5A
:10FF50001092340D1092350D1092360D80911B0DBC
:10FF600090911C0DA0911D0DB0911E0D4091330D6F
:10FF70005091340D6091350D7091360D84179507B1
:10FF8000A607B70744F48093330D9093340DA093E4
:10FF9000350DB093360D80916F028823A9F08091C2
:10FFA0001F0D9091200D2091330D3091340D820F53
:10FFB000931F9A838983CE01019660DABC018091F8
:10FFC000250D9091260D11DF80913D0D82FF1DC002
:10FFD000E091230DF091240D80911F0D9091200D43
:10FFE0002091330D3091340D820F931F91838083C4
:10FFF0004091270D5091280D60E070E021E0809144
:020000021000EC
:10000000290D90912A0D0E944F660F900F90DF915D
:10001000CF9108954F925F926F927F928F929F92AD
:10002000AF92BF92CF92DF92EF92FF920F931F9306
:10003000CF93DF934C015B017A018091330D909156
:10004000340DA091350DB091360D892B8A2B8B2B59
:1000500009F47BC00E948741E501CC0FDD1FCC0F66
:10006000DD1F8E010E5B154F6091330D7091340DC5
:10007000882777FD8095982F0E941AB020910F0D48
:100080003091100D4091110D5091120D0E944DB202
:10009000F80120813181428153810E949FAE2B0162
:1000A0003C0120E030E0A9010E9478AFF80187FD13
:1000B00005C0408251826282738204C01082118224
:1000C00012821382B701882777FD8095982F0E94AE
:1000D0001AB06B017C018E010E5B154F9B01AC01C8
:1000E000F80160817181828193810E947BB1181631
:1000F0002CF4F801C082D182E282F3821092330D97
:100100001092340D1092350D1092360DCD55DA4FF8
:1001100020E030E040E752E4688179818A819B8168
:100120000E947FAFDEE2CD2EDAE0DD2E7B018C0176
:100130002EE43AE04AE45AE066E47AE082E49AE0A7
:100140000E944F9B81E080936F0280916F02882311
:1001500059F0C501880F991F880F991F8E5B954F25
:100160006FD8BC01C40141DE80913D0D82FF18C0F3
:1001700021E040E050E0BA0188EF99E6DF91CF91AD
:100180001F910F91FF90EF90DF90CF90BF90AF90B5
:100190009F908F907F906F905F904F900C944F66E0
:1001A000DF91CF911F910F91FF90EF90DF90CF9053
:1001B000BF90AF909F908F907F906F905F904F9087
:1001C000089546ED50E060E070E08FE790E122CFC7
:1001D00046EC50E061E070E081E890E11BCF49EC33
:1001E00050E062E070E083E890E114CF8F929F923C
:1001F000AF92BF92CF92DF92EF92FF920F931F9335
:10020000CF93DF93CDB7DEB728970FB6F894DEBF54
:100210000FBECDBF80912D0D882321F0815080939A
:100220002D0D03C081E080936F0280916F028823BF
:1002300009F456C28091980D8F5F8093980D8E318E
:1002400029F40E94BA6B1092980D0EC06AE00E94C9
:1002500022B3911109C020E044E064E18EE39DE007
:100260000E94092A0E94906520E030E040E05FE3B0
:1002700060913E0870913F0880914008909141083C
:100280000E949FAE0E94E7AF78876F836091460817
:1002900070914708882777FD8095982F0E941AB0A3
:1002A00020E030E040E05FE30E949FAE0E94E7AFB5
:1002B0007E836D8340E060E08EE39DE00E94F9283C
:1002C00062E08EE39DE00E9497AECE010796D6D8FD
:1002D000BC018EE39DE00E9496AE6FE28EE39DE04E
:1002E0000E9497AECE0105960CDDBC018EE39DE029
:1002F0000E9496AE82E29FE067DD60E973E08EE3E4
:100300009DE00E9496AE40E06AE08EE39DE00E9490
:10031000F9286FE975E08EE39DE00E9496AE2CEA25
:1003200035EC47E257E360914A0A70914B0A80919D
:100330004C0A90914D0A0E949FAE69837A838B8309
:100340009C83CE0101960E946C79BC018EE39DE0F6
:100350000E9496AE60E28EE39DE00E9497AE41E07F
:1003600060E08EE39DE00E94F92820E030E040E06C
:100370005FE3609138087091390880913A08909154
:100380003B080E949FAE0E94E7AF78876F83609121
:10039000440870914508882777FD8095982F0E9422
:1003A0001AB020E030E040E05FE30E949FAE0E9480
:1003B000E7AF7E836D8360E08EE39DE00E9497AEA1
:1003C000CE0107965BD8BC018EE39DE00E9496AEFD
:1003D0006FE28EE39DE00E9497AECE01059691DC20
:1003E000BC018EE39DE00E9496AE8FE19FE0ECDCC5
:1003F00060E973E08EE39DE00E9496AE41E06AE022
:100400008EE39DE00E94F92860E973E08EE39DE0B1
:100410000E9496AE66E08EE39DE00E9497AE8DE569
:1004200092E02CD8BC018EE39DE00E9496AE65E27E
:100430008EE39DE00E9497AE6DE873E08EE39DE051
:100440000E9496AE42E060E08EE39DE00E94F928B3
:100450008CE19FE0B9DC80915D0A8823A9F180914D
:10046000460C882319F18091F00C9091F10CA09129
:10047000F20CB091F30C0097A105B105B9F0BC01E5
:10048000CD016D597F4F8F4F9F4F24E630E040E004
:1004900050E00E9456B36091F80C7091F90C809175
:1004A000FA0C9091FB0C0E9456B301C020E030E0A2
:1004B0003A832983CE0101960E943E7ABC018EE3E5
:1004C0009DE00E9496AE03C088E19FE07DDC65E27E
:1004D0008EE39DE00E9497AE6CE873E08EE39DE0B2
:1004E0000E9496AE42E06AE08EE39DE00E94F92809
:1004F00060E973E08EE39DE00E9496AE67E08EE3D4
:100500009DE00E9497AE8091500890915108A09173
:100510005208B0915308892B8A2B8B2BE1F10E9452
:1005200009AA20E6C22E2AEED22EE12CF12CA70138
:1005300096010E9456B349015A016091500870918A
:1005400051088091520890915308A70196010E948A
:1005500056B3C401821B930B6CE370E00E942FB36F
:10056000182F6983CE0101960E940879BC018EE3A1
:100570009DE00E9496AE6AE38EE39DE00E9497AEF6
:100580001983CE0101960E940879BC018EE39DE09B
:100590000E9496AE03C082E19FE016DC60E973E042
:1005A0008EE39DE00E9496AE43E060E08EE39DE026
:1005B0000E94F9286EE773E082E792E00E9406B796
:1005C000892B09F074C06CE67AE083E59DE00E9417
:1005D00006B7892BD1F0E3E5FDE0DF010D900020A7
:1005E000E9F7AD014150510943555D4060E070E0CD
:1005F000CF010E94D6B66CE67AE083E59DE00E94CA
:100600000FB71092890D1092880DECE6FAE0019078
:100610000020E9F7ED56FA40759708F445C00091BF
:10062000880D1091890DC12CD12C8091880D90914D
:10063000890D9801281B390B2431310534F00196BE
:100640009093890D8093880D38C0C114D104B9F7F7
:10065000F801E55AF54F7F019189602F681B43E04F
:10066000911115C08EE39DE00E94F928D7015096A4
:100670006C918EE39DE00E9497AE1092890D1092CE
:10068000880D00E010E0CC24C394D12CCECF8EE3B3
:100690009DE00E94F928F70160898EE39DE00E94A9
:1006A00097AE0F5F1F4FC1CF63E57DE002C062E7E9
:1006B00072E08EE39DE00E9496AE02E712E0D80160
:1006C0008D918D0180322CF460E28EE39DE00E94DA
:1006D00097AEB2E006381B0791F78AE080932D0DA4
:1006E00080913D0D82FB882780F990912C0D9923F4
:1006F00099F090912B0D992339F0811119C0109226
:100700002B0D10922C0D14C0882391F00E942D66A1
:1007100081E080932B0D0CC0882351F021E040E054
:1007200050E0BA0183E493E70E944F660E94BA6BDF
:1007300080915D0290915E022091330D3091340DD5
:100740008436910534F4820F931F853691054CF45D
:1007500016C08436910599F0820F931F8436910557
:1007600074F41092330D1092340D1092350D1092D6
:10077000360D84E690E090935E0280935D022091B6
:100780005D0230915E028091330D9091340D2436DC
:10079000310569F48B3091051CF0865A9F4F09C0D2
:1007A000863FEFEF9E078CF482599F4F02C0820F65
:1007B000931F90935E0280935D021092330D10920E
:1007C000340D1092350D1092360D80915D0290918E
:1007D0005E028A3091051CF48AE090E005C0883EF4
:1007E000934034F087EE93E090935E0280935D0235
:1007F00028960FB6F894DEBF0FBECDBFDF91CF9124
:100800001F910F91FF90EF90DF90CF90BF90AF902E
:100810009F908F900895CF93DF93CCEBDEE0FE01A5
:100820008491882341F09091C00095FFFCCF809384
:10083000C6003196F5CFE9EFF4E18491882341F0C9
:100840009091C00095FFFCCF8093C6003196F5CF04
:100850008091C00085FFFCCF8AE08093C600FE0136
:100860008491ECEBFEE0882349F09091C00095FF65
:10087000FCCF8093C60031968491F5CF40919F13B1
:100880005091A0136091A1137091A21381EF94E194
:100890000E94C43E4091A3135091A4136091A513EC
:1008A0007091A6138EEE94E10E94C43E4091A7136E
:1008B0005091A8136091A9137091AA138BEE94E143
:1008C0000E94C43E4091AB135091AC136091AD13A4
:1008D0007091AE1388EE94E10E94C43E8091C000F6
:1008E00085FFFCCF8AE08093C600FE018491ECEB8B
:1008F000FEE0882349F09091C00095FFFCCF8093E3
:10090000C60031968491F5CFEEECF4E18491882312
:1009100041F09091C00095FFFCCF8093C6003196C6
:10092000F5CF8091C00085FFFCCF8AE08093C600A0
:10093000FE018491ECEBFEE0882349F09091C00029
:1009400095FFFCCF8093C60031968491F5CF4091FE
:10095000AF135091B0136091B1137091B21385EC45
:1009600094E10E94C43E4091B3135091B41360913E
:10097000B5137091B61382EC94E10E94C43E40918D
:10098000B7135091B8136091B9137091BA138FEBEC
:1009900094E10E94C43E4091BB135091BC136091FE
:1009A000BD137091BE138CEB94E10E94C43E809104
:1009B000C00085FFFCCF8AE08093C600FE018491D1
:1009C000ECEBFEE0882349F09091C00095FFFCCF4E
:1009D0008093C60031968491F5CFEEE9F4E18491DD
:1009E000882341F09091C00095FFFCCF8093C60012
:1009F0003196F5CF8091C00085FFFCCF8AE08093CF
:100A0000C600FE018491ECEBFEE0882349F0909152
:100A1000C00095FFFCCF8093C60031968491F5CF3E
:100A200040918F1350919013609191137091921394
:100A300085E994E10E94D63E40919313509194131E
:100A4000609195137091961382E994E10E94D63ECD
:100A500040919713509198136091991370919A1344
:100A60008FE894E10E94D63E40919B1350919C13D5
:100A700060919D1370919E138CE894E10E94D63E84
:100A80008091C00085FFFCCF8AE08093C600FE0104
:100A90008491ECEBFEE0882349F09091C00095FF33
:100AA000FCCF8093C60031968491F5CFE7E5F4E161
:100AB0008491882341F09091C00095FFFCCF8093F2
:100AC000C6003196F5CF8091C00085FFFCCF8AE04B
:100AD0008093C600FE018491ECEBFEE0882349F090
:100AE0009091C00095FFFCCF8093C6003196849111
:100AF000F5CF4091871350918813609189137091BD
:100B00008A138EE494E10E94C43E40918313509175
:100B1000841360918513709186138BE494E10E9495
:100B2000C43E8091C00085FFFCCF8AE08093C60060
:100B3000FE018491ECEBFEE0882349F09091C00027
:100B400095FFFCCF8093C60031968491F5CFE8E9FC
:100B5000F3E18491882341F09091C00095FFFCCF90
:100B60008093C6003196F5CF8091C00085FFFCCF01
:100B70008AE08093C600FE018491ECEBFEE08823BE
:100B800049F09091C00095FFFCCF8093C60031964C
:100B90008491F5CF40918B1350918C1360918D13FC
:100BA00070918E138FE893E10E94C43E40917313BD
:100BB0005091741360917513709176138CE893E1E2
:100BC0000E94C43E4091BF135091C0136091C11365
:100BD0007091C21389E893E10E94D63E40917F1341
:100BE00050918013609181137091821386E893E194
:100BF0000E94C43E40917B1350917C1360917D1301
:100C000070917E1383E893E10E94C43E4091771374
:100C1000509178136091791370917A1380E893E181
:100C20000E94C43E8091C00085FFFCCF8AE0809383
:100C3000C600FE018491ECEBFEE0882349F0909120
:100C4000C00095FFFCCF8093C60031968491F5CF0C
:100C5000EEE6F3E18491882341F09091C00095FF86
:100C6000FCCF8093C6003196F5CF8091C00085FF00
:100C7000FCCF8AE08093C600FE018491ECEBFEE09D
:100C8000882349F09091C00095FFFCCF8093C60067
:100C900031968491F5CF4091360A5091370A609190
:100CA000380A7091390A85E693E10E94C43E40916A
:100CB0003A0A50913B0A60913C0A70913D0A82E6E3
:100CC00093E10E94C43E40913E0A50913F0A6091D8
:100CD000400A7091410A8FE593E10E94C43E8091E1
:100CE000C00085FFFCCF8AE08093C600FE0184919E
:100CF000ECEBFEE0882349F09091C00095FFFCCF1B
:100D00008093C60031968491F5CFE1E5F3E18491BB
:100D1000882341F09091C00095FFFCCF8093C600DE
:100D20003196F5CF8091C00085FFFCCF8AE080939B
:100D3000C600FE018491ECEBFEE0882349F090911F
:100D4000C00095FFFCCF8093C60031968491F5CF0B
:100D5000409118025091190260911A0270911B0281
:100D600087E493E10E94C43E6091140270911502E1
:100D700080911602909117020E943828AB01BC01A5
:100D800084E493E10E94C43E6091100270911102CC
:100D900080911202909113020E944428AB01BC0181
:100DA00081E493E10E94C43E8091C00085FFFCCFA6
:100DB0008AE08093C600FE018491ECEBFEE088237C
:100DC00049F09091C00095FFFCCF8093C60031960A
:100DD0008491F5CFEDE0F3E18491882341F0909187
:100DE000C00095FFFCCF8093C6003196F5CF80916F
:100DF000C00085FFFCCF8AE08093C600FE0184918D
:100E0000ECEBFEE0882349F09091C00095FFFCCF09
:100E10008093C60031968491F5CF40913302509172
:100E20003402609135027091360283E093E10E94B2
:100E3000C43E20E030E040E752E460912B02709124
:100E40002C0280912D0290912E020E944DB2AB0196
:100E5000BC0180E093E10E94C43E4091260A50917B
:100E6000270A6091280A7091290A8DEF92E10E9469
:100E7000C43E8091C00085FFFCCF8AE08093C6000D
:100E8000FE018491ECEBFEE0882349F09091C000D4
:100E900095FFFCCF8093C60031968491F5CFE1EDAC
:100EA000F2E18491882341F09091C00095FFFCCF3E
:100EB0008093C6003196F5CF8091C00085FFFCCFAE
:100EC0008AE08093C600FE018491ECEBFEE088236B
:100ED00049F09091C00095FFFCCF8093C6003196F9
:100EE0008491F5CF4091220A5091230A6091240AFF
:100EF0007091250A87EC92E10E94C43E20E030E028
:100F000040E752E460912702709128028091290203
:100F100090912A020E944DB2AB01BC0184EC92E197
:100F20000E94C43E8091C00085FFFCCF8AE0809380
:100F3000C600FE018491ECEBFEE0882349F090911D
:100F4000C00095FFFCCF8093C60031968491F5CF09
:100F5000EAE6F2E18491882341F09091C00095FF88
:100F6000FCCF8093C6003196F5CF8091C00085FFFD
:100F7000FCCF8AE08093C600FE018491ECEBFEE09A
:100F8000882349F09091C00095FFFCCF8093C60064
:100F900031968491F5CF40912B0A50E060E070E0EB
:100FA00080E692E10E94D63E8091C00085FFFCCF92
:100FB0008AE08093C600FE018491ECEBFEE088237A
:100FC00049F09091C00095FFFCCF8093C600319608
:100FD0008491F5CF8091520A8823A1F1EDE4F2E1EA
:100FE0008491882341F09091C00095FFFCCF8093BD
:100FF000C6003196F5CF8091C00085FFFCCF8AE016
:101000008093C600FE01C491ECEBFEE0CC2349F0D6
:101010008091C00085FFFCCFC093C6003196C4917B
:10102000F5CF409153025091540260915502709156
:10103000560283E492E10E94C43E8091C00085FF85
:10104000FCCF11C0E7E2F2E18491882341F0909156
:10105000C00095FFFCCF8093C6003196F5CF8091FC
:10106000C00085FFFCCF8AE08093C600DF91CF915E
:101070000895AF92BF92CF92DF92EF92FF920F93BB
:101080001F93CF93DF93CDB7DEB7E0970FB6F894F9
:10109000DEBF0FBECDBF80E1EFEEF2E0DE01919644
:1010A00001900D928A95E1F780E1EFEFF2E0DE0129
:1010B000519601900D928A95E1F780E1EFE0F3E01F
:1010C000DE01119601900D928A95E1F76E0181E2A1
:1010D000C80ED11C8FE9E82E83E1F82E8E010F5E39
:1010E0001F4F6FEA73E1AE014F5F5F4F9FE8A92E7C
:1010F00093E1B92E20E030E0F60181919191A19128
:10110000B1916F01F70181939193A193B1937F0105
:10111000F80181919191A191B1918F01FB0181938E
:101120009193A193B193BF01FA0181919191A19102
:10113000B191AF01F50181939193A193B1935F01B7
:101140002F5F3F4F24303105B9F60E94E8A580E0BB
:1011500090E8ABE3B5E48093871390938813A09352
:101160008913B0938A138093831390938413A0936D
:101170008513B093861310928B1310928C131092D8
:101180008D1310928E1380E29EE4A0E0B0E0809375
:10119000BF139093C013A093C113B093C2131092C6
:1011A000731310927413109275131092761380E0DB
:1011B00090E0A0EAB1E480937F1390938013A09312
:1011C0008113B09382138DEC9CECACECBEE3809366
:1011D0007B1390937C13A0937D13B0937E1380E0D8
:1011E00090E0A0EAB0E48093771390937813A093F3
:1011F0007913B0937A1310923E0A10923F0A10921C
:10120000400A1092410A10923A0A10923B0A109238
:101210003C0A10923D0A1092360A1092370A109238
:10122000380A1092390A82ED90E09093960D8093DF
:10123000950D82E390E09093940D8093930D10921E
:10124000920D1092910D8FEF90E09093900D8093FE
:101250008F0D84E690E090938E0D80938D0D10920B
:101260008C0D10928B0D83E393EBA3E2B2E4809399
:10127000180290931902A0931A02B0931B0260E027
:1012800070E08CE990E40E9432286093140270931D
:101290001502809316029093170265E87BE28CEAB0
:1012A00092E40E943E286093100270931102809392
:1012B0001202909313020E94A01E80E090E0A0E82A
:1012C000BFE380930C0290930D02A0930E02B093A3
:1012D0000F0210922B0A80E090E0A0E4B0E480932B
:1012E000330290933402A0933502B093360240E06B
:1012F00050E064E372E440932B0250932C0260931D
:101300002D0270932E021092260A1092270A109234
:10131000280A1092290A1092220A1092230A109287
:10132000240A1092250A40E050E060E071E4409306
:101330002702509328026093290270932A02109288
:10134000520A8093530290935402A0935502B09393
:1013500056020E94CF4BECEBFEE08491882341F0D3
:101360009091C00095FFFCCF8093C6003196F5CFD9
:10137000E5E0F2E18491882341F09091C00095FF6F
:10138000FCCF8093C6003196F5CF8091C00085FFD9
:10139000FCCF8AE08093C600E0960FB6F894DEBFDB
:1013A0000FBECDBFDF91CF911F910F91FF90EF90B6
:1013B000DF90CF90BF90AF9008951F920F920FB61D
:1013C0000F9211240BB60F922F933F934F935F937D
:1013D0006F938F939F93EF93FF936091C60020913B
:1013E0001B0E30911C0EC90101968F7799274091F1
:1013F0001D0E50911E0E8417950741F0F901E55618
:10140000F24F608390931C0E80931B0EFF91EF911F
:101410009F918F916F915F914F913F912F910F907D
:101420000BBE0F900FBE0F901F9018959A01AB0145
:10143000211581EE38074105510549F182E080937D
:10144000C00060E079E08DE390E00E9478B3215025
:10145000310941095109CA01B90122E030E040E0F7
:1014600050E00E9478B33093C5002093C40080916F
:10147000C10080618093C1008091C1008860809329
:10148000C1008091C10080688093C10008951092CE
:10149000C00020E130E0E7CF20911D0E30911E0EFC
:1014A00080911B0E90911C0E8217930771F0F90129
:1014B000E556F24F80812F5F3F4F2F7733273093D0
:1014C0001E0E20931D0E90E008958FEF9FEF08955C
:1014D00080911D0E90911E0E90931C0E80931B0EFA
:1014E00008954F925F926F927F928F929F92AF92E8
:1014F000BF92CF92DF92EF92FF920F931F93CF9301
:10150000DF93CDB7DEB7A0970FB6F894DEBF0FBE5E
:10151000CDBF5C014115510561057105E9F420E07D
:1015200030E040E350E060E070E0A0960FB6F89441
:10153000DEBF0FBECDBFDF91CF911F910F91FF9006
:10154000EF90DF90CF90BF90AF909F908F907F9063
:101550006F905F904F905BC08E010F5F1F4FC12C4B
:10156000D12C76014801422E512C612C712C8FEF29
:10157000C81AD80AE80AF80ACB01BA01A3019201F5
:101580000E9456B3CA01F80161938F01A901BC0101
:10159000411551056105710551F7F1E0CF1AD108E8
:1015A000E108F108F401EC0DFD1D80818A3010F492
:1015B00040E301C047E3480F552747FD5095652F8D
:1015C000752F20E030E0C50122D081E0C81AD10893
:1015D000E108F108EFEFCE16DE06EE06FE0611F783
:1015E000A0960FB6F894DEBF0FBECDBFDF91CF91AE
:1015F0001F910F91FF90EF90DF90CF90BF90AF9031
:101600009F908F907F906F905F904F9008952115DD
:10161000310539F48091C00085FFFCCF4093C600AE
:1016200008952A30310509F424C05BCF9A01462F72
:10163000552747FD5095652F752FE9CFCF93DF9341
:10164000EC0120E030E04DE050E060E070E0DFDFF2
:1016500020E030E04AE050E060E070E0CE01DF9151
:10166000CF91D5CF9A01AB01662757FD6095762FB4
:10167000CECFCF92DF92EF92FF92CF93DF93EC0128
:101680006A017B0177FF0FC020E030E04DE250E0BF
:1016900060E070E0BCDFF094E094D094C094C11C92
:1016A000D11CE11CF11C2AE0B701A601CE01DF919B
:1016B000CF91FF90EF90DF90CF9013CF21153105A0
:1016C00039F48091C00085FFFCCF4093C600089597
:1016D00008CF9A01462F50E060E070E0EFCFCF9343
:1016E000DF93EC019A01AB0160E070E0E7DFCE012F
:1016F000DF91CF91A3CF8F929F92AF92BF92CF9263
:10170000DF92EF92FF921F93CF93DF93EC016A0178
:101710007B01122F20E030E0A901C701B6010E9431
:1017200078AF87FF0CC020E030E04DE250E060E091
:1017300070E0CE016CDFF7FAF094F7F8F094B12C7A
:1017400060E070E080E09FE3B11641F020E030E01F
:1017500040E251E40E947FAFB394F6CF9B01AC010D
:10176000C701B6010E949FAE6B017C010E94ECAFE5
:101770004B015C010E9418B09B01AC01C701B6018E
:101780000E949EAE6B017C012AE0B501A401CE014E
:10179000A8DE112361F0EFE5F3E08191882339F0B1
:1017A0009091C00095FFFCCF8093C600F6CF112327
:1017B00019F120E030E040E251E4C701B6010E9497
:1017C0004DB26B017C010E94E7AF4B01AA2497FC4C
:1017D000A094BA2CB501A401CE014BDFC501B40120
:1017E0000E941AB09B01AC01C701B6010E949EAED7
:1017F0006B017C011150DBCFDF91CF911F91FF90E6
:10180000EF90DF90CF90BF90AF909F908F90089512
:1018100072CFCF93DF931F92CDB7DEB7698341E0DC
:1018200050E0BE016F5F7F4F04960E94FC160F9040
:10183000DF91CF910895FB0101900020E9F7AF01FE
:1018400041505109461B570B04960C94FC1680918D
:10185000370E811109C08091360E811105C080912B
:10186000350E811101C00895ECEBFEE084918823D0
:1018700041F09091C00095FFFCCF8093C600319657
:10188000F5CFE4E6F5E18491882341F09091C00022
:1018900095FFFCCF8093C6003196F5CF8091370E2F
:1018A0008823F1F06091380E7091390E80913A0ED4
:1018B00090913B0E0E941AB020919F133091A0137B
:1018C0004091A1135091A2130E947FAFAB01BC01C4
:1018D00080E695E10E94C43E80E595E10E94D776BE
:1018E0008091360E8823F1F060913C0E70913D0E90
:1018F00080913E0E90913F0E0E941AB02091A3134A
:101900003091A4134091A5135091A6130E947FAF6C
:10191000AB01BC018CE495E10E94C43E8CE395E1EF
:101920000E94D7768091350E8823F1F06091400EA9
:101930007091410E8091420E9091430E0E941AB018
:101940002091A7133091A8134091A9135091AA1385
:101950000E947FAFAB01BC0188E395E10E94C43EC9
:1019600088E295E10E94D7768091C00085FFFCCF88
:101970008AE08093C6001092370E1092360E1092B5
:10198000350E08951092370E1092360E1092350EC5
:10199000089580939B020895EFE6F0E080818260D5
:1019A000808308951F920F920FB60F9211240BB6E9
:1019B0000F920F931F932F933F934F935F936F93C8
:1019C0007F938F939F93AF93BF93EF93FF938091F8
:1019D000680E9091690E892B09F084C190916B0E6D
:1019E00080916A0E981771F0E0916A0E8DE4E89F7D
:1019F000F0011124E459F14FDF01A45BBF4F81E0F6
:101A00008C9302C0E0E0F0E0F093690EE093680E82
:101A1000309709F461C1DF01A45BBF4F81E08C9373
:101A200010924B0E10924C0E10924D0E10924E0EC4
:101A300060AD71AD61349CE9790728F461329EE4B0
:101A4000790748F002C060E47CE976956795769561
:101A5000679584E007C0613197E2790730F07695A9
:101A6000679582E08093480E07C08093480E6032ED
:101A7000710510F460E270E060527109611588E050
:101A80007807D0F0872F9927880F991F880F991F03
:101A90008D58964EFC01329645915491AA27659F28
:101AA0009001649F210D3A1F06942A1F3A1F1124AA
:101AB000FC01859194911DC0CB01969587958C7FF3
:101AC0008D589A4EFC01459154910296FC018591E6
:101AD0009491FB01E770FF278E9F90018F9F300D3F
:101AE0009E9F300D1124E3E036952795EA95E1F7A6
:101AF000CA01821B930B8436910598F4EBEBF5E059
:101B00008191882339F09091C00095FFFCCF80939C
:101B1000C600F6CF4AE050E08AE99DE0E0DD84E6C9
:101B200090E09093470E8093460E8091480E99273F
:101B300087FD90959093450E8093440EE091680E3A
:101B4000F091690E64AD75AD70934A0E6093490EC5
:101B500061349CE9790728F461328EE4780748F013
:101B600002C060E47CE9769567957695679584E098
:101B700007C0613197E2790730F07695679582E08A
:101B80008093480E08C081E08093480E6032710552
:101B900010F460E270E060527109611588E0780726
:101BA000E0F0872F9927880F991F880F991F8D586C
:101BB000964EFC01329625913491AA27639FA0018D
:101BC000629F410D5A1F06944A1F5A1F1124FC019F
:101BD00025913491241B350B1EC0CB01969587951A
:101BE0008C7F8D589A4EFC01259134910296FC0110
:101BF00045915491FB01E770FF274E9FC0014F9F15
:101C0000900D5E9F900D1124F3E096958795FA95BF
